:0800000C32342E312E302E3467
:0100000B01F3
:1000000AF63F3325F0261518FE2323012B2F04442F
:1000000A31202309272A0C1712151418161D1C173C
:1000000A5E52440F645761461E62573D185D696D22
:1000000A4C2742482A44482D373A363B3F3A3A3E33
:1000000A423D3A5D3F613268575A40806B6F44699E
:0400000A6F47876550
:020000040800F2
:4080000058ED00102D81040835810408A18D0408398104083B8104083D81040800000000000000000000000000000000158300084181040800000000CD830008318400085A
:40804000478104084781040847810408478104084781040847810408DD631408E7631408F1631408FB631408056414084781040847810408478104088D8E00084781040864
:4080800047810408478104081BE50008EFE80008F9E8000803E90008478104080F641408478104084781040847810408478104084781040847810408478104084781040851
:4080C000478104085F5F1408695F140847810408478104084781040847810408978E00083564140847810408478104084781040847810408478104084781040847810408F0
:408100004781040847810408478104084781040847810408478104086964140893761408F7E400080FE5000803E50008257414082F74140847810408478104080DE9000850
:4081400017E9000821E90008478104084781040847810408478104084781040847810408478104084781040847810408478104084781040847810408478104080000000021
:40818000478104084781040847810408478104084781040847810408478104084781040800000000000000004781040800F002F800F05AF80AA090E8000C82448344AAF1C9
:4081C0000107DA4501D100F04FF8AFF2090EBAE80F0013F0010F18BFFB1A43F001031847444E0A00844E0A0010F8013B0A4413F0030408BF10F8014B1D1108BF10F8015BC9
:40820000641E05D010F8016B641E01F8016BF9D1002D15D010F8014B03F00C030C2BA1EB04040ABF10F8013BA4EB8314A4EB032405F1010314F8016B5B1E01F8016BF9D588
:40824000914238BF10F8013BD1D370470023002400250026103A28BF78C1FBD8520728BF30C148BF0B6070478DF105F8114637F10FFF0FB400F00CF80FBC39F1DEFE8CF15F
:408280001DFA03B437F11EFF03BC40F041FC000004B08DF171FE044800218DF123FF8DF17DFE8CF10BFA0000E020001080F309887047EFF309807047684680F3098804486B
:4082C0000078C00714BF0220032080F31488704758BF1908DFF818C0EFF305831B0618BF6047EFF31483DB0708BF604700DF704745611908DFF818C0EFF305831B0618BF3A
:408300006047EFF31483DB0708BF604700DF7047FD960408EFF30980816911F8021CE1BB90E80F1010B5E047BDE81040EFF3098C8CE80700214B93E80600914208BF7047D8
:4083400041B91EF0100F16D11D49086820F00100086010E01EF0100F06BF2CED108A0120002081F825002CE9F00FC1F828C00CB441F0F8FC0CBC1A60D2F828C0BCE8F00FFB
:4083800092F8250000280EBF6FF0020E6FF0120EBCEC108A8CF30988704710B5094A1268914209D8084C54F8214090E80F10A047EFF3098C8CE80F0010BD0000FC2000106A
:4083C00034EF00E07C5A19087C5A190810B58DF1CDFFBDE81040154B93E80600914208BF7047EFF3098C1EF0100F06BF2CED108A0120002081F825002CE9F00FC1F828C0A6
:408400000CB441F0AFFC0CBC1A60D2F828C0BCE8F00F92F8250000280EBF6FF0020E6FF0120EBCEC108A8CF309887047FC20001010B541F04BFDCCE710B541F0E5F841F04D
:4084400045FDC6E740BA7047C0BA704770B505466FF07F40281A00D100BF0A2001F062FC002410E09FED180A204601F0C9FF9FED160A204601F0F1FF9FED130A204602F07D
:4084800015F8601CC4B2042CECDB9FED0F0A002002F00CF89FED0C0A002002F028F8002002F052F8012002F0F9F8012002F009F9012002F019F9002002F06CF8002002F015
:4084C0007BF900BF00BF70BD0000000010B5044600202070606838B1606818B1606802685168884700206060A06838B1A06818B1A0680268516888470020A060E06838B1B5
:40850000E06818B1E0680268516888470020E060206938B1206918B1206902685168884700202061606938B1606918B1606902685168884700206061A06938B1A06918B10C
:40854000A0690268516888470020A061E06938B1E06918B1E0690268516888470020E061206A38B1206A18B1206A02685168884700202062606A38B1606A18B1606A0268A1
:408580005168884700206062A06A38B1A06A18B1A06A0268516888470020A062E06A38B1E06A18B1E06A0268516888470020E062206B38B1206B18B1206B02685168884744
:4085C00000202063606B38B1606B18B1606B02685168884700206063A06B38B1A06B18B1A06B0268516888470020A063E06B38B1E06B18B1E06B0268516888470020E06320
:40860000206C38B1206C18B1206C02685168884700202064606C38B1606C18B1606C02685168884700206064A06C38B1A06C18B1A06C0268516888470020A064E06C38B141
:40864000E06C18B1E06C0268516888470020E064206D38B1206D18B1206D02685168884700202065606D38B1606D18B1606D02685168884700206065A06D38B1A06D18B197
:40868000A06D0268516888470020A065E06D38B1E06D18B1E06D0268516888470020E06510BD10B5044600206060A060E06020616061A061E06120626062A062E06220631B
:4086C0006063A063E06320646064A064E06420656065A065E0652046FFF7F8FE204610BD10B504462046FFF7F1FE204610BD2DE9F04704460F462046FFF7E8FE27702078DE
:4087000000287DD0012802D002287AD100E000BF0C2040F00FFD05460022522183F1C9F9054660600C2040F005FD05460022532183F1BFF90546A0600C2040F0FBFC0546D8
:408740000022542183F1B5F90546E0600C2040F0F1FC05460022552183F1ABF9054620610C2040F0E7FC05460022512183F1A1F905466061082040F0DDFC06463D2183F11E
:40878000CBF90646A062082040F0D4FC06463E2183F1C2F90646E062082040F0CBFC0646132183F1B9F906462063082040F0C2FC0646142183F1B0F9064660631C2040F054
:4087C000B9FC804601223F213DF022FC8046A0630C2040F0AFFC054600223B2183F169F90546E0630C2040F0A5FC054600223C2183F15FF905462064606C68B90C2001E0D7
:4088000061E061E040F096FC81460022242183F1D3F98146606400BFA06C50B90C2040F089FC814600221D2183F1C1F88146A06400BFE06C50B90C2040F07CFC8146002256
:408840001E2183F1B4F88146E06400BF206D50B90C2040F06FFC814600221C2183F1A7F88146206500BF606D50B90C2040F062FC81460122172183F19AF88146606500BF2B
:40888000A06D50B90C2040F055FC81460122182183F18DF88146A06500BF606D08B9A06D80B1E06D70B90C2040F044FC8146172183F100F88146E065E06D01688A6A01212D
:4088C000904700BF00E000BF00BFBDE8F08710B5044602F001FE10BD0146087870470246002053680B600B6803B1012070470246002093680B600B6803B10120704702467B
:408900000020D3680B600B6803B1012070470246002013690B600B6803B1012070470246002053690B600B6803B1012070470246002093690B600B6803B101207047024680
:408940000020D3690B600B6803B10120704702460020136A0B600B6803B10120704702460020536A0B600B6803B10120704702460020936A0B600B6803B10120704702463C
:408980000020D36A0B600B6803B10120704702460020136B0B600B6803B10120704702460020536B0B600B6803B10120704702460020936B0B600B6803B1012070470246F8
:4089C0000020D36B0B600B6803B10120704702460020136C0B600B6803B10120704702460020536C0B600B6803B10120704702460020936C0B600B6803B1012070470246B4
:408A00000020D36C0B600B6803B10120704702460020136D0B600B6803B10120704702460020536D0B600B6803B10120704702460020936D0B600B6803B10120704710B5F2
:408A40000448FFF72EFE0446034AAFF26B313FF0EDFC10BD140400200080000870470146B1F1006F04D3B1F1026F01D8012070470020FCE70146B1F1805F02D39D4881421D
:408A800005D9B1F1005F04D39B48814201D8012070470020FCE70146002070470146974A974800681318914203D3994201D8012070470020FCE770B5044600252046FFF7C6
:408AC000EDFF08B1032510E02046FFF7E4FF08B104250AE02046FFF7CDFF08B1022504E02046FFF7BCFF00B10125284670BD01460020844A1288914202D2834A52F821008B
:408B0000704730B5002500240AE02046FFF7EFFF034623B15878022801D11D4604E0641C784800888442F0D3284630BD70B5FFF7E8FF04460025FF22C82174488BF182FE0D
:408B4000681E73490860002C3DD0206B0860E08C002838D0E08C0121C1EB900631E0E16A51F82600FFF7A7FF052828D2DFE800F026030D0E0F00322D06D2E06A50F826002C
:408B8000624941F825006D1C19E000BF17E0322D13D212D2E16A51F826100868FFF78BFF052809D2DFE800F004030506070003E000BF00BF00BF00BF00BF00E000BF00BFBE
:408BC000761E002ECBD15348007840B10020514908702A464D494E480068FFF73FFF70BD10B5FFF7A3FF10BD10B504462046FFF755FF10BD10B50446002010BD10B50446BB
:408C00002046FFF774FF0346DFED430AB0EE600A1BB3D88C08B304201CE0D96A095CCC2917D0D98C00EE901AB8EE601A00EE900AF8EE600A71EE600A9FED381A20EE811A25
:408C400000EE901AF8EE600AC1EE201AB0EE610A03E0401CD98C8142DFD810BD10B504462046FFF744FF0346DFED2B0AB0EE600AE3B1D88CD0B1D98CD86A0844996A8842F6
:408C800014D3D3E90A01401AD98C081A00EE900AF8EE600A9FED211A20EE811A00EE901AF8EE600AC1EE201AB0EE610A10BD30B50025002408E02046FFF719FF034613B19F
:408CC000587800B16D1C641C0E4800888442F2D3284630BD0B48008870477047704710B50F48FFF7FAFF04460E4AAFF20F013FF09DFB10BD0000011000000320504302204B
:408D000074BF190840BF190814B7022008210010080000100C000010000000000000C8420400001000800008B0EE402AF0EE602AB4EEE11AF1EE10FA01D2B0EE611AB5EE3A
:408D4000C01AF1EE10FA02D0C1EE810A01E0F7EE000A20EE823AF7EE003A73EEE03AB0EE430A03EEA20A70470246B4EEE00AF1EE10FA01D2B0EE600AB5EEC00AF1EE10FAC3
:408D800002D080EE801A01E0B7EE001A01EE902AF8EEE11A21EE212AF7EE001A71EEC12A01EE901AF8EEE11A02EEA12AFDEEC21A11EE900A7047000010B5002807DA0A07E1
:408DC000140E7B4A00F00F031B1FD45403E00A07130E784A135410BD774A0168116001791171704710B57548754908604FF4E13048604FF44071724881610C2141610021AB
:408E00000161C1608160C1613EF069F96D486E4908604FF00060486040216B4881600021C1604FF480610161002141618161C1614FF40031016200214162032181624FF498
:408E40000001C162891001633DF0AEFB00BF5E485B49086308465C49886300BF00210E20FFF7AAFF0E2000F097F80D212720FFF7A3FF272000F090F80122544950483EF0FD
:408E80008FFB10B101205249087010BD10B54E483DF0E1FD10BD10B549483EF0EAFF10BD10B50122494946483EF07AFB044614B1012047490870204610BD10B50446454847
:408EC0000078012826D1002007E0434909880144424A515C1154411C88B2414909883E4A1288891A8142F0DC3D4800883A490988401A3B4908800020374908803848008816
:408F0000C0F180020021354880308BF19BFC0020304908702D480178314802880088401C2F4B18802D48815418460088802802DB0020194608803AF13CF91B2805D02949FF
:408F4000886F032140F01CFB05E02649D1F88000022140F015FB01221C4919483EF020FB10B101201A49087010BD704710B504461D4839F129FF022804DB1A49886F0221D0
:408F800040F0FEFA10BD70B504460D462A4621460B483EF09EFB70BD00F01F02012191404209920002F1E022C2F800117047000018ED00E000E400E04013002000480040E0
:408FC000A012002058600240E0120020890000208A0000201A010020160100206013002014010020B0090020D023001000487047E4E700103DF029BAFFFFFFFFFFFFFFFF48
:409000008CF1CAB910B50446F94800688047E060002020746074A074E07420756075206881682046884710BD10B50446204622F0F9F90446EF4820602046FFF7E3FF204686
:4090400010BD10B50446204622F0F2F90446204610BD70B504462046FFF7F3FF054640F061F870BD70B50546012406E0E24B00222146284622F08CFA641C202CF6D370BD7D
:4090800001460020DD4A12680A600A6802B10120704710B5D948006848B9182040F04AF80446FFF7C1FF0446D448046000BF10BD10B5D248006870B1D048006830B1CF4812
:4090C000006800684168CD48006888470020CB4908603BF0EFFA10BD3EB5002000900190029068468BF14AFBC4B22146684600F073FE002000F08FFEC14800F09FFE0120B9
:4091000000F0AFFE012000F0BFFE002000F0CFFE002000F0DFFE002000F0EFFE002000F0FFFE002000F00FFF002000F029FFB54800F038FFB44800F048FFB44800F058FF00
:40914000B34800F068FF002000F0D6FF002000F0E6FF002000F0F6FF002001F006F8002001F016F8002001F026F8002001F036F8002001F0DFFAFA2000F060FF4FF4FA6032
:4091800000F06FFF41F2707000F07DFF40F27E3000F08CFF40F6F85000F09BFF3EBD0146487D70470146087C704710B5044600F0A2FD10BD2DE9F04107460C46154600265D
:4091C00000F099FDA04208D0204600F098FD2B4632460321384622F0DBF93046BDE8F08110B5044600F0F5FD10BD2DE9F04707460D4614469846002600F0EBFD8146142C5F
:4092000001DA204600E014200246294648463FF040F948B12146284600F0DEFD434632460421384622F0B4F93046BDE8F08710B5044600F0ECFD10BD2DE9F04107460C4603
:409240001546002600F0E3FDA04208D0204600F0E2FD2B4632460521384622F099F93046BDE8F08110B5044600F0E4FD10BD2DE9F04107460C461546002600F0DBFDA04233
:4092800008D0204600F0DAFD2B4632460621384622F07EF93046BDE8F08110B5044600F0DCFD10BD2DE9F04107460C461546002600F0D3FDA04208D0204600F0D2FD2B46EA
:4092C00032460721384622F063F93046BDE8F08110B5044601F02AFA10BD2DE9F04107460C46154600263846FFF7F2FFA04208D0204601F01FFA2B4632460821384622F0CD
:4093000047F93046BDE8F08110B5044600F0B8FD10BD2DE9F04107460C461546002600F076FEA04208D0204600F075FE2B4632461321384622F02CF93046BDE8F0812DE91E
:40934000F04107460C461546002600F04DFEA04208D0204600F04CFE2B4632461221384622F016F93046BDE8F0812DE9F04107460C461546002600F024FEA04208D0204627
:4093800000F023FE2B4632461121384622F000F93046BDE8F0812DE9F04107460C461546002600F0FBFDA04208D0204600F0FAFD2B4632461021384622F0EAF83046BDE86F
:4093C000F0812DE9F04107460C461546002600F0C9FDA04208D0204600F0D2FD2B4632460F21384622F0D4F83046BDE8F08100002803002074C60A08A38F0408000000101A
:40940000E4D914013A9B220089C31400C5610A00EC7503002DE9F04107460C461546002600F08DFDA04208D0204600F08CFD2B4632460E21384622F0ABF83046BDE8F0811E
:409440002DE9F04107460C461546002600F064FDA04208D0204600F063FD2B4632460D21384622F095F83046BDE8F0812DE9F04107460C461546002600F03BFDA04208D0BB
:40948000204600F03AFD2B4632460C21384622F07FF83046BDE8F0812DE9F04107460C461546002600F0FFFCA04230D0204600F0FEFC2A4600213846FFF7D8FF2A46002185
:4094C0003846FFF7BDFF2A4600213846FFF7A2FF2A4600213846FFF774FF2A46FC493846FFF759FF2A46FB493846FFF73EFF2A46F9493846FFF723FF2A46F8493846FFF7CB
:4095000008FF2B4632460A21384622F041F83046BDE8F0812DE9F04107460C461546002600F0AEFCA0420DD0204600F0ADFC2A4600213846FFF7B0FF2B46324609213846B7
:4095400022F026F83046BDE8F08110B5044600F0AAFC10BD10B5044600F0B8FC10BD2DE9F04107460C461546002600F0AFFCA04208D0204600F0AEFC2B4632460B213846EE
:4095800022F006F83046BDE8F08110B5044600F0B0FC10BD10B5044600F0BEFC10BD10B5044600F0CCFC10BD10B5044600F0DAFC10BD10B5044600F0F1FC10BD10B5044613
:4095C00000F0FFFC10BD10B5044600F00DFD10BD10B5044600F01BFD10BD10B5044600F029FD10BD2DE9F04107460C461546002600F020FDA04208D0204600F01FFD2B46F6
:4096000032461421384621F0C3FF3046BDE8F08110B5044600F021FD10BD2DE9F04107460C461546002600F018FDA04208D0204600F017FD2B4632461521384621F0A8FFD1
:409640003046BDE8F08110B5044600F018FD10BD2DE9F04107460C461546002600F00FFDA04208D0204600F00EFD2B4632461621384621F08DFF3046BDE8F08110B5044629
:4096800000F010FD10BD2DE9F04107460C461546002600F007FDA04208D0204600F006FD2B4632461721384621F072FF3046BDE8F08110B5044600F008FD10BD2DE9F041AD
:4096C00007460C461546002600F0FFFCA04208D0204600F0FEFC2B4632461821384621F057FF3046BDE8F08110B5044600F000FD10BD2DE9F04107460C461546002600F0A2
:40970000F7FCA04208D0204600F0F6FC2B4632461921384621F03CFF3046BDE8F08110B5044600F0F8FC10BD2DE9F04107460C461546002600F0EFFCA04208D0204600F0A9
:40974000EEFC2B4632461A21384621F021FF3046BDE8F08110B5044600F0F0FC10BD2DE9F04107460C461546002600F0E7FCA04208D0204600F0E6FC2B4632461B21384619
:4097800021F006FF3046BDE8F08110B5044600F0E8FC10BD2DE9F04107460C461546002600F0DFFCA04208D0204600F0DEFC2B4632461C21384621F0EBFE3046BDE8F08111
:4097C00010B5044600F0E0FC10BD2DE9F04107460C461546002600F0D7FCA04208D0204600F0D6FC2B4632461D21384621F0D0FE3046BDE8F08110B5044600F0D8FC10BD05
:409800002DE9F04107460C461546002600F0CFFCA04208D0204600F0CEFC2B4632461E21384621F0B5FE3046BDE8F08110B5044600F0D0FC10BD2DE9F04107460C4615465D
:40984000002600F0C7FCA04208D0204600F0C6FC2B4632461F21384621F09AFE3046BDE8F08101214174704700B502461046FFF796FC08B10120907400BD0121C17470474F
:4098800001210175704770B504460D46607DA84206D06575124B00220121204621F078FE70BD70B504460D46207CA8420ED000212046FFF7E8FF25740A4800688047E06081
:4098C000074B00220221204621F062FE70BD00003A9B220089C31400C5610A00EC750300A38F04082803002070B504462046FFF759FC09287ED2DFE800F0050C264E6C9E72
:40990000E9F6F500FFF7E8FB01212046FFF7C9FF22E12046FFF764FC0546142298A13EF0B8FD20B101212046FFF7ADFF03E000212046FFF7A8FFA07C012803D10221204634
:40994000FFF7AFFF08E12046FFF771FC78B12046FFF788FC58B12046FFF79FFC38B100F0E5FE20B101212046FFF78DFF03E000212046FFF788FFA07C012804D10321204666
:40998000FFF78FFF06E0607C012803D101212046FFF787FFE0E001212046FFF774FFA07C01280ED12046FFF7D0FD012804D104212046FFF776FF0BE006212046FFF771FF90
:4099C00006E0607C012803D102212046FFF769FFC2E02046FFF7D9FD90B12046FFF7DAFD70B12046FFF7DBFD50B12046FFF7DCFD30B100E0ABE001212046FFF744FF03E0FE
:409A000000212046FFF73FFF2046FFF79EFD10B92046FFF729FFA07C012804D105212046FFF73FFF06E0607C012803D103212046FFF737FF90E02046FFF7BBFD58B32046E3
:409A4000FFF7BCFD38B32046FFF7BDFD18B32046FFF7BEFDF8B12046FFF7ABFD05462046FFF7ACFD854216D32046FFF7A7FD05462046FFF7A8FD85420DD32046FFF7A3FDB8
:409A800005462046FFF7A4FD854204D301212046FFF7F9FE03E000212046FFF7F4FE2046FFF753FD10B92046FFF7DEFEA07C012804D106212046FFF7F4FE06E0607C0128D2
:409AC00003D104212046FFF7ECFE45E001212046FFF7D9FEA07C012806D107212046FFF7E0FE12E032E011E0607C01280DD12046FFF72BFD012804D105212046FFF7D1FE84
:409B000003E003212046FFF7CCFE25E001212046FFF7B9FEA07C012810D108212046FFF7C0FE36F120FE00220121164848F1ABFF154A01212046FFF73DFB06E0607C01288B
:409B400003D106212046FFF7ACFE05E004E008212046FFF7A6FE00BF00BF00206074A074E074207570BD10B504462046FFF7BCFE2046FFF717FB082801D1FFF799FA10BD6B
:409B80000000000064390010A38F0408F74890F8A001704710B5044600BFF44880F8A041012200F5D071F24800F01AFE00BF10BDEE4901F5D47103C9704770B504460D465A
:409BC00000BFEA4800F5D47030C00822E949E848083000F005FE00BF70BDE748704710B5044600BFE148C0F8B041042200F5D871DF48103000F0F4FD00BF10BDDB4840681F
:409C0000704710B5044600BFD84844600422011DDA4800F0E5FD00BF10BDD4480068704710B5044600BFD1480460042201464FF0D04000F0D5FD00BF10BDCC4880687047D4
:409C400010B5044600BFC9488460042200F10801CA48001D00F0C4FD00BF10BDC348D0F8BC01704770B506460D46FFF7F7FF0446012E0CD12C4300BFBC48C0F8BC4104223B
:409C800000F5DE71BA481C3000F0AAFD0CE0AC4300BFB648C0F8BC41042200F5DE71B4481C3000F09DFD00BF70BDB048D0F8DC01704710B5044600BFAC48C0F8DC410422F5
:409CC00000F5EE71AA48743000F08AFD00BF10BDA64890F8C801704710B5044600BFA34880F8C841012200F5E471A148603000F077FD00BF10BD9D4890F8E001704710B5A7
:409D0000044600BF994880F8E041012200F5F0719748783000F064FD00BF10BD934890F8E101704710B5044600BF904880F8E141012200F2E1118E48793000F051FD00BF04
:409D400010BD8A4890ED740A704710B52DED028BB0EE408A00BF854880ED748A042200F5E8718348683000F03BFD00BFBDEC028B10BD7E4890ED750A704710B52DED028B21
:409D8000B0EE408A00BF794880ED758A042200F5EA7177486C3000F023FD00BFBDEC028B10BD724890ED760A704710B52DED028BB0EE408A00BF6D4880ED768A042200F56E
:409DC000EC716B48703000F00BFD00BFBDEC028B10BD68483A30704770B504460D46142164483A303EF0D2FB142D01DA284600E01420024621465F483A303EF010FC142252
:409E00005C493A315A487A3000F0EAFC70BD5748D0F8F801704710B5044600BF5348C0F8F841042200F5FC715148903000F0D8FC00BF10BD4D48D0F8FC01704710B5044601
:409E400000BF4A48C0F8FC41042200F5FE714848943000F0C5FC00BF10BD444890F80002704710B5044600BF404880F80042012200F500713E48983000F0B2FC00BF10BDA3
:409E80003A4890F80102704710B5044600BF374880F80142012200F201213548993000F09FFC00BF10BD314890F80202704710B5044600BF2D4880F80242012200F202214F
:409EC0002B489A3000F08CFC00BF10BD274890F80302704710B5044600BF244880F80342012200F2032122489B3000F079FC00BF10BD1E48B0F80402704710B5044600BF7F
:409F00001A48A0F80442022200F5017118489C3000F066FC00BF10BD1448B0F80602704710B5044600BF1148A0F80642022200F206210F489E3000F053FC00BF10BD0B4802
:409F4000B0F80802704710B5044600BF0748A0F80842022200F502710548A03000F040FC00BF10BD0148B0F80A02704778040020A001006820060020C0D401000400006878
:409F800010B5044600BFFC48A0F80A42022200F20A21FA4800F024FC00BF10BDF648D0F8F802704710B5044600BFF348C0F8F842042200F53E71F148EE3000F011FC00BFFD
:409FC00010BDED48D0F8FC02704710B5044600BFE948C0F8FC42042200F53F71E748F23000F0FEFB00BF10BDE348D0F80003704710B5044600BFE048C0F80043042200F5A3
:40A000004071DE48F63000F0EBFB00BF10BDDA48D0F80403704710B5044600BFD648C0F80443042200F54171D448FA3000F0D8FB00BF10BDD048D0F80803704710B504461B
:40A0400000BFCD48C0F80843042200F54271CB48FE3000F0C5FB00BF10BDC748D0F80C03704710B5044600BFC348C0F80C43042200F54371C24800F0B3FB00BF10BDBE4838
:40A08000D0F81003704710B5044600BFBA48C0F81043042200F54471B948001D00F0A0FB00BF10BDB448D0F81403704710B5044600BFB148C0F81443042200F54571B048FD
:40A0C000083000F08DFB00BF10BDAB48D0F81803704710B5044600BFA748C0F81843042200F54671A6480C3000F07AFB00BF10BDA14890F80C02704710B5044600BF9E48F0
:40A1000080F80C42012200F503719C48801C00F067FB00BF10BD984890F80D02704710B5044600BF944880F80D42012200F20D219248C01C00F054FB00BF10BD8E4890F8AE
:40A140000E02704710B5044600BF8B4880F80E42012200F20E218948001D00F041FB00BF10BD854890F80F02704710B5044600BF814880F80F42012200F20F217F48401DDF
:40A1800000F02EFB00BF10BD7B48B0F81002704710B5044600BF7848A0F81042022200F504717648801D00F01BFB00BF10BD724890F81202704710B5044600BF6E4880F8CA
:40A1C0001242012200F212216C48083000F008FB00BF10BD684890F81302704710B5044600BF654880F81342012200F213216348093000F0F5FA00BF10BD5F48D0F81402EF
:40A20000704710B5044600BF5B48C0F81442042200F5057159480A3000F0E2FA00BF10BD5548D0F81802704710B5044600BF5248C0F81842042200F5067150480E3000F01C
:40A24000CFFA00BF10BD4C48D0F81C02704710B5044600BF4848C0F81C42042200F507714648123000F0BCFA00BF10BD4248D0F82002704710B5044600BF3F48C0F82042B5
:40A28000042200F508713D48163000F0A9FA00BF10BD3948D0F82402704710B5044600BF3548C0F82442042200F5097133481A3000F096FA00BF10BD2F48D0F8280270470B
:40A2C00010B5044600BF2C48C0F82842042200F50A712A481E3000F083FA00BF10BD2648D0F82C02704710B5044600BF2248C0F82C42042200F50B712048223000F070FA87
:40A3000000BF10BD1C48D0F83002704710B5044600BF1948C0F83042042200F50C711748263000F05DFA00BF10BD1348D0F83402704710B5044600BF0F48C0F8344204227A
:40A3400000F50D710D482A3000F04AFA00BF10BD0948D0F83802704710B5044600BF0648C0F83842042200F50E7104482E3000F037FA00BF10BD000078040020420200686A
:40A3800044030068FC48D0F83C02704710B5044600BFF948C0F83C42042200F50F71F74800F01EFA00BF10BD01460020042902DAF34A52F82100704770B504460D46042C79
:40A3C0000EDA00BFEE4840F82450EC4A121D02EB8400EB4A02EB8401042200F001FA00BF70BDDFEDE80AB0EE600A042807DAE449103101EB8001D1ED000AB0EE600A704725
:40A4000010B52DED028B0446B0EE408A042C12DA00BFDB48103000EB840080ED008AD74A143202EB8400D64A103202EB8401042200F0D6F900BFBDEC028B10BDDFEDD10A60
:40A44000B0EE600A042807DACD49203101EB8001D1ED000AB0EE600A704710B52DED028B0446B0EE408A042C12DA00BFC448203000EB840080ED008AC04A243202EB8400E0
:40A48000BF4A203202EB8401042200F0A9F900BFBDEC028B10BDDFEDBB0AB0EE600A20B9B549D1ED9C0AB0EE600A704710B52DED028B0446B0EE408A5CB900BFAE4880ED6D
:40A4C0009C8A042200F51C71AC48343000F088F900BFBDEC028B10BDDFEDAA0AB0EE600A20B9A549D1ED9D0AB0EE600A704710B52DED028B0446B0EE408A5CB900BF9E48B8
:40A5000080ED9D8A042200F51D719C48383000F067F900BFBDEC028B10BD9748D0F87802704710B5044600BF9348C0F87842042200F51E7191483C3000F052F900BF10BDD7
:40A540008D4890F87C02704710B5044600BF8A4880F87C42012200F51F718848403000F03FF900BF10BD8448D0F88002704710B5044600BF8048C0F88042042200F520714E
:40A580007E48443000F02CF900BF10BD7A48D0F8F402704710B5044600BF7748C0F8F442042200F53D717548B83000F019F900BF10BD7148D0F83803704710B5044600BFD1
:40A5C0006D48C0F83843042200F54E716E4800F007F900BF10BD6848D0F83C03704710B5044600BF6448C0F83C43042200F54F716548001D00F0F4F800BF10BD5E48D0F8CD
:40A600004003704710B5044600BF5B48C0F84043042200F550715C48083000F0E1F800BF10BD5548D0F84403704710B5044600BF5148C0F84443042200F5517152480C30AB
:40A6400000F0CEF800BF10BD4B48D0F84803704710B5044600BF4848C0F84843042200F552714948103000F0BBF800BF10BD4248D0F84C03704710B5044600BF3E48C0F858
:40A680004C43042200F553713F48143000F0A8F800BF10BD384890F88402704710B5044600BF354880F88442012200F521713348483000F095F800BF10BD2F4890F885024B
:40A6C000704710B5044600BF2B4880F88542012200F285212948493000F082F800BF10BD254890F88602704710B5044600BF224880F88642012200F2862120484A3000F04E
:40A700006FF800BF10BD1C48B0F8CC01704710B5044600BF1848A0F8CC41022200F5E6711648703800F05CF800BF10BD124890F8F002704710B5044600BF0F4880F8F04223
:40A74000012200F53C710D48B43000F049F800BF10BD0948D0F81C03704710B5044600BF0548C0F81C43042200F547710348E03000F036F800BF10BD7804002074020068AB
:40A78000B806002000000000107500681248D0F82003704710B5044600BF0F48C0F82043042200F548710D4800F01AF800BF10BD094890F82403704710B5044600BF064808
:40A7C00080F82443012200F549710448001D00F007F800BF10BD000078040020580300682DE9F04104460F4615460026FE4884420ED36019401EFD49884209D8FA48211ACC
:40A800002A4638463CF13AFA00B915E0202613E0B4F1D04F0FD36019401EF54988420AD8A4F1D0412A4638463CF190FC08B9002602E0202600E0082626B1EE480088304309
:40A84000EC4908803046BDE8F08110B50024FFF75AFF032800D10124204610BD2DE9F04107460C4615460026DF4884420ED36019401EDE49884209D8DB48211A2A463846D9
:40A880003CF12AFA00B924E0202622E0B4F1D04F0FD36019401ED64988420AD8A4F1D0412A4638463CF1F4FC08B9002611E020260FE0B4F1006F0BD36019401ECE49884292
:40A8C00006D82A462146384689F177FF002600E0082626B1C74800883043C64908803046BDE8F0812DE9FE4F06468946174698460020009083464FF480720023384641466E
:40A9000089F19DFC05464FF4807200233846414689F195FC924615B9BAF1000F2AD0ADB1002411E006EB0420029009EB042001904FF48072DDE90110FFF790FF009000987B
:40A940004BEA000B601CC4B2AC42EBD3BAF1000F12D006EB0520029009EB052001901FFA8AF2DDE90110FFF779FF009000984BEA000B01E04FF0400B5846BDE8FE8F2DE978
:40A98000FE4F06468946174698460020009083464FF4807200233846414689F150FC05464FF4807200233846414689F148FC924615B9BAF1000F2AD0ADB1002411E006EB34
:40A9C0000420029009EB042001904FF48072DDE90110FFF705FF009000984BEA000B601CC4B2AC42EBD3BAF1000F12D006EB0520029009EB052001901FFA8AF2DDE9011092
:40AA0000FFF7EEFE009000984BEA000B01E04FF0400B5846BDE8FE8FFEB5002001900090002600274FF45E7174483DF0D1FDEC200290012202A97248FFF7D2FE68B900205A
:40AA4000029001226E4902A8FFF708FF28B99DF80800EC2801D1781CC7B212200290012202A96748FFF7BCFE68B9002002900122634902A8FFF7F2FE28B99DF80800122877
:40AA800001D1781CC7B2022F07D05A48008840F08000584908800124D7E00122594901A8FFF7DCFE08B9701CC6B201225549491C6846FFF7D3FE08B9701CC6B2022E07D165
:40AAC0009DF80400012803D19DF80000122831D04FF4E47149483DF07BFD4FF4E472002346494FF0D040FFF74AFF4FF4B072002345494348DC30FFF742FF2822002343496C
:40AB00004348FFF73CFF28220023404928314148FFF735FF01200190012201A93948FFF75FFE12200090012269463648401CFFF757FE07E04FF4E47200234FF0D0412F48E1
:40AB4000FFF7D0FE02222E49DE312F48801CFFF785FE05462948B0F8CA01012800D10DB301244FF4B07128483DF032FD4FF4B072002325492248DC30FFF701FF28220023CE
:40AB8000224928312348FFF7FAFE00BF01211B48A0F8CA11022200F5E5711948DE30FFF71FFE0FE002244FF4B07200231449DC311548FFF797FE2822002316491348283062
:40ABC000FFF790FE022212491048FFF747FE05460A48B0F82803022800D15DB300BF02200649A1F8280317E000010168FF000169FF7F006810000010FF7F0F08780400204F
:40AC0000240100681B00006840060020A00700200075006800500068022201F54A716248FFF7DEFD00BF2822002360495E48FFF7A6FE05E0282200235B495C48FFF752FEFD
:40AC4000FFF703FE08B97EF18FFA2046FEBD7FB500200090019002900390012054490880544908703BF13AFC0020514908800846008800285BD1FFF7CFFE4F4908804F4BC3
:40AC80004FA20F2168463DF06BFB0025002408E04C48005D1DF80410884200D00125601C84B20F2CF4DB4448008801280DD10020404908700F22694642483DF035FC0F2236
:40ACC00040494148FFF78CFD35E0012D33D10020FEF7B6FFFFF7AEF910B9FA20FFF7AEF9FFF7BBF918B94FF4FA60FFF7BAF9FFF7C6F918B941F27070FFF7C5F9FFF7D2F9C6
:40AD000018B940F27E30FFF7D1F9FFF7DEF918B940F6F850FFF7DDF90F22694629483DF003FC0F2227492848FFF75AFD03E020480088214908807FBD1E48007870471E48E3
:40AD4000008870471C49098881431B4A1180704717480088704770B504460D4600261B4884420BD31A48854208D8184AA91AA01A3BF1C3FE00B902E0202600E0082626B105
:40AD80000B48008830430A490880304670BD10B50446012C03D10320FFF7B9FC02E00020FFF7B5FC10BD000000750068A007002010000010120000100E0000109CBE00080D
:40ADC00025730000840400200C00006800010168FF00016970472DE9F04104460D4617469846069EA0B2324629462FF0D6FB32462946204635F1C8FE33462A462146F9485F
:40AE000018F014FCBDE8F0812DE9F84305460C4616461F46DDF820800F2C3ED2DFE804F008162425262728292A2B2C2D2E3D3C00E0B23B463246002100902846FFF7CBFFF6
:40AE4000E2B2414628467EF17BFD2FE0E0B23B463246002100902846FFF7BDFFE2B2414628467EF16DFD21E000BF00BF00BF00BF00BF00BF00BF00BF00BF00BFE0B23B460B
:40AE80003246002100902846FFF7A5FFE2B2414628467EF155FD09E000BFE0B23B463246002100902846FFF796FF00BF00BFBDE8F88338B504460020034602460E210090F5
:40AEC0002046FFF7A1FF38BDC7480068704738B5044600200090694620461CF070F940B100980068C149C269009890471720FFF7E0FF38BDBE480068704710B50446FFF702
:40AF0000F9FFA04207D0BA4804601620FFF7D1FF2046FFF7DCFF10BDB6480068704710B50446FFF7F9FFA04207D0B24804601520FFF7BFFF0020FFF7E0FF10BD10B504460F
:40AF4000FFF7C2FFA04207D0A74804601420FFF7B0FF0020FFF7E3FF10BD10B51420FFF7A8FF10BD10B51520FFF7A3FF10BD10B51620FFF79EFF10BD9F480068704738B560
:40AF80000446FFF7F9FFA04215D09B48046000200090694620461DF008FB009820B19748009976F194FD02E0944876F1FFFB1820FFF77FFF00BF38BD91480068704710B561
:40AFC0000446FFF7F9FFA04204D08D4804601920FFF76FFF10BD10B51920FFF76AFF10BD88480068704710B50446FFF7F9FFA04204D0844804601A20FFF75BFF10BD10B5A8
:40B000001A20FFF756FF10BD7F480068704710B50446FFF7F9FFA04207D07B4804601B20FFF747FF0020FFF7CAFF10BD10B51B20FFF73FFF10BD75480068704710B50446EC
:40B04000FFF7F9FFA04204D0704804601C20FFF730FF10BD10B51C20FFF72BFF10BD6C480068704710B50446FFF7F9FFA04204D0674804601D20FFF71CFF10BD10B51D203E
:40B08000FFF717FF10BD63480068704710B50446FFF7F9FFA04204D05E4804601E20FFF708FF10BD10B51E20FFF703FF10BD5A480068704710B50446FFF7F9FFA04204D0EC
:40B0C000554804601F20FFF7F4FE10BD10B51F20FFF7EFFE10BD51480068704738B504464F4875F19FF8A0420DD0002000906946204619F06DFF4A48009975F161F9202000
:40B10000FFF7D7FE00BF38BD46480068704738B5044643484C381DF0A9FBA0420ED0002000906946204677F133FA3D484C3800991DF09BFE2120FFF7BCFE00BF38BD3A4863
:40B140000078704710B5044637480078A04204D0354804702220FFF7ACFE10BD3348704710B504462CB12068304982692046904703E014212D483DF009FA2320FFF799FE70
:40B1800010BD2B48704710B504462CB12068284982692046904703E0142125483DF0F6F92420FFF786FE10BD2248704710B504462CB120681F4982692046904703E0142122
:40B1C0001C483DF0E3F92520FFF773FE10BD1A48704710B504468CB32068174982692046904730E0D00100101800002040080020200000201C000020240000202C3A00102B
:40B20000280000202C0000203000002034000020380000203C0000204000002044000020803B0010480000204C000020F007002004080020180800202C080020FFE71421CD
:40B2400004483DF0A3F92620FFF733FE10BD0248704700002C08002040080020F8B50746002405E0804800EBC4000471601CC4B2152CF7DB7D488AF1F9FE7D4908607D48A4
:40B280008AF1F4FE7A4948607B488AF1EFFE78498860FFF7DCFC79480068804705460AE04A203AF1B6FC18B10A203EF0F1F802E03CF1DCF80546284620F0B5F9B0F5FA6F36
:40B2C000EED33BF18BF9FFF737FD10B90020FEF703FD43F1A3FA6A483EF03AF969490860002169488AF1FEFE5F49086507E064203EF0CEF8654800686430644908605A48BA
:40B3000090F855000B2805DA6048006842F210718842ECD301220021B5203AF146FD03F01FF935F1C5FA002159488AF1DBFE4E498861002157488AF1D5FE4B490861002197
:40B3400055488AF1CFFE48498860002153488AF1C9FE45490867002151488AF1C3FE4249886500214F488AF1BDFE3F49086600214D488AF1B7FE3C49886400214B488AF19C
:40B38000B1FE39490863002149488AF1ABFE36498862002147488AF1A5FE3349C1F89800002145488AF19EFE2F490862002143488AF198FE2C498867002141488AF192FE9A
:40B3C0002949C1F8800000213E488AF18BFE2649C1F890006846FDF753FE28B100213A488AF180FE20498866002138488AF17AFE1D49C1F8A000002088638AF18BFE0646D2
:40B400008AF194FEF8BD10B500211F488AF16AFE1549086510BD10B51348006C28B900212B488AF15FFE1049086410BD10B50E48D0F8880030B9002126488AF153FE0A4915
:40B44000C1F8880010BD10B50748006A50B1064890F82500032805D10349086A4FF400413EF08EF810BD0000B009002000991908580A0020049919080899190828030020A0
:40B480000C99190880000020F89919088400002038991908289919081899190848991908E8991908089A1908D8991908A8991908B8991908C8991908989919086899190867
:40B4C0005899190888991908289A1908389A1908189A19087899190810B53AF06EFF04462CB13AF162FE0020F749087002E00120F5490870204610BD2DE9F0472DED028B57
:40B500000446002720463AF07BFF00F0FF08B8F1560F79DA20688168204688471B2874D2DFE800F00E1420262C327338FD43494F555B736174B2C3D4FCFBFAF9F8F7F600F9
:40B54000002140463CF1D2FB07464CE1B8F1510F07DBB8F1550F04DC012140463CF1C6FB074640E1032140463CF1C0FB07463AE1042140463CF1BAFB074634E10121404643
:40B580003CF1B4FB07462EE1022140463CF1AEFB074628E1404643F14FFDB0F1FF3F01D0012000E0002007461DE10A2140463CF19DFB074617E1092140463CF197FB0746E5
:40B5C00011E10B2140463CF191FB07460BE1062140463CF18BFB074605E1072140463CF185FB0746FFE00C2140463CF17FFB074625462068416A20468847064628683146CE
:40B60000826A28469047EEE0EEE0EBE0404643F170FA81460F2140463CF168FB0746AB4800EB890090ED000AB5EEC00AF1EE10FA0DD02068416B20468847A44800EB89000A
:40B64000D0ED000AB4EE600AF1EE10FA01D1012000E00020074025462068416B20468847B0EE408A2C462868816B2846884726462068C16A20468847B0EE408A344630689F
:40B68000016B30468847AEE00D2140463CF12EFB074625462068416A20468847064628683146826A284690479DE00E2140463CF11DFB074625462068416A204688470646BA
:40B6C00028683146826A284690478CE0404643F110FA8146102140463CF108FB07467B4800EB890090ED000AB5EEC00AF1EE10FA0DD02068416B20468847744800EB89005D
:40B70000D0ED000AB4EE600AF1EE10FA0AD107E067E065E063E061E05FE05DE01DE05AE0012000E00020074025462068416B20468847B0EE408A2C462868816B28468847F9
:40B7400026462068C16A20468847B0EE408A34463068016B3046884745E0404643F15BFB8146112140463CF1C1FA0746574800EB890090ED000AB5EEC00AF1EE10FA0DD094
:40B780002068416B20468847504800EB8900D0ED000AB4EE600AF1EE10FA01D1012000E00020074025462068416B20468847B0EE408A2C462868816B2846884726462068C3
:40B7C000C16A20468847B0EE408A34463068016B3046884707E000BF00BF00BF00BF00BF00BF00BF00BF00BF3846BDEC028BBDE8F08770B5044620463AF002FEC5B20021B9
:40B8000028463CF173FA70BD002008E09FED300A2E4901EB800181ED000A411CC8B20F28F4D3704710B50446E0B243F1D2FB10BD10B50446E0B244F14BF810BD10B50446B9
:40B84000E0B243F1F9FB10BD10B50446E0B244F186FB10BD70B504460D46E0B2294643F196F870BD10B52DED028B0446B0EE408AE0B2B0EE480A43F19DF8BDEC028B10BDFF
:40B8800010B52DED028B0446B0EE408AE0B2B0EE480A43F1FAF8BDEC028B10BD70B504460D46E0B2294643F1DCF970BD10B52DED028B0446B0EE408AE0B2B0EE480A43F1F2
:40B8C0000BFABDEC028B10BD88000020942300100000000010B52DED028B0446B0EE408AE0B2B0EE480A43F162FABDEC028B10BD0148007870470000880000202DE9F04137
:40B9000006460C4615460027002E61D0B4F1D04F0ED36019401E8149884209D8A4F1D0412A4630463BF1B4FC002851D101274FE07B4884420ED36019401E7A49884209D8DF
:40B940007748211A2A4630463BF1C6F900283FD101273DE0744884420ED36019401E72493F31884208D87048211A2A4630463BF1B9FA68BB01272BE0B4F1805F0BD3601987
:40B98000401E6A49884206D82A462146304688F114FF01271CE0B4F1005F0BD36019401E6349884206D82A462146304688F105FF01270DE0B4F1006F0AD36019401EB0F17C
:40B9C000026F05D22A462146304688F1F6FE01273846BDE8F0812DE9F04106460C4615460027002E51D0B4F1D04F0ED36019401E4A49884209D8A4F1D0412A4630463BF161
:40BA0000A5FB002841D101273FE0454884420DD36019401E4349884208D84148211A2A4630463BF12BF908BB01272EE03E4884420ED36019401E3C493F31884208D83A488D
:40BA4000211A2A4630463BF1FBF978B901271CE0B4F1805F0BD36019401E3449884206D82A463146204688F1A8FE01270DE0B4F1005F0AD36019401E2D49884205D82A460C
:40BA80003146204688F199FE01273846BDE8F08170B504460D460026002D3CD0B4F1D04F0CD36019401E1D49884207D8A4F1D04029463BF149FC00BB01262CE0184884429A
:40BAC0000ED36019401E1749884209D8144AA21A5119134AA01A3BF110F870B901261AE0B4F1805F0AD36019401E1049884205D8294620463CF04AFD01260CE0B4F1005FD3
:40BB000009D36019401E0A49884204D8294620463CF03CFD0126304670BD0000FF7F006800010168FF00016900000168FFFF0010FFFF0220084B03604160027270477047CC
:40BB400070B504462046FFF7FAFF05463DF0EAFA70BD014600207047A4C20A082DE9F04104460D4616461F463A4631462046FFF7E1FF04462C482060E5602046BDE8F0810B
:40BB800010B504462046FFF7DAFF0446204610BD70B504462046FFF7F3FF05463DF0C2FA70BD01460120704770B504460D46002600202860E06820B12946E06849F1A8FD48
:40BBC0000646304670BD2DE9F04104460D4616460027E06828B132462946E06849F1B1FD07463846BDE8F0812DE9F04104460D4616461F464FF00008E06830B13B463246C8
:40BC00002946E06849F1BBFD80464046BDE8F08170B504464FF0FF35E06818B1E06849F1CDFD0546284670BDF4C1190870B504460025022614B9544D00BF00BF00BF25B1C1
:40BC400032462946514849F194FF70BD70B504460D466FF00040206015B1012D06D100E008E0206840F00040206003E00020FFF7DDFF00BF00BF204670BD70B504460E46B5
:40BC8000154626F00040206015B1012D06D100E008E0206840F00040206003E00020FFF7C5FF00BF00BF204670BD0A680260704770470A680260704770B5044606252046AD
:40BCC00089F1D0FF28B1012805D12068C0F3826501E0002500BF00BF284670BD0146086800F0807008B1012070470020FCE70146086800F0007008B1012070470020FCE70C
:40BD000070B504464FF0FF35204689F1ABFF01280DD1206800F47000B0F5700F04D21C49206801EA102502E02068C0F31125284670BD70B50446FF25204689F193FF012881
:40BD400002D12068C0F30745284670BD70B50446FF25204689F186FF012808D1206800F47000B0F5700F02D22088C0F30725284670BD70B50446FF25204689F173FF0128C0
:40BD800000D12578284670BD0DE40408FEE3040800FF03002DE9F04104460D4616461F463A4631462046FFF7C5FE04460C482060E5602046BDE8F08110B504462046FFF789
:40BDC000BEFE0446204610BD70B504462046FFF7F3FF05463DF0A6F970BD01460320704704C60A080EB50321104880F8951000BF4FF4FA7100208AF169F98DE80700009832
:40BE0000082810D1019800F4804060B10021074880F8951000200549C1F890008AF17AF904468AF183F903F04AF9E1E7B009002010B5FDF7DBF8343010BD704700000000D5
:40BE40000000000000000000000000003037373031373134353500000000000030373730313731343335000000000000526176656E20496E647573747269657320496E633A
:40BE80000000000000000000000000004A756E2D32382D32303138000000000032342E312E302E340000000000000000556E766572666572746820477261696E20436172D1
:40BEC00074204D6F64756C6500000000303737303137313533380000000000000000000000000000000000000000000000000000000000000000000000000000FFFFFFFF45
:40BF0000FFFFFFFFFFFFFFFFFFFFFFFFFFFFFFFFFFFFFFFFFFFFFFFFFFFFFFFFFFFFFFFFFFFFFFFFFFFFFFFFFFFFFFFFFFFFFFFFFFFFFFFFFFFFFFFFFFFFFFFFFFFFFFFF41
:40BF4000FFFFFFFFFFFFFFFFFFFFFFFFFFFFFFFFFFFFFFFFFFFFFFFFFFFFFFFFFFFFFFFFFFFFFFFFFFFFFFFFFFFFFFFFFFFFFFFFFFFFFFFFFFFFFFFFFFFFFFFFFFFFFFFF01
:40BF8000FFFFFFFFFFFFFFFFFFFFFFFFFFFFFFFFFFFFFFFFFFFFFFFFFFFFFFFFFFFFFFFFFFFFFFFFFFFFFFFFFFFFFFFFFFFFFFFFFFFFFFFFFFFFFFFFFFFFFFFFFFFFFFFFC1
:40BFC000FFFFFFFFFFFFFFFFFFFFFFFFFFFFFFFFFFFFFFFFFFFFFFFFFFFFFFFF000014083FCF190800C000087FEC0A0804880008FBBF000800800008FF870008F8E96C35DF
:40C00000704770477CB505460E461DB1052D01D0042D02D10020401C00BFFA21FC4800688AF148F860BBFB480088ADF804008DF806508DF80760F84C0198009004F1080070
:40C04000216800EB8100009901602068401C01462060204689F128FD2060D4E90001884202D16068401C00E06068606000BFE84800683DF061FA0221E84877F1DAFE00BF89
:40C080007CBDE74A116070472DE9F04786B00446E448007800F0010070B9E2483DF05EF850B1E1481BF002FA0646E04AE0493CF0BDF9DC48AFF30080DE48007800F001002F
:40C0C00070B9DC483DF04AF850B1DB4819F016FD0646D64AD9493CF0A9F9D648AFF30080D748007800F0010070B9D5483DF036F850B1D4481AF0E0FA0646CC4AD2493CF0D5
:40C1000095F9CF48AFF30080D048007800F0010070B9CE483DF022F850B1CD481DF011F80646C24ACB493CF081F9C848AFF30080C948007800F0010070B9C7483DF00EF8DC
:40C1400050B1C64875F10DF90646B84AC4493CF06DF9C148AFF30080C248007800F0010070B9C0483CF0FAFF50B1BF4874F1B4F90646AE4ABD493CF059F9BA48AFF300805D
:40C18000BB48007800F0010070B9B9483CF0E6FF50B1B8481DF0CAF90646A44AB6493CF045F9B348AFF3008000270025A846A946AA46002000902078002871D10090607814
:40C1C00007286ED2DFE800F00495FEFDFCFBFA00AA48006880470646314690481438FFF750FF142101A83CF0F3F91422A11D01A888F1E3FA0020A2490870A078E17840EA40
:40C200000120844908802079617940EA01209D4908809D48007D30B914229B4901A83CF038F9002850D0994A694601A81BF06FFD80B1964800680068C168944800688847DC
:40C2400093490860934B52460921744814381FF09FF92CE01BF050FC322823D272481BF037FA8C4B142201A96F481BF0FCF96E487BF1C7FE70B1032000906B481BF068F93B
:40C2800083490860834B52460A21644814381FF07FF90CE004200090401F7D49086006E0F3E3F3E305200090801F79490860744801789DF80000FFF7A5FE4FF0FF3076496D
:40C2C00008607649086007E0022000906C4801789DF80000FFF796FE14216B483CF078F9142201A968483CF01FF90020664908753EE262480068804706463146474814388E
:40C30000FFF7BFFE142101A83CF062F91422A11D01A888F152FA012059490870A078E17840EA01203B4908802079617940EA01205449088056480068B0F1FF3F66D05248E8
:40C34000007D012806D114224F4901A83CF0A1F800285BD0524B6A464D48016801A81AF08EF880B14E4800680068C1684C480068884749490860474B52460B212748143897
:40C380001FF006F937E019F069FFB0F5FA7F2DD2294819F0E6FC3F4B142201A9264819F098FC3C4A3A480168234819F0B9FC22487BF127FEA0B10320009004E067E391E2BF
:40C3C000D7E12EE183E01C4819F0EAFB32490860304B52460C21114814381FF0D9F80AE004200090401F2C49086004E005200090801F29490860224801789DF80000FFF7BF
:40C4000001FE4FF0FF302549086053E04AE00000140000101A00001010240010E4230010200000105C0000103425001000800008D37402085800001060250010235B020850
:40C440005400001090250010DF66020850000010D8250010699102084C0000100C260010891318084800001040260010FF041808440000107C260010539502082803002045
:40C48000400000101C000010AC260010600000107C000010A98F040880000010840000106400001002200090FE4801789DF80000FFF7A8FD1421FC483CF08AF8142201A99E
:40C4C000F9483CF031F80120F74908756FE3F7480068804706463146F548FFF7D2FDA079E17900EB0120217A00EB0140617A00EB0167142101A83CF06BF8142204F10A012C
:40C5000001A888F15AF90220E6490870A078E17840EA0120E74908802079617940EA0120E5490880E5480068B0F1FF3F64D0DE48007D022806D11422DB4901A83BF0A9FFB3
:40C54000002859D0DE4B6A46DC48016801A81AF087FEF8B1DA4800680068416AD848006888470646B7420ED0D5480168D5481AF04AFAD54A3946D3481AF016FAD0480168C7
:40C58000D0487BF1C2FFD04B52460D21C8481EF0FFFF2AE01AF06BFDB0F57A7F23D2C9481AF023FAC84A3946C6481AF0FDF9C64B142201A9C3481AF096F9C34ABF48016841
:40C5C000C0481AF0DEF9BF487BF11BFD40B103200090BD4B52460E21B5481EF0D9FF04E00420009001E005200090AE4801789DF80000FFF707FD07E002200090A948017842
:40C600009DF80000FFF7FEFC1421A7483BF0E0FF142201A9A4483BF087FF0220A2490875C5E2A2480068804706463146A048FFF728FDA079E17900EB0120217A00EB014074
:40C64000617A00EB016564204543142101A83BF0BFFF142204F10A0101A888F1AEF8032090490870A078E17840EA0120914908802079617940EA01208F4908808A48007DBE
:40C68000032806D11422884901A83BF002FF00285AD08E4A694601A876F143FC48B38B4800680068C16989480068884706466420B6FBF0F0301AA84205D26420B6FBF0F023
:40C6C0003044A8420ED88148016881481CF09CFE7D4A29467E481CF055FE7C4801687C487CF167F9784B52460F2171481EF050FF23E076F120FB32281DD275481CF076FE90
:40C70000714A294672481CF03DFE6F4B142201A96F481CF010FE6E487BF173FC40B103200090694B5246102161481EF031FF04E00420009001E0052000905A4801789DF8EC
:40C740000000FFF75FFC07E002200090554801789DF80000FFF756FC142153483BF038FF142201A950483BF0DFFE03204E4908751DE24E4800688047064631464C48FFF7E2
:40C7800080FCA079E17900EB0120217A00EB0140617A00EB0165142101A83BF019FF142204F10A0101A888F108F804203D490870A078E17840EA01203E49088020796179B2
:40C7C00040EA01203C4908803748007D042805D11422354901A83BF05CFEE8B33D4A694601A819F07EF8F0B13A4800680068C169384800688847A8420ED036480168364807
:40C8000074F112FF304A2946334874F1CBFE3148016831487CF130F92B4B5246112124481EF0B6FE25E018F066FF64281FD22A4874F1ECFE244A2946274874F1B3FE224B12
:40C84000142201A9244874F186FE23487BF1D9FB50B10320009000E012E01B4B5246122113481EF095FE04E00420009001E0052000900C4801789DF80000FFF7C3FB07E0FA
:40C8800002200090074801789DF80000FFF7BAFB142105483BF09CFE142201A902483BF043FE1BE040000010AC26001028030020D02300101A0000101C0000108000001080
:40C8C0006800001090250010A98F04086C000010D8250010700000100C2600100420F649087564E1F5480068804706463146F448FFF7C7FBA079E17900EB0120217A00EB1F
:40C900000140617A00EB0168A07AE17A00EB0120217B00EB0140617B00EB0169142101A83BF056FE142204F10F0101A887F145FF0520E4490870A078E17840EA0120E2495F
:40C9400008802079617940EA0120E0490880DA48007D052806D11422D74901A83BF099FD00287DD0DA4A694601A874F1EFFBB8B3A07B28BBD64800680068C169D448006818
:40C980008847404508D1D24800680068016AD04800688847484513D0CD480168CD4873F148FFCD4A4146CB4873F1D9FECA4A4946C84873F1E7FEC6480168C6487BF18BFF95
:40C9C000C54B52461321BE481EF0E2FDC04800680068C168BE4800688847C049086038E0FFE774F1A8FA19282ED2A07B58BBB94873F111FFB84A4146B64873F1B0FEB64A37
:40CA00004946B44873F1BEFEB34B142201A9B14873F17EFEAF487BF1F4FA68B103200090AC4873F1ABFDAD490860AB4B52461421A3481EF0ADFD0CE004200090401FA749C4
:40CA4000086006E00CE0FFE705200090801FA34908609C4801789DF80000FFF7D3FA07E002200090974801789DF80000FFF7CAFA142191483BF0ACFD142201A98E483BF036
:40CA800053FD05208C49087591E092E07FE08B4800688047064631468948FFF7F2FA142101A83BF095FD1422A11D01A887F185FE062084490870A078E17840EA01208249D0
:40CAC00008802079617940EA01208049088083480068B0F1FF3F45D07748007D062805D11422754901A83BF0D4FC70B37C4B6A467A48016801A81DF093F930B1764B52465F
:40CB000015216F481EF044FD25E01DF07CF864281FD274481CF03DFE6F4B142201A971481CF0EFFD6C4A6D4801686E481CF010FE6C487BF166FA48B103200090664B52464F
:40CB400016215F481EF024FD05E00BE00420009001E0052000905B4801789DF80000FFF751FA07E002200090564801789DF80000FFF748FA142150483BF02AFD142201A920
:40CB80004D483BF0D1FC06204B4908750FE0142101A83BF01DFD142147483BF019FD0820454908754FF6FE704749088000BF00BF00BF00BF06B0BDE8F08701464A4800787D
:40CBC00070470EB50121494880F88D10032180F88D1000BF3A48FFF7F0FF012819D1811E434800683CF086FC8DE80700009820280ED1019C3CB12046FFF746FA21463C48F5
:40CC000000683CF069FC2146394800683CF064FCE0E70021354880F88D1000203349C1F8880089F177FA044689F180FAD2E710B5044620680169204688470020E06210BD81
:40CC400010B50446204689F10AF820B907211C48143077F1EEF810BD10B50446204688F1FEFF20B906211648143077F1E2F810BD10B50446204688F1F2FF20B9052110482D
:40CC8000143077F1D6F810BD10B50446204688F1E6FF20B904210A48143077F1CAF810BD10B50446204688F1DAFF20B903210448143077F1BEF810BDAC2600102803002063
:40CCC000D0230010400000101A0000101C0000107400001040260010A98F040884000010780000107C26001018000010B00900203C00001070B50546284688F1B0FF98B1E3
:40CD0000FE4C204688F1C7FE60B904F10800616800EB8100002101606068411C204688F1C3FE606000BF00BF70BD2DE9F04FA1B006460F46F5B2B9464FF0000A092D73D257
:40CD4000DFE805F0FA051379C2FEF8F7F600EC4836F13AF8022803DBEA480CF0B2FB08B1012000E00020824692E100201F902090E24888F190FE00285AD13221E24800685A
:40CD800089F198F9002853D1DC4C0DF178088346204688F180FE48B94FF0010B04F10800616800EB81000068C8F8000000BFBBF1010F3DD101208DF87C009DF87B008DF86A
:40CDC0007D009DF87A008DF87E00BDF87800C0B28DF87F00BDF87800000A8DF88000FF208DF881008DF882008DF88300C64800683CF0A2FBC24835F1E7FF022812DB002005
:40CE0000AFF20F110290CDE9030105900620BF49BC4B0822CDE900101FA94FF6B2200FF0C7FA10B9012001E031E10020824601E04FF0010A2CE1682107A83BF0C9FB082040
:40CE40008DF81C00FEF78AF90446142221460DF11D0087F1B2FCFEF794F90446142221460DF1310087F1A9FCFEF79EF90446142221460DF1450087F1A0FCFEF7A8F9044612
:40CE8000142221460DF1590087F197FC1422A0490DF16D0087F191FC0020AFF2FB110290CDE90301059006209849964B6522CDE9001007A94FF6B0200FF07AFA08B90120E7
:40CEC00000E000208246E3E018211BA83BF080FB00208DF86C00FEF741F9834687F14EFC142801D9142004E0FEF738F9834687F145FC0446FEF732F98046224641460DF147
:40CF00006D0087F15AFC0020AFF283210290CDE90301059006207D497A4B1522CDE900101BA94FF6B0200FF043FA30B9012005E0ACE073E03BE003E0A7E000208246A7E0EB
:40CF400018211BA83BF044FB01208DF86C00FEF718F9834687F112FC142801D9142004E0FEF70FF9834687F109FC0446FEF709F98046224641460DF16D0087F11EFC002060
:40CF8000AFF213310290CDE90301059006205F495C4B1522CDE900101BA94FF6B0200FF007FA08B9012000E00020824670E018211BA83BF00DFB02208DF86C00FEF7F4F843
:40CFC000834687F1DBFB142801D9142004E0FEF7EBF8834687F1D2FB0446FEF7E5F88046224641460DF16D0087F1E7FB0020AFF297310290CDE90301059006204349414BC8
:40D000001522CDE900101BA94FF6B0200FF0D0F908B9012000E00020824639E018211BA83BF0D6FA05208DF86C00FEF7D0F8834687F1A4FB142801D9142004E0FEF7C7F803
:40D04000834687F19BFB0446FEF7C1F88046224641460DF16D0087F1B0FB0020AFF21F410290CDE90301059006202849254B1522CDE900101BA94FF6B0200FF099F908B96D
:40D08000012000E00020824602E000BF00BF00BF00BFBAF1000F04D1294609F1140076F1C8FE21B0BDE8F08F38B50446204635F13DFE044617482060AFF2913302220821A2
:40D0C00004F11400009476F1CFFDA0F1140400230D22114920461EF0D8F92046FFF7A7FD0E4888F1C3FF0849086000210C483CF0DBF90C490860204638BD000010240010AB
:40D10000D0230010E05B001014000010182500109CBE000868C70A0809AE0008489A1908549A19083C00001010B50446FD48206004F1140076F1C2FDA0F11404204635F138
:40D1400004FE0446204610BD70B504462046FFF7EBFF05463BF0E6FF70BDF34A117070472DE9F04105460C4617461E46002E4AD00D2E66D00E2E73D1242C20D004DC182C3C
:40D1800007D0232C3CD10FE0252C23D0262C37D12BE0E64835F118FE022804DB0321E348143076F146FE2CE0E04835F10DFE022804DB0421DD48143076F13BFE21E0DB4833
:40D1C00035F102FE022804DB0521D848143076F130FE16E0D54835F1F7FD022804DB0621D248143076F125FE0BE0D04835F1ECFD022804DB0721CD48143076F11AFE00E0A1
:40D2000000BF00BF2DE08D2C0CD0902C0BD0B92C14D1C74845F133FC18B92868C168284688470CE000BF0121C048143076F101FE0321BE48143076F1FCFD00E000BF00BF87
:40D240000FE0192C02D01C2C07D100E000BF0021B648FFF782FF01E002E000BF00BF00E000BF00BFBDE8F081704710B504466421E06A1EF0B1F938B104F1140076F125FDD6
:40D28000AC4800688047E06210BD70B505460C46284635F199FDA04213D06C7200231A46042128461EF074F9012C08D1002211469F4845F1E8FB00209F49087000E000BF7E
:40D2C00000BF70BD2DE9F04781460D4692461C4625F0E0062778607847EA00272CB3072E21D2DFE806F0201D041E1F200C0000BF03218E48FFF7C9FF00BF00BF14E02078E8
:40D300000006617840EA0140A17840EA0120E17840EA01080822211D404635F18BFD03E000BF00BF00BF00BF00BFBDE8F08770B504461546084640F08006314621F0E00225
:40D34000012A0AD0022A04D0032A07D0042A07D105E000BF00BF00BF03E000BF00BF00BF00BF00BF70BD014674480068704770B505466E48FFF7F7FF04466C4835F124FD38
:40D38000012814DB6948FFF718FC01280FD143F6982120461EF020F948B104216348FFF7DCFE674B00221A2160481EF0F1F870BD0146644800887047624A11807047014631
:40D3C000614800887047604A1180704701465F48006870475D4A1160704701465C48006870475B4A1160704701465A4800687047584A116070470146574800687047564A29
:40D400001160704770B506460C460025204635F159FF022035F15CFF284670BD2DE9F04180460C46002500260027D4F80160D4F80570304635F13AFF384635F13DFF0120A5
:40D4400035F146FF2846BDE8F0812DE9FC410446002001900027206801A9C2682046904701287FD100BF04F10C00FEF749FCA0F57A40B138002876D0012803D0B0F5A26FE4
:40D4800072D1F6E00198007800286ED0022802D004286BD17FE03149086A6FF001013CF087F82E49886D6FF001013CF081F82B49886800213CF07CF82849086900213CF05B
:40D4C00077F82649D1F8800000213CF071F82349886F00213CF06CF82049886A01213CF067F8144800688047054629460F48FEF7C8FD14211A483BF049F8082018490875D4
:40D5000001988078019AD27800EB022081B20748FFF752FF01980079019A527900EB022081B224E068C70A0818000010D0230010643900102803002024010020200000100A
:40D54000A98F04081A0000101C00001024000010280000102C00001030000010B0090020C12600109DE06AE099E048E065E06E48FFF729FF01216C48FFF7EFFDFDF756FFD7
:40D580004FF6FF7069490880694B3A461B2166481DF0FEFF51E06448FFF711FF06466248FFF706FF401C1FFA80F8002E05DD642008FB00F0B0FBF6F500E00025642D01D907
:40D5C000642500E000BF642D0AD102215648FFF7C4FD574B3A46192153481DF0D9FF09E003215148FFF7B9FD514B3A461C214E481DF0CEFF00214C48FEF743FD1DE03221EE
:40D600004C48006888F100FD06462068816920468847232804D8206881692046884700E0232005462A463046019987F1C6F83146404800683BF069FF00BF00BF30E0019872
:40D6400000780F2812D10198407800F0010060B1002000906A460021374844F10BF918B1334900981DF0DAFA00BF00E000BF00BF16E001980078112802D012280CD105E0A3
:40D680000199491C2848FFF7C9FE06E0019841882548FFF7B7FE00E000BF00BF00E000BF00BFBDE8FC8110B50446AFF261224FF6B221204611F086FDAFF271224FF6B12180
:40D6C000204611F07FFDAFF27D224FF6C171204611F078FD10BD38B51348FFF7E5FC0446164AAFF2BB513AF0A1FE154C002020606060642104F108003AF048FF00BF2546CA
:40D700000E4A104928463AF091FEAFF2650001230D4A194600900D4811F013FA0446074A0B493AF083FE38BDD02300101A000010A98F04083C0000106439001000800008BD
:40D7400010240010CF8D04084C9A19081825001081EF010810B5002807DA0A07140EFE4A00F00F031B1FD45403E00A07130EFB4A135410BD70B504460D460026082C0BDAF4
:40D780000120A040C6B23146B32038F1CDFA0021B42038F1C9FA27E0082C09D110260021B32038F1C1FA3146B42038F1BDFA1BE0092C09D120260021B32038F1B5FA3146F4
:40D7C000B42038F1B1FA0FE00F2C05DAA4F10A0084B20120A040C6B20021B32038F1A4FA3146B42038F1A0FA2946B12038F19CFA70BD10B5044601EE102AF8EE411A01EECD
:40D80000103AB8EE411A81EE812AB0EE420AB7EE001AB4EEC10AF1EE10FA04DDB7EE001AB0EE410A08E0B5EEC00AF1EE10FA03D29FEDCB1AB0EE410AB7EE001A71EE401A16
:40D8400001EE101AB8EE411A61EE811A01EE104AB8EE411AF0EE610A41EE000ABCEEE01A11EE100A10BD10B5044604F00F040121692037F156F804F00101412037F151F84F
:40D88000C4F34001392037F14CF8C4F38001602037F147F8E108692037F143F810BD7FB506460C461546072002900020039001940095694630467EF18CFF7FBDF8B50446D5
:40D8C0000D46164600BF00200090A648006840F48000A44908600846006800F48000009000BF2560002060600021A160012121610021A16121626162E162A162E160E661D0
:40D90000216301216161984885421ED19748A063846397489549086000204860002193488160C1602915016189004161890081610021C1614FF400310162002141620121FF
:40D9400081620021C162016346E08A48854220D18948A063846386483030874908604FF000704860002184488160C1602915016189004161890081610021C1614FF4003118
:40D98000016200214162012181620021C162016322E07A4885421FD17948A063846374481830774908604FF080604860002174488160C16029150161890041618900816165
:40D9C0000021C1614FF40031016200214162012181620021C162016320467EF1D6FAA06B38F0E2FDA06B00686149884207D100213820FFF7AFFE382000F09AFD1AE0A06B26
:40DA000000685B493031884207D100213A20FFF7A1FE3A2000F08CFD0CE0A06B006854491831884206D100213920FFF793FE392000F07EFDF8BD8CB04FF0020800270025C3
:40DA40000321504880F85D104F480021016041608160C160062244494C48FFF72FFF052244494B48FFF72AFF082244494948FFF725FF00210846FFF77DFE44480068406898
:40DA800040F02000414909684860082201213F48FFF705FF032202213C48FFF700FF0F2203213A48FFF7FBFE092204213748FFF7F6FE112205213548FFF7F1FE1222062150
:40DAC0003248FFF7ECFE0A2201213148FFF7E7FE0B2202212E48FFF7E2FE0C2203212C48FFF7DDFE0D2204212948FFF7D8FE0E2205212748FFF7D3FE002201212548FFF733
:40DB0000CEFE012202212348FFF7C9FE022203212048FFF7C4FE062204211E48FFF7BFFE072205211B48FFF7BAFE092206211948FFF7B5FE0E2207211648FFF7B0FE0F2296
:40DB400008211448FFF7ABFE1348006820F480000549C1F8040321E018ED00E000E400E0000000003038024000200140B418002010640240002101401419002000220140B3
:40DB800074190020B0090020A4180020D41900201C1A0020641A00200423014000BF0021084688F193FA09AB07C3099808280FD10A9800F4804058B10021F74880F85D1093
:40DBC0000020F549886588F1A5FA044688F1AEFA0026EEE33046FFF746FE06203BF058FC36F18AFF022805D1EC48007838F111F8EB498855EB480068806840F00100E94986
:40DC000009688860062201A9E6487EF101FD814641F28831012088F159FA09AB07C3099808287DD1B9F1000FFBD1DF48006880470446DE48C0F8F840C0F8FC40DC490598F0
:40DC4000C1F8F8000698C1F8FC00DA490598C1F8F8000698C1F8FC00102E1ED2DFE806F0081E344A61778DA3B9F1F0EFEEEDECEBCE4804600464C0F88040CD490198086099
:40DC8000029808640398C1F88000CA4901980860029808640398C1F88000B0E2C34844604464C0F88440C24901984860029848640398C1F88400BF4901984860029848643E
:40DCC0000398C1F884009AE2B84884608464C0F88840B74901988860029888640398C1F88800B44901988860029888640398C1F8880084E2AD48C460C464C0F88C40AC49A1
:40DD00000198C8600298C8640398C1F88C00A9490198C8600298C8640398C1F88C006EE26FE2A24804610465C0F89040A04901980861029808650398C1F890009D490198ED
:40DD40000861029808650398C1F8900057E2974844614465C0F89440954901984861029848650398C1F89400924901984861029848650398C1F8940041E28C4884618465FD
:40DD8000C0F898408A4901988861029888650398C1F89800874901988861029888650398C1F898002BE28148C461C465C0F89C407F490198C8610298C8650398C1F89C004D
:40DDC0007C490198C8610298C8650398C1F89C0015E2764804620466C0F8A040442042F102F930B1502042F1FEF840B10020019005E0502042F1F7F808B9002001903A20D7
:40DE000042F1F1F830B1452042F1EDF840B10020029005E0452042F1E6F808B900200290392042F1E0F868B1382042F1DCF878B1002003900CE017E100E1E9E0D2E0BBE064
:40DE400060E016E0382042F1CEF808B900200390574901980862029808660398C1F8A000544901980862029808660398C1F8A000C5E14E4844624466C0F8A440362042F1BB
:40DE8000B2F830B1372042F1AEF840B10020019005E0372042F1A7F808B900200190322042F1A1F830B1332042F19DF840B10020029005E0332042F196F808B9002002905C
:40DEC0002E2042F190F830B12F2042F18CF840B10020039005E02F2042F185F808B900200390334901984862029848660398C1F8A400304901984862029848660398C1F8DF
:40DF0000A4007CE1294884628466C0F8A840352042F169F830B1342042F165F840B10020019005E0342042F15EF808B900200190312042F158F830B1302042F154F840B106
:40DF40000020029005E0302042F14DF808B900200290172042F147F830B1182042F143F840B10020039005E0182042F13CF808B9002003900E490198886202988866039806
:40DF8000C1F8A8000B4901988862029888660398C1F8A80033E10000B0090020AD000010A4180020D4190020C4BE190870170020081500203C160020FE48C462C466C0F8CB
:40DFC000AC40FD490198C8620298C8660398C1F8AC00FA490198C8620298C8660398C1F8AC000CE1F34804630467C0F8B040F24901980863029808670398C1F8B000EF4970
:40E0000001980863029808670398C1F8B000F6E0E84844634467C0F8B440E74901984863029848670398C1F8B400E44901984863029848670398C1F8B400E0E0DD48846378
:40E040008467C0F8B840DC4901988863029888670398C1F8B800D94901988863029888670398C1F8B800CAE0D248C463C467C0F8BC40D1490198C8630298C8670398C1F8C7
:40E08000BC00CE490198C8630298C8670398C1F8BC00B8F10E0F13D2DFE808F007131F2B37434F5B67737F8B97A3C248C0F8C040C1490498C1F8C000C0490498C1F8C000E1
:40E0C0009BE0BC48C0F8C440BB490498C1F8C400BA490498C1F8C4008FE0B648C0F8C840B5490498C1F8C800B4490498C1F8C80083E0B048C0F8CC40AF490498C1F8CC0012
:40E10000AE490498C1F8CC0077E0AA48C0F8D040A9490498C1F8D000A8490498C1F8D0006BE0A448C0F8D440A3490498C1F8D400A2490498C1F8D4005FE09E48C0F8D84068
:40E140009D490498C1F8D8009C490498C1F8D80053E09848C0F8DC4097490498C1F8DC0096490498C1F8DC0047E09248C0F8E04091490498C1F8E00090490498C1F8E0007C
:40E180003BE08C48C0F8E4408B490498C1F8E4008A490498C1F8E4002FE08648C0F8E84085490498C1F8E80084490498C1F8E80023E08048C0F8EC407F490498C1F8EC00F1
:40E1C0007E490498C1F8EC0017E07A48C0F8F04079490498C1F8F00078490498C1F8F0000BE07448C0F8F44073490498C1F8F40072490498C1F8F40000BF00BF00BF00BFD1
:40E2000000BF6F487EF1ABFA6D487DF18AFF6D480068806840F001006A4909688860052201A968487EF1F4F9814641F28831012087F14CFF09AB07C30998082867D1B9F1C1
:40E24000000F64D138460FF0E2FB04465E480068804707465748C0F80071C0F80471C0F80871C0F80C71C0F8107153490198C1F800010298C1F804010398C1F808010498C0
:40E28000C1F80C010598C1F810014C4AD2F80011494A0C23D2F800012246FFF7AAFA4749C1F800010A46D2F80411434A0C23D2F804012246FFF79DFA4049C1F804010A46A1
:40E2C000D2F808113C4A0C23D2F808012246FFF790FA3A49C1F808010A46D2F80C11364A0C23D2F80C012246FFF783FA3349C1F80C010A46D2F810112F4A0C23D2F81001EE
:40E300002246FFF776FA2D49C1F8100100BF2D487EF125FA2B487DF104FF2C480068806840F00100294909688860082201A927487EF16EF9814641F28831012087F1C6FE40
:40E3400009AB07C3099808287ED1B9F1000F7BD128460FF05CFB04461B480068804705461448C0F81451C0F81851C0F81C51C0F82051C0F82451C0F82851C0F82C51C0F8DC
:40E3800030510D490198C1F814010298C1F818010398C1F81C010498C1F820010598C1F824010698C1F828010798C1F82C0108980EE081E070170020081500203C16002007
:40E3C000D41900201C1A0020C4BE1908641A0020C1F830015C4AD2F814115C4A0C23D2F814012246FFF705FA5749C1F814010A46D2F81811554A0C23D2F818012246FFF729
:40E40000F8F95149C1F818010A46D2F81C114F4A0C23D2F81C012246FFF7EBF94A49C1F81C010A46D2F82011484A0C23D2F820012246FFF7DEF94449C1F820010A46D2F831
:40E440002411424A0C2300E02FE0D2F824012246FFF7CFF93C49C1F824010A46D2F828113A4A0C23D2F828012246FFF7C2F93649C1F828010A46D2F82C11344A0C23D2F804
:40E480002C012246FFF7B5F92F49C1F82C010A46D2F830112D4A0C23D2F830012246FFF7A8F92949C1F8300100BF29487EF157F927487DF136FE761C102EFFF48BAB08F17C
:40E4C00001001FFA80F8B8F10D0F01DD4FF0020800214046FFF74EF9FFF761BB10B504461C4890F85D00032804D11A49886D01213BF046F810BD10B51749886B38F0ABFABB
:40E5000010BD10B51549886B38F0A5FA10BD10B50F49886B38F09FFA10BD10B50E487DF171FF0E487DF16EFF09487DF16BFF10BD00F01F02012191404209920002F1E022D0
:40E54000C2F80011704700003C16002008150020641A0020B0090020D41900201C1A00207CB500260020FA4981F8CC00F94981F8CC00F748D0F8C80028B9F74887F176FD30
:40E58000F349C1F8C800F348D0F8C80028B9F34887F16CFDEF49C1F8C8000020092103460246CDE900100221ED48007836F112FA0020092103460246CDE900100221E94884
:40E5C000007836F107FA0020092103460246CDE900100221E448007836F1FCF90020092103460246CDE900100221E048007836F1F1F9DF48D64908600C2048600021D448C3
:40E6000081604FF08071C1604FF4202101614FF4001141610021017601214176002181760121C17600210177012141770020C84988620021C648C1620163416381630121FC
:40E64000C163002101640121416481640021C164C848C04908600C2048600021BD4881604FF08071C1604FF4202101614FF4001141610021017601214176002181760121CA
:40E68000C17600210177012141770020B14988620021B048C16201634163012181630E21C163002101640121416481640E21C16413207FF1DFFB15207FF1DCFB14207FF1EC
:40E6C000D9FB3F207FF1D6FB41207FF1D3FB40207FF1D0FB9E487EF1DAFD0446ACB99C4928319B487EF1DCFE044674B998487EF167FF04464CB9032195487FF1CBF904462D
:40E700001CB90120924981F8CC0092487EF1BFFD0546ADB98F4928318E487EF1C1FE054675B98C487EF14CFF05464DB9112189487FF1B0F905461DB90120864981F8CC000E
:40E7400004B1264605B12E4630467CBD70B588B0054600260020009000BF287D18B1022803D17B4C03E07B4C01E0002400BF00BF002C76D094F8CC00012872D10121D4F8DE
:40E78000C80087F197FC0028F7D100BF00BFE86800F0004008B1012000E0002000BF50B1012809D1284687F14AFA0390002002900420049008E000BF284687F140FA02907B
:40E7C00000200390049000BF00BF002005902868816928468847069000208DF81C005D48844203D13F207FF152FB05E05848844202D113207FF14BFB286801A9C26828465D
:40E800009047012834D16B4602A92046019A7EF15BFF30B1012825D0022824D0032824D122E00098012804D0022809D0042815D10DE02822294604F1500039F075FE0DE050
:40E840002822294604F1780039F06EFE06E02822294604F1A00039F067FE00BF00BF012605E016E000BF00BF00BF002600BF00BF3848844203D13F207FF1FCFA05E034487A
:40E88000844202D113207FF1F5FAD4F8C8003AF053FE304608B070BD2DE9F84305460C4691464FF002082B48854202D14FF0000804E02748854201D14FF00208B8F1020F72
:40E8C00013DAA06820B1042803D16668012703E000BF2668002700BF00BFCDF80080237C4A46314638461DF063F9BDE8F88310B517487FF108F910BD10B515487FF103F9A5
:40E9000010BD10B512487FF1FEF810BD10B511487FF1F9F810BD10B50E487FF1F4F810BD10B50C487FF1EFF810BD10B504460948844204D1012150300DF00DFE06E0044814
:40E94000844203D1012150300DF005FE10BD0000CC1A00209C1B00209CDD0408A0DD04089E0000109F000010A0000010A1000010006400400068004010B504464748844235
:40E9800004D1012178300DF0E6FD06E04448844203D1012178300DF0DEFD10BD10B504463E48844204D10121A0300DF0D4FD06E03B48844203D10121A0300DF0CCFD10BDE5
:40E9C00010B504463548844204D1002150300DF0C2FD06E03248844203D1002150300DF0BAFD10BD10B504462C48844204D1002178300DF0B0FD06E02948844203D10021D4
:40EA000078300DF0A8FD10BD10B504462348844204D10021A0300DF09EFD06E02048844203D10021A0300DF096FD10BD10B58AB0044604E001AA03A92046FFF72DFF01AB33
:40EA400003AA002120467EF14CFF0028F2D00AB010BD10B58AB0044604E001AA03A92046FFF71AFF01AB03AA012120467EF139FF0028F2D00AB010BD10B509483AF0A8F964
:40EA80000446084A084939F0D1FC04483AF0A0F90446044A044939F0C9FC10BD9C1B0020CC1A002000800008C75A190838B5044660680090009D206880F3088800BFA847B8
:40EAC00038BD10B572B66FF0040000F0FCF96FF0010000F0F8F94FF0FF3000F0F4F9042000F0F1F9052000F0EEF9062000F0EBF9072000F0E8F9082000F0E5F9092000F065
:40EB0000E2F90A2000F0DFF90B2000F0DCF90C2000F0D9F90D2000F0D6F90E2000F0D3F90F2000F0D0F9102000F0CDF9112000F0CAF9122000F0C7F9132000F0C4F91420AC
:40EB400000F0C1F9152000F0BEF9162000F0BBF9172000F0B8F9182000F0B5F9192000F0B2F91A2000F0AFF91B2000F0ACF91C2000F0A9F91D2000F0A6F91E2000F0A3F9AD
:40EB80001F2000F0A0F9202000F09DF9212000F09AF9222000F097F9232000F094F9242000F091F9252000F08EF9262000F08BF9272000F088F9282000F085F9292000F0A6
:40EBC00082F92A2000F07FF92B2000F07CF92C2000F079F92D2000F076F92E2000F073F92F2000F070F9302000F06DF9312000F06AF9322000F067F9332000F064F93420AC
:40EC000000F061F9352000F05EF9362000F05BF9372000F058F9382000F055F9392000F052F93A2000F04FF93B2000F04CF93C2000F049F93D2000F046F93E2000F043F9CC
:40EC4000402000F040F9412000F03DF9422000F03AF9432000F037F9442000F034F9452000F031F9462000F02EF9472000F02BF9482000F028F9492000F025F94A2000F03A
:40EC800022F94B2000F01FF94C2000F01CF94D2000F019F94E2000F016F9502000F013F9512000F010F96FF0040000F015F96FF0010000F011F94FF0FF3000F00DF9042060
:40ECC00000F00AF9052000F007F9062000F004F9072000F001F9082000F0FEF8092000F0FBF80A2000F0F8F80B2000F0F5F80C2000F0F2F80D2000F0EFF80E2000F0ECF8B0
:40ED00000F2000F0E9F8102000F0E6F8112000F0E3F8122000F0E0F8132000F0DDF8142000F0DAF8152000F0D7F8162000F0D4F8172000F0D1F8182000F0CEF8192000F004
:40ED4000CBF81A2000F0C8F81B2000F0C5F81C2000F0C2F81D2000F0BFF81E2000F0BCF81F2000F0B9F8202000F0B6F8212000F0B3F8222000F0B0F8232000F0ADF82420C2
:40ED800000F0AAF8252000F0A7F8262000F0A4F8272000F0A1F8282000F09EF8292000F09BF82A2000F098F82B2000F095F82C2000F092F82D2000F08FF82E2000F08CF8D3
:40EDC0002F2000F089F8302000F086F8312000F083F8322000F080F8332000F07DF8342000F07AF8352000F077F8362000F074F8382000F071F8392000F06EF83A2000F0A1
:40EE00006BF83B2000F068F83C2000F065F83D2000F062F83E2000F05FF83F2000F05CF8402000F059F8412000F056F8422000F053F8432000F050F8442000F04DF84520B6
:40EE400000F04AF8462000F047F8472000F044F8482000F041F8492000F03EF84A2000F03BF84B2000F038F84C2000F035F84D2000F032F84E2000F02FF8502000F02CF8E7
:40EE8000512000F029F862B610BD00BF00BF00BF00BF00BFBFF34F8F00BF00BF00BF1348006800F4E06012490843001D0F49086000BF00BF00BFBFF34F8F00BF00BF00BFDF
:40EEC00000BF00BFFDE700F01F0201219140094A430942F82310704700F01F0201219140054A430942F82310704700000CED00E00000FA0580E100E080E200E02DE9F04184
:40EF000007460C460025012F02D0022F04D101E0C02602E0C42600E000BF00BF27B1012F2DD0022F49D12BE004F0010028B10121BA48007835F1F5FC04E00021B7480078BC
:40EF400035F1EFFC04F0020028B10121B448007835F1E7FC04E00021B148007835F1E1FC04F0040028B10121AE48007835F1D9FC04E00021AB48007835F1D3FC1EE000BF1B
:40EF800004F0010010B145F0030501E045F0010504F0020010B145F00C0501E045F0040504F0040010B145F0300501E045F010052946304636F1B8FE00E000BF00BFBDE813
:40EFC000F081024600210CE0974800EB01100078904205D1944800EB0110407B00B102E0491C0B29F0D300BFC8B27047F8B5044600250B2C5FD2DFE804F006101517282C09
:40F00000435153575C0089480AF098F8064641F288311CF0E1FA05464EE003F051F880F0010549E0012547E000200090804842F18AFA48B169467E4843F19BFB20B100984B
:40F0400074F110F900B1012536E041F197FE054632E0774843F14EFC00EE100AF8EE400A9FED741A80EE810AF2EE070AB4EEE00AF1EE10FA01D2012000E0002005461BE0E9
:40F080006B4843F137FC4FF47A7190FBF1F0102801DD012000E0002005460DE001250BE07AF154F9054607E0634814F037FF054602E0012500E000BF00BF2846F8BD70B554
:40F0C00000264FF4FA715D4800681CF085FA00287DD001265A48006880475849086059490978491CC9B2574A1170084601EBD0714910A0EB4101117000253BE0ECB22046A3
:40F10000FFF774FF78B3484800EB0410407B58B94B4800688047444901EB041188600120414901EB041148733F4800EB04104068F8B13D4A02EB0412526851083A4A02EB5C
:40F14000041290681CF048FA98B13E480078364901EB041108733A4800688047324901EB0411886005E0FFE700202F4901EB041148736D1C0B2DC1D30020FFF722FF0446E7
:40F180000B2C0FDA284A02EB0412521C264B03EB04131B7BD15C244A02EB04121078FFF7ADFE03E000210846FFF7A8FE0120FFF708FF04460B2C11DA1B4A02EB0412521C2B
:40F1C000194B03EB04131B7BD15C174A00E023E002EB04121078FFF791FE03E000210120FFF78CFE0220FFF7ECFE04460B2C0FDA0D4A02EB0412521C0B4B03EB04131B7BC5
:40F20000D15C094A02EB04121078FFF777FE03E000210220FFF772FE304670BDA8000010A6000010A70000106C0100202C3900206439001000007A44BC3D00201C02002030
:40F2400028030020200200202DE9F04104460025A01C02F052FF31287ED2DFE800F0193141537E8C9CBEC7FEFCFBFAF9F8F7F6F5F4F3F2F1F0EFEEEDECEBEAE9E8E7E6E559
:40F2800065AEE4E3E2E1E0DFDEDDDCDBDAD9D800E01D02F032FF064604F1080002F02DFF074604F1090002F028FF804606EB460040000A30022111FB070011FB080553E20F
:40F2C000A01D02F01AFF0646E01D02F016FF074606EB460040000830022111FB070543E204F1080002F009FF064604F1090002F004FF074606EB460040000A30022111FB37
:40F30000070531E204F1080002F0F7FE064604F1090002F0F2FE074606EB460040000A30022111FB07051FE204F10E0002F0E5FE064604F10F0002F0E0FE074604F110001A
:40F3400002F0DBFE804670001130062111FB0700022111FB080507E204E2201D02F0CDFE0646601D02F0C9FE07467000801D022111FB0705F8E1601D02F0BFFE0646A01DE7
:40F3800002F0BBFE074606EB46004000C01D022111FB0705E8E104F10B0002F0AEFE064604F10C0002F0A9FE074606EB460040000D30022111FB0705D6E104F1080002F097
:40F3C0009CFE064604F1090002F097FE074670000A30022111FB0705C6E104F10C0002F08CFE0646700000F10D05BDE104F1100002F083FE064604F11201881902F07DFE15
:40F40000074606F11300022111FB0705ACE1EAE065E1F1E056E1B2E070E16DE163E14FE142E133E153E0A8E09AE190E186E17CE172E165E155E11BE112E109E100E1F3E0F2
:40F44000F0E0AEE090E086E07CE06BE061E057E04DE033E01AE009E0FFE704F1250002F04CFE0646700000F126057DE104F10A0002F043FE064604F10C0002F03EFE0746AA
:40F4800070000D30022111FB07056DE104F10E0002F033FE804604F10F0002F02EFE08EB002086B204F11001881902F026FE074606F11100022111FB070555E104F11C0029
:40F4C00002F01BFE0646700000F11D054CE104F10A0002F012FE064604F10B0002F00DFE074670000C30022111FB07053CE104F10A0002F002FE0646700000F10B0533E1A8
:40F5000004F10C0002F0F9FD0646700000F10D052AE104F10E0002F0F0FD0646700000F10F0521E104F10C0002F0E7FD064604F10D0002F0E2FD0746B0000E30022111FB13
:40F54000070511E104F1140002F0D7FD0646700000F1150508E104F1170002F0CEFD0646700000F11805FFE004F11A0002F0C5FD0646700000F11B05F6E02225F4E004F126
:40F580000F0002F0BAFD064604F1100002F0B5FD074606EB460040001130022111FB0705E2E004F10C0002F0A8FD804604F10D0002F0A3FD08EB002804F10E0002F09DFD00
:40F5C00008EB004804F10F0002F097FD08EB006604F1100002F091FD074606F11100022111FB0705C0E004F10B0002F086FD0646700000F10C05B7E0201D02F07EFD074677
:40F60000601D02F07AFD07EB0027A01D02F075FD07EB0047E01D02F070FD07EB006606F10805A1E007259FE0E01C02F066FD0746201D02F062FD07EB002086B2751D93E012
:40F64000E01D02F05AFD0646700000F108058BE0E01D02F052FD0646700000F1080583E0E01D02F04AFD0646700000F108057BE0201D02F042FD0646611D881902F03DFD74
:40F680000746B01D022111FB07056DE0201D02F034FD0646611D881902F02FFD0746B01D042111FB07055FE0E01C02F026FD0746201D02F022FD07EB002086B2751D53E06E
:40F6C0000C2551E0201D02F018FD0746601D02F014FD07EB002086B2B000851D44E0092542E0052540E004F10C0002F006FD0646700000F10D0537E00C2535E0092533E0EA
:40F70000E01C02F0FAFC0746201D02F0F6FC07EB002086B2751D27E0601D02F0EEFC064606EB46004000851D1EE0A01D02F0E5FC064606EB46004000C51D15E0601D02F03F
:40F74000DCFC064606EB46004000851D0CE0601D02F0D3FC064606EB46004000851D03E0062501E0002500BF00BF2846BDE8F08170477047704770477047704770477047EF
:40F78000704770477047704770477047704770477047704770B5044601260125ACB1072C09DC601E05FA00F0C5B202F030FC284058B9002609E0A4F1080005FA00F0C5B265
:40F7C00002F028FC284000B90026304670BD70B50446254601E0681EC5B22846FFF7DAFF0028F8D0284670BD70B52DED028B044600259FEDF70AB0EE408A02F039FC10B171
:40F8000001280AD104E002F0F1FBB0EE408A04E002F0F0FBB0EE408A00BF00BF9FEDED0AB4EEC08AF1EE10FA0BDB9FEDEB0AB4EEC08AF1EE10FA04D82046FFF7C8FF054615
:40F84000F5E30F2C70D2DFE814F00F00BD003A01AB016802E502560304048604F704A405210692064A07C707B3EE080AB4EEC08AF1EE10FA04DB0E20FFF7A9FF0546A0E0F9
:40F880009FEDD60AB4EEC08AF1EE10FA04DB0D20FFF79DFF054694E0B3EE000AB4EEC08AF1EE10FA04DB0C20FFF791FF054688E0B2EE080AB4EEC08AF1EE10FA04DB0B2055
:40F8C000FFF785FF05467CE09FEDC50AB4EEC08AF1EE10FA04DB0A20FFF779FF054670E0B2EE000AB4EEC08AF1EE10FA04DB0920FFF76DFF054664E0B1EE080AB4EEC08A90
:40F90000F1EE10FA04DB0820FFF761FF054658E09FEDB40AB4EEC08AF1EE10FA05DB0720FFF755FF05464CE0DBE3B1EE000AB4EEC08AF1EE10FA04DB0620FFF748FF05464E
:40F940003FE0B0EE080AB4EEC08AF1EE10FA04DB0520FFF73CFF054633E09FEDA30AB4EEC08AF1EE10FA04DB0420FFF730FF054627E0B0EE000AB4EEC08AF1EE10FA04DB6C
:40F980000320FFF724FF05461BE0B7EE080AB4EEC08AF1EE10FA04DB0220FFF718FF05460FE09FED920AB4EEC08AF1EE10FA04DB0120FFF70CFF054603E02046FFF707FF63
:40F9C000054626E2B3EE080AB4EEC08AF1EE10FA04DB0E20FFF7FBFE05466FE0B3EE000AB4EEC08AF1EE10FA04DB0D20FFF7EFFE054663E0B2EE080AB4EEC08AF1EE10FA12
:40FA000004DB0B20FFF7E3FE054657E0B2EE000AB4EEC08AF1EE10FA04DB0A20FFF7D7FE05464BE0B1EE080AB4EEC08AF1EE10FA04DB0820FFF7CBFE05463FE0B1EE000A3B
:40FA4000B4EEC08AF1EE10FA04DB0720FFF7BFFE054633E0B0EE080AB4EEC08AF1EE10FA04DB0520FFF7B3FE054627E0B0EE000AB4EEC08AF1EE10FA04DB0420FFF7A7FEFD
:40FA800005461BE0B7EE080AB4EEC08AF1EE10FA04DB0220FFF79BFE05460FE0B7EE000AB4EEC08AF1EE10FA04DB0120FFF78FFE054603E00020FFF78AFE054681E7B3EE83
:40FAC000000AB4EEC08AF1EE10FA04DB0E20FFF77EFE054663E0B2EE080AB4EEC08AF1EE10FA04DB0C20FFF772FE054657E0B2EE000AB4EEC08AF1EE10FA04DB0B20FFF721
:40FB000066FE05464BE0B1EE080AB4EEC08AF1EE10FA04DB0920FFF75AFE05463FE0B1EE000AB4EEC08AF1EE10FA04DB0820FFF74EFE054633E0B0EE080AB4EEC08AF1EE05
:40FB400010FA04DB0620FFF742FE054627E0B0EE000AB4EEC08AF1EE10FA04DB0520FFF736FE05461BE0B7EE080AB4EEC08AF1EE10FA04DB0320FFF72AFE05460FE0B7EE72
:40FB8000000AB4EEC08AF1EE10FA04DB0220FFF71EFE054603E00020FFF719FE054610E7B2EE080AB4EEC08AF1EE10FA04DB0E20FFF70DFE0546AFE09FED090AB4EEC08ABC
:40FBC000F1EE10FA14DB0D20FFF701FE0546A3E000000000A4707D3FAE47813F52B8AA4152B82A4148E1AA4048E12A401F85AB3FB2EE000AB4EEC08AF1EE10FA04DB0C2090
:40FC0000FFF7E5FD054687E0B1EE080AB4EEC08AF1EE10FA04DB0B20FFF7D9FD05467BE01FED100AB4EEC08AF1EE10FA04DB0A20FFF7CDFD05466FE0B1EE000AB4EEC08A45
:40FC4000F1EE10FA04DB0920FFF7C1FD054663E0B0EE080AB4EEC08AF1EE10FA04DB0820FFF7B5FD054657E01FED210AB4EEC08AF1EE10FA04DB0720FFF7A9FD05464BE077
:40FC8000B0EE000AB4EEC08AF1EE10FA04DB0620FFF79DFD05463FE0B7EE080AB4EEC08AF1EE10FA04DB0520FFF791FD054633E01FED320AB4EEC08AF1EE10FA04DB042036
:40FCC000FFF785FD054627E0B7EE000AB4EEC08AF1EE10FA04DB0320FFF779FD05461BE0B6EE080AB4EEC08AF1EE10FA04DB0220FFF76DFD05460FE09FEDFA0AB4EEC08A60
:40FD0000F1EE10FA04DB0120FFF761FD054603E00020FFF75CFD054653E6B2EE080AB4EEC08AF1EE10FA04DB0E20FFF750FD05466FE0B2EE000AB4EEC08AF1EE10FA04DB96
:40FD40000D20FFF744FD054663E0B1EE080AB4EEC08AF1EE10FA04DB0B20FFF738FD054657E0B1EE000AB4EEC08AF1EE10FA04DB0A20FFF72CFD05464BE0B0EE080AB4EEE6
:40FD8000C08AF1EE10FA04DB0820FFF720FD05463FE0B0EE000AB4EEC08AF1EE10FA04DB0720FFF714FD054633E0B7EE080AB4EEC08AF1EE10FA04DB0520FFF708FD0546CE
:40FDC00027E0B7EE000AB4EEC08AF1EE10FA04DB0420FFF7FCFC05461BE0B6EE080AB4EEC08AF1EE10FA04DB0220FFF7F0FC05460FE0B6EE000AB4EEC08AF1EE10FA04DB37
:40FE00000120FFF7E4FC054603E00020FFF7DFFC054610E2B2EE000AB4EEC08AF1EE10FA04DB0E20FFF7D3FC054663E0B1EE080AB4EEC08AF1EE10FA04DB0C20FFF7C7FC46
:40FE4000054657E0B1EE000AB4EEC08AF1EE10FA04DB0B20FFF7BBFC05464BE0B0EE080AB4EEC08AF1EE10FA04DB0920FFF7AFFC05463FE0B0EE000AB4EEC08AF1EE10FA40
:40FE800004DB0820FFF7A3FC054633E0B7EE080AB4EEC08AF1EE10FA04DB0620FFF797FC054627E0B7EE000AB4EEC08AF1EE10FA04DB0520FFF78BFC05461BE0B6EE080ADB
:40FEC000B4EEC08AF1EE10FA04DB0320FFF77FFC05460FE0B6EE000AB4EEC08AF1EE10FA04DB0220FFF773FC054603E00020FFF76EFC05469FE1B1EE080AB4EEC08AF1EEA2
:40FF000010FA04DB0E20FFF762FC0546A0E01FEDCB0AB4EEC08AF1EE10FA04DB0D20FFF756FC054694E0B1EE000AB4EEC08AF1EE10FA04DB0C20FFF74AFC054688E0B0EEAC
:40FF4000080AB4EEC08AF1EE10FA04DB0B20FFF73EFC05467CE01FEDDC0AB4EEC08AF1EE10FA04DB0A20FFF732FC054670E0B0EE000AB4EEC08AF1EE10FA04DB0920FFF7AF
:40FF800026FC054664E0B7EE080AB4EEC08AF1EE10FA04DB0820FFF71AFC054658E01FEDED0AB4EEC08AF1EE10FA04DB0720FFF70EFC05464CE0B7EE000AB4EEC08AF1EE9F
:40FFC00010FA04DB0620FFF702FC054640E0B6EE080AB4EEC08AF1EE10FA04DB0520FFF7F6FB054634E09FED3F0AB4EEC08AF1EE10FA04DB0420FFF7EAFB054628E0B6EE3F
:020000040801F1
:40000000000AB4EEC08AF1EE10FA04DB0320FFF7DEFB05461CE0B5EE080AB4EEC08AF1EE10FA05DB0220FFF7D2FB054610E0F7E39FED2D0AB4EEC08AF1EE10FA04DB0120CD
:40004000FFF7C5FB054603E00020FFF7C0FB0546F1E0B1EE080AB4EEC08AF1EE10FA04DB0E20FFF7B4FB054674E0B1EE000AB4EEC08AF1EE10FA04DB0D20FFF7A8FB05466A
:4000800068E0B0EE080AB4EEC08AF1EE10FA04DB0B20FFF79CFB05465CE0B0EE000AB4EEC08AF1EE10FA04DB0A20FFF790FB054650E0B7EE080AB4EEC08AF1EE10FA04DB68
:4000C0000820FFF784FB054644E0B7EE000AB4EEC08AF1EE10FA09DB0720FFF778FB054638E0EBE31F852B3F7B14AE3EB6EE080AB4EEC08AF1EE10FA04DB0520FFF767FB5B
:40010000054627E0B6EE000AB4EEC08AF1EE10FA04DB0420FFF75BFB05461BE0B5EE080AB4EEC08AF1EE10FA04DB0220FFF74FFB05460FE0B5EE000AB4EEC08AF1EE10FACE
:4001400004DB0120FFF743FB054603E00020FFF73EFB0546B3E3B1EE000AB4EEC08AF1EE10FA04DB0E20FFF732FB054663E0B0EE080AB4EEC08AF1EE10FA04DB0C20FFF72B
:4001800026FB054657E0B0EE000AB4EEC08AF1EE10FA04DB0B20FFF71AFB05464BE0B7EE080AB4EEC08AF1EE10FA04DB0920FFF70EFB05463FE0B7EE000AB4EEC08AF1EE1D
:4001C00010FA04DB0820FFF702FB054633E0B6EE080AB4EEC08AF1EE10FA04DB0620FFF7F6FA054627E0B6EE000AB4EEC08AF1EE10FA04DB0520FFF7EAFA05461BE0B5EE8B
:40020000080AB4EEC08AF1EE10FA04DB0320FFF7DEFA05460FE0B5EE000AB4EEC08AF1EE10FA04DB0220FFF7D2FA054603E00020FFF7CDFA054642E3B0EE080AB4EEC08A71
:40024000F1EE10FA04DB0E20FFF7C1FA05469FE09FEDF70AB4EEC08AF1EE10FA04DB0D20FFF7B5FA054693E0B0EE000AB4EEC08AF1EE10FA04DB0C20FFF7A9FA054687E069
:40028000B7EE080AB4EEC08AF1EE10FA04DB0B20FFF79DFA05467BE09FEDE60AB4EEC08AF1EE10FA04DB0A20FFF791FA05466FE0B7EE000AB4EEC08AF1EE10FA04DB092074
:4002C000FFF785FA054663E0B6EE080AB4EEC08AF1EE10FA04DB0820FFF779FA054657E01FED800AB4EEC08AF1EE10FA04DB0720FFF76DFA05464BE0B6EE000AB4EEC08AA0
:40030000F1EE10FA04DB0620FFF761FA05463FE0B5EE080AB4EEC08AF1EE10FA04DB0520FFF755FA054633E01FED910AB4EEC08AF1EE10FA04DB0420FFF749FA054627E0D9
:40034000B5EE000AB4EEC08AF1EE10FA04DB0320FFF73DFA05461BE0B4EE080AB4EEC08AF1EE10FA04DB0220FFF731FA05460FE09FEDB10AB4EEC08AF1EE10FA04DB012085
:40038000FFF725FA054603E00020FFF720FA054695E2B0EE080AB4EEC08AF1EE10FA04DB0E20FFF714FA05466FE0B0EE000AB4EEC08AF1EE10FA04DB0D20FFF708FA05460C
:4003C00063E0B7EE080AB4EEC08AF1EE10FA04DB0B20FFF7FCF9054657E0B7EE000AB4EEC08AF1EE10FA04DB0A20FFF7F0F905464BE0B6EE080AB4EEC08AF1EE10FA04DB6B
:400400000820FFF7E4F905463FE0B6EE000AB4EEC08AF1EE10FA04DB0720FFF7D8F9054633E0B5EE080AB4EEC08AF1EE10FA04DB0520FFF7CCF9054627E0B5EE000AB4EEBF
:40044000C08AF1EE10FA04DB0420FFF7C0F905461BE0B4EE080AB4EEC08AF1EE10FA04DB0220FFF7B4F905460FE0B4EE000AB4EEC08AF1EE10FA04DB0120FFF7A8F9054687
:4004800003E00020FFF7A3F9054618E2B0EE000AB4EEC08AF1EE10FA04DB0E20FFF797F9054663E0B7EE080AB4EEC08AF1EE10FA04DB0C20FFF78BF9054657E0B7EE000A82
:4004C000B4EEC08AF1EE10FA04DB0B20FFF77FF905464BE0B6EE080AB4EEC08AF1EE10FA04DB0920FFF773F905463FE0B6EE000AB4EEC08AF1EE10FA04DB0820FFF767F9FA
:40050000054633E0B5EE080AB4EEC08AF1EE10FA04DB0620FFF75BF9054627E0B5EE000AB4EEC08AF1EE10FA04DB0520FFF74FF905461BE0B4EE080AB4EEC08AF1EE10FA9F
:4005400004DB0320FFF743F905460FE0B4EE000AB4EEC08AF1EE10FA04DB0220FFF737F9054603E00020FFF732F90546A7E1B7EE080AB4EEC08AF1EE10FA04DB0E20FFF794
:4005800026F90546AAE09FED2B0AB4EEC08AF1EE10FA04DB0D20FFF71AF905469EE0B7EE000AB4EEC08AF1EE10FA04DB0C20FFF70EF9054692E0B6EE080AB4EEC08AF1EE09
:4005C00010FA04DB0B20FFF702F9054686E09FED1B0AB4EEC08AF1EE10FA04DB0A20FFF7F6F805467AE0B6EE000AB4EEC08AF1EE10FA04DB0920FFF7EAF805466EE0B5EE8E
:40060000080AB4EEC08AF1EE10FA04DB0820FFF7DEF8054662E09FED0A0AB4EEC08AF1EE10FA0FDB0720FFF7D2F8054656E0000048E12A401F85AB3F0C022B3E1F852B3F06
:400640007B14AE3EB5EE000AB4EEC08AF1EE10FA04DB0620FFF7BBF805463FE0B4EE080AB4EEC08AF1EE10FA04DB0520FFF7AFF8054633E01FED100AB4EEC08AF1EE10FAE2
:4006800004DB0420FFF7A3F8054627E0B4EE000AB4EEC08AF1EE10FA04DB0320FFF797F805461BE09FEDFE0AB4EEC08AF1EE10FA04DB0220FFF78BF805460FE09FEDF90A5A
:4006C000B4EEC08AF1EE10FA04DB0120FFF77FF8054603E00020FFF77AF80546EFE0B7EE080AB4EEC08AF1EE10FA04DB0E20FFF76EF805466FE0B7EE000AB4EEC08AF1EEDF
:4007000010FA04DB0D20FFF762F8054663E0B6EE080AB4EEC08AF1EE10FA04DB0B20FFF756F8054657E0B6EE000AB4EEC08AF1EE10FA04DB0A20FFF74AF805464BE0B5EE8D
:40074000080AB4EEC08AF1EE10FA04DB0820FFF73EF805463FE0B5EE000AB4EEC08AF1EE10FA04DB0720FFF732F8054633E0B4EE080AB4EEC08AF1EE10FA04DB0520FFF76C
:4007800026F8054627E0B4EE000AB4EEC08AF1EE10FA04DB0420FFF71AF805461BE09FEDC00AB4EEC08AF1EE10FA04DB0220FFF70EF805460FE09FEDBC0AB4EEC08AF1EE78
:4007C00010FA04DB0120FFF702F8054603E00020FEF7FDFF054672E0B7EE000AB4EEC08AF1EE10FA04DB0E20FEF7F1FF054664E0B6EE080AB4EEC08AF1EE10FA04DB0C2088
:40080000FEF7E5FF054658E0B6EE000AB4EEC08AF1EE10FA05DB0B20FEF7D9FF05464CE04EE0B5EE080AB4EEC08AF1EE10FA04DB0920FEF7CCFF05463FE0B5EE000AB4EE51
:40084000C08AF1EE10FA04DB0820FEF7C0FF054633E0B4EE080AB4EEC08AF1EE10FA04DB0620FEF7B4FF054627E0B4EE000AB4EEC08AF1EE10FA04DB0520FEF7A8FF054638
:400880001BE09FED870AB4EEC08AF1EE10FA04DB0320FEF79CFF05460FE09FED830AB4EEC08AF1EE10FA04DB0220FEF790FF054603E00020FEF78BFF054600E000BF00BF96
:4008C0002846BDEC028B70BD30B5039C994204D3CD1AA54201D2CD1A425530BD2DE9F84304460D4616461F46201D01F006FC8146FEF77AFF804633464246042128460097E0
:40090000FFF7E2FFBDE8F88370477047704770B504460D46002615B1012D2FD111E001F065FBF0EE400A00EE104AB8EE401AB6EE000A01EE200ABCEEC00A10EE100A86B282
:400940001CE001F057FBF7EE000AB4EEE00AF1EE10FA11D201F04EFBF0EE400A00EE104AB8EE401AB6EE000A01EE200ABCEEC00A10EE100A86B200E0264600BF00BF30467C
:4009800070BD2DE9F84304460F4690461D46E01C01F0B3FB8146201D01F0AFFB09EB002086B201F065FB814649463046FFF7AFFF0646F2B24346032138460095FFF784FF71
:4009C00032124346042138460095FFF77DFF601D01F093FB8146A01D01F08FFB09EB002086B201F045FB814649463046FFF78FFF0646F2B24346052138460095FFF764FFAD
:400A000032124346062138460095FFF75DFFBDE8F8832DE9F84304460F4690461D46E01C01F06BFB8146201D01F067FB09EB002086B201F01DFB814649463046FFF767FFED
:400A40000646F2B24346032138460095FFF73CFF32124346042138460095FFF735FFBDE8F883704770472DE9F84304460F4690461D46E01C01F041FB8146201D01F03DFB59
:400A800009EB002086B201F0F3FA814649463046FFF73DFF0646F2B243460321384605E00000C03D9FCDAA3D0000803D0095FFF70BFF32124346042138460095FFF704FF6E
:400AC000601D01F01AFB8146A01D01F016FB09EB002086B201F0CCFA814649463046FFF716FF0646F2B24346052138460095FFF7EBFE32124346062138460095FFF7E4FEA3
:400B000004F10C0001F0F9FA814604F10D0001F0F4FA09EB002086B201F0AAFA814649463046FFF7F4FE0646F2B243460C2138460095FFF7C9FE321243460D21384600950F
:400B4000FFF7C2FEBDE8F8832DE9F84304460F4690461D46E01C01F0D0FA8146201D01F0CCFA09EB002086B201F082FA814649463046FFF7CCFE0646F2B2434603213846A4
:400B80000095FFF7A1FE32124346042138460095FFF79AFE601D01F0B0FA8146A01D01F0ACFA09EB002086B201F062FA814649463046FFF7ACFE0646F2B243460521384623
:400BC0000095FFF781FE32124346062138460095FFF77AFEBDE8F8832DE9F84304460F4690461D46E01C01F088FA8146201D01F084FA09EB002086B201F03AFA8146494684
:400C00003046FFF784FE0646F2B24346032138460095FFF759FE32124346042138460095FFF752FEBDE8F8832DE9F0412DED048B04460D461646002715B1052D5DD100E048
:400C400000BF01F0D7F9F7EE000AB4EEE00AF1EE10FA24D201F0E7F900EE100AF8EE408A01F0C8F9B0EE409A79F152F800EE100AF8EE400AB0EE680A09EE600AF0EE000AA2
:400C8000C0EE208A01F0B6F9F0EE400A00EE104AB8EEC00AB0EE688A00EE208A17E001F0C2F900EE100AF8EE408A79F131F800EE100AB8EE400A38EEC00AB0EE001AC0EEF8
:400CC000010A00EE104AB8EEC00A30EE808A002C09DAB6EE000A38EE400ABDEEC00A10EE100A07B208E0B6EE000A38EE000ABDEEC00A10EE100A07B251E016B1012E4CD146
:400D000025E0002C11DA01F071F9F0EE400A00EE104AB8EEC01AB6EE000A11EE200ABDEEC00A10EE100A07B210E001F05FF9F0EE400A00EE104AB8EEC01AB6EE000A01EE69
:400D4000200ABDEEC00A10EE100A07B225E0002C11DA01F04FF9F0EE400A00EE104AB8EEC01AB6EE000A11EE200ABDEEC00A10EE100A07B210E001F03DF9F0EE400A00EE74
:400D8000104AB8EEC01AB6EE000A01EE200ABDEEC00A10EE100A07B200BF00BF00BF00BF3846BDEC048BBDE8F0812DE9F0412DED048B04460D461646002715B1052D5DD14E
:400DC00000E000BF01F016F9F7EE000AB4EEE00AF1EE10FA24D201F023F900EE100AF8EE408A01F007F9B0EE409A78F18FFF00EE100AF8EE400AB0EE680A09EE600AF0EE4E
:400E0000000AC0EE208A01F0F5F8F0EE400A00EE104AB8EEC00AB0EE688A00EE208A17E001F0FEF800EE100AF8EE408A78F16EFF00EE100AB8EE400A38EEC00AB0EE001A5E
:400E4000C0EE010A00EE104AB8EEC00A30EE808A002C09DAB6EE000A38EE400ABDEEC00A10EE100A07B208E0B6EE000A38EE000ABDEEC00A10EE100A07B251E016B1012E33
:400E80004CD125E0002C11DA01F0B0F8F0EE400A00EE104AB8EEC01AB6EE000A11EE200ABDEEC00A10EE100A07B210E001F09EF8F0EE400A00EE104AB8EEC01AB6EE000A3E
:400EC00001EE200ABDEEC00A10EE100A07B225E0002C11DA01F08EF8F0EE400A00EE104AB8EEC01AB6EE000A11EE200ABDEEC00A10EE100A07B210E001F07CF8F0EE400A76
:400F000000EE104AB8EEC01AB6EE000A01EE200ABDEEC00A10EE100A07B200BF00BF00BF00BF3846BDEC048BBDE8F0812DE9F84F0646884691461F4606F10C0001F0DDF898
:400F40008246F01C01F0D9F88346301D01F0D5F80BEB002085B201F08BF8834659462846FFF7D5FC0546EAB24B46032140460097FFF7AAFC2A124B46042140460097FFF74F
:400F8000A3FC701D01F0B9F88346B01D01F0B5F80BEB002085B201F06BF8834659462846FFF7B5FC0546EAB24B46052140460097FFF78AFC2A124B46062140460097FFF7D3
:400FC00083FC002457E00E2101EB8401881901F094F883460F2101EB8401881901F08DF80BEB002085B201F043F883465A46102128B2FFF7DAFE85B2EAB20E2000EB8401AC
:401000004B4640460097FFF75FFC2A120F2000EB84014B4640460097FFF756FC102101EB8401881901F069F88346112101EB8401881901F062F80BEB002085B201F018F8A5
:4010400083465A46102128B2FFF7EEFD85B2EAB2102000EB84014B4640460097FFF734FC2A12112000EB84014B4640460097FFF72BFC601CC4B25445A5DBBDE8F88F2DE9DF
:40108000F84304460F4690461D46601D01F035F88146A01D01F031F809EB002086B200F0E7FF814649463046FFF731FC0646F2B24346052138460095FFF706FC321243465C
:4010C000062138460095FFF7FFFBE01D01F015F8814604F1080001F010F809EB002086B200F0C6FF814649463046FFF710FC0646F2B24346072138460095FFF7E5FB321271
:401100004346082138460095FFF7DEFBBDE8F8832DE9F84304460F4690461D46601D00F0ECFF8146A01D00F0E8FF09EB002086B200F09EFF814649463046FFF7E8FB064655
:40114000F2B24346052138460095FFF7BDFB32124346062138460095FFF7B6FBE01D00F0CCFF814604F1080000F0C7FF09EB002086B200F07DFF814649463046FFF7C7FB3F
:401180000646F2B24346072138460095FFF79CFB32124346082138460095FFF795FBBDE8F8832DE9F84304460F4690461D46601D00F0A3FF8146A01D00F09FFF09EB0020E1
:4011C00086B200F055FF814649463046FFF79FFB0646F2B24346052138460095FFF774FB32124346062138460095FFF76DFBE01D00F083FF814604F1080000F07EFF09EB07
:40120000002086B200F034FF814649463046FFF77EFB0646F2B24346072138460095FFF753FB32124346082138460095FFF74CFBBDE8F8832DE9F84304460F4690461D4671
:40124000E01C00F05AFF8146201D00F056FF09EB002086B200F00CFF814649463046FFF756FB0646F2B24346032138460095FFF72BFB32124346042138460095FFF724FBA0
:40128000601D00F03AFF8146A01D00F036FF09EB002086B200F0ECFE814649463046FFF736FB0646F2B24346052138460095FFF70BFB32124346062138460095FFF704FB1C
:4012C000BDE8F8832DE9F84304460F4690461D46E01C00F012FF8146201D00F00EFF09EB002086B200F0C4FE814649463046FFF70EFB0646F2B24346032138460095FFF738
:40130000E3FA32124346042138460095FFF7DCFA601D00F0F2FE8146A01D00F0EEFE09EB002086B200F0A4FE814649463046FFF7EEFA0646F2B24346052138460095FFF712
:40134000C3FA32124346062138460095FFF7BCFABDE8F8832DE9F84304460F4690461D46E01C00F0CAFE8146201D00F0C6FE09EB002086B200F07CFE814649463046FFF7D0
:40138000C6FA0646F2B24346032138460095FFF79BFA32124346042138460095FFF794FA601D00F0AAFE8146A01D00F0A6FE09EB002086B200F05CFE814649463046FFF724
:4013C000A6FA0646F2B24346052138460095FFF77BFA32124346062138460095FFF774FABDE8F8832DE9F84304460F4690461D46E01C00F082FE8146201D00F07EFE09EBAC
:40140000002086B200F034FE814649463046FFF77EFA0646F2B24346032138460095FFF753FA32124346042138460095FFF74CFA601D00F062FE8146A01D00F05EFE09EB33
:40144000002086B200F014FE814649463046FFF75EFA0646F2B24346052138460095FFF733FA32124346062138460095FFF72CFABDE8F8832DE9F84304460F4690461D46B7
:40148000E01C00F03AFE8146201D00F036FE09EB002086B200F0ECFD814649463046FFF736FA0646F2B24346032138460095FFF70BFA32124346042138460095FFF704FA25
:4014C000601D00F01AFE8146A01D00F016FE09EB002086B200F0CCFD814649463046FFF716FA0646F2B24346052138460095FFF7EBF932124346062138460095FFF7E4F9A2
:40150000BDE8F8832DE9F84304460F4690461D46E01C00F0F2FD8146201D00F0EEFD09EB002086B200F0A4FD814649463046FFF7EEF90646F2B24346032138460095FFF77C
:40154000C3F932124346042138460095FFF7BCF9601D00F0D2FD8146A01D00F0CEFD09EB002086B200F084FD814649463046FFF7CEF90646F2B24346052138460095FFF796
:40158000A3F932124346062138460095FFF79CF9BDE8F8832DE9F84304460F4690461D46201D00F0AAFD8146601D00F0A6FD09EB002086B200F05CFD814649463046FFF7B2
:4015C000A6F90646F2B24346042138460095FFF77BF932124346052138460095FFF774F9BDE8F88370472DE9FC5F0446894692461E4604F10B0000F080FD0190E01C00F041
:401600007CFD8346201D00F078FD0BEB002087B200F02EFD834659463846FFF778F90746FAB25346032148460096FFF74DF93A125346042148460096FFF746F9601D00F029
:401640005CFD8346A01D00F058FD0BEB002087B200F00EFD834659463846FFF758F90746FAB25346052148460096FFF72DF93A125346062148460096FFF726F900256DE020
:4016800005EB45010F2202EB4101081900F035FD834605EB4501102202EB4101081900F02CFD0BEB00200FFA80F800F0E1FC83465A4606214046FFF778FB804608F0FF0215
:4016C00005EB45000F2303EB4001534648460096FFF7FAF805EB4500102202EB40015346C8F3072248460096FFF7EEF805EB4501112202EB4101081900F0FFFC834605EB40
:401700004501122202EB4101081900F0F6FC0BEB00200FFA80F800F0ABFC83465A4606214046FFF781FA804608F0FF0205EB4500112303EB4001534648460096FFF7C4F882
:4017400005EB4500122202EB40015346C8F3072248460096FFF7B8F8681CC5B2019885428EDBBDE8FC9F2DE9F84F0546884691461E46681D00F0C1FC8246002469E004EB80
:401780004401092202EB4101481900F0B6FC834604EB44010A2202EB4101481900F0ADFC0BEB002007B200F063FC83465A4605213846FFF7FAFA0746FAB204EB44000923C8
:4017C00003EB40014B4640460096FFF77DF804EB44000A2202EB40014B46C7F3072240460096FFF771F804EB44010B2202EB4101481900F082FC834604EB44010C2202EBAF
:401800004101481900F079FC0BEB002007B200F02FFC83465A4605213846FFF705FA0746FAB204EB44000B2303EB40014B4640460096FFF749F804EB44000C2202EB4001B8
:401840004B46C7F3072240460096FFF73DF8601CC4B2544593DBBDE8F88F704770472DE9FC5F0446894692461E4604F1080000F044FC0190E01C00F040FC8346201D00F078
:401880003CFC0BEB002087B200F0F2FB834659463846FFF73CF80746FAB25346032148460096FFF711F83A125346042148460096FFF70AF8601D00F020FC8346A01D00F0B6
:4018C0001CFC0BEB002087B200F0D2FB834659463846FFF71CF80746FAB25346052148460096FEF7F1FF3A125346062148460096FEF7EAFF00256DE005EB45010C2202EB42
:401900004101081900F0F9FB834605EB45010D2202EB4101081900F0F0FB0BEB00200FFA80F800F0A5FB83465A4603214046FFF73CFA804608F0FF0205EB45000C2303EB90
:401940004001534648460096FEF7BEFF05EB45000D2202EB40015346C8F3072248460096FEF7B2FF05EB45010E2202EB4101081900F0C3FB834605EB45010F2202EB41011B
:40198000081900F0BAFB0BEB00200FFA80F800F06FFB83465A4603214046FFF745F9804608F0FF0205EB45000E2303EB4001534648460096FEF788FF05EB45000F2202EB49
:4019C00040015346C8F3072248460096FEF77CFF681CC5B2019885428EDBBDE8FC9F2DE9F84F0546884691461E4605F1080000F084FB8246002469E004EB44010C2202EBEF
:401A00004101481900F079FB834604EB44010D2202EB4101481900F070FB0BEB002007B200F026FB83465A4602213846FFF7BDF90746FAB204EB44000C2303EB40014B46D7
:401A400040460096FEF740FF04EB44000D2202EB40014B46C7F3072240460096FEF734FF04EB44010E2202EB4101481900F045FB834604EB44010F2202EB4101481900F0FC
:401A80003CFB0BEB002007B200F0F2FA83465A4602213846FFF7C8F80746FAB204EB44000E2303EB40014B4640460096FEF70CFF04EB44000F2202EB40014B46C7F3072245
:401AC00040460096FEF700FF601CC4B2544593DBBDE8F88F2DE9F84F0546884691461E46A81D00F00AFB8246002469E004EB44010A2202EB4101481900F0FFFA834604EB80
:401B000044010B2202EB4101481900F0F6FA0BEB002007B200F0ACFA83465A4601213846FFF743F90746FAB204EB44000A2303EB40014B4640460096FEF7C6FE04EB440002
:401B40000B2202EB40014B46C7F3072240460096FEF7BAFE04EB44010C2202EB4101481900F0CBFA834604EB44010D2202EB4101481900F0C2FA0BEB002007B200F078FA8D
:401B800083465A4601213846FFF74EF80746FAB204EB44000C2303EB40014B4640460096FEF792FE04EB44000D2202EB40014B46C7F3072240460096FEF786FE601CC4B299
:401BC000544593DBBDE8F88F2DE9F84F0546884691461E46E81D00F090FA8246002469E004EB44010C2202EB4101481900F085FA834604EB44010D2202EB4101481900F040
:401C00007CFA0BEB002007B200F032FA83465A4600213846FFF7C9F80746FAB204EB44000C2303EB40014B4640460096FEF74CFE04EB44000D2202EB40014B46C7F307220A
:401C400040460096FEF740FE04EB44010E2202EB4101481900F051FA834604EB44010F2202EB4101481900F048FA0BEB002007B200F0FEF983465A4600213846FEF7D4FF70
:401C80000746FAB204EB44000E2303EB40014B4640460096FEF718FE04EB44000F2202EB40014B46C7F3072240460096FEF70CFE601CC4B2544593DBBDE8F88F2DE9F04153
:401CC00004460D4616461F46A01C00F016FA312875D2DFE800F01920272E3C434A585F666D757C8A91989FA6ADB4C9F3FAF0EFEEEDECEBEAE9E8E7E63551BB83E5E4E3E227
:401D0000E1E0C2DFD7DED0003B46324629462046FFF75AFF66E13B46324629462046FFF7D9FE5FE13B46324629462046FFF757FE58E13B46324629462046FFF790FD51E1A8
:401D40003B46324629462046FFF788FD4AE13B46324629462046FFF780FD43E13B46324629462046FFF7FFFC3CE13B46324629462046FFF738FC35E13B46324629462046D2
:401D8000FFF730FC2EE13B46324629462046FFF701FC27E13B46324629462046FFF7B2FB20E13B46324629462046FFF763FB19E13B46324629462046FFF714FB12E110E1E4
:401DC0003B46324629462046FFF7C4FA0AE13B46324629462046FFF775FA03E13B46324629462046FFF726FAFCE03B46324629462046FFF7D6F9F5E03B4632462946204669
:401E0000FFF786F9EEE03B46324629462046FFF736F9E7E03B46324629462046FFF786F8E0E03B46324629462046FEF7D5FED9E03B46324629462046FEF786FED2E03B46DA
:401E4000324629462046FEF70EFECBE03B46324629462046FEF706FEC4E03B46324629462046FEF7FEFDBDE03B46324629462046FEF7CFFDB6E03B46324629462046FEF7BB
:401E800080FDAFE03B46324629462046FEF73EFDA8E059E051E073E06BE063E046E03EE036E097E08FE087E07FE077E06FE052E027E01FE017E00FE007E0FFE73B463246B5
:401EC00029462046FEF721FD8CE03B46324629462046FEF719FD85E03B46324629462046FEF7FCFC7EE03B46324629462046FDF750FC77E03B46324629462046FDF748FCCC
:401F000070E03B46324629462046FDF740FC69E03B46324629462046FDF738FC62E03B46324629462046FDF730FC5BE03B46324629462046FDF728FC54E03B463246294627
:401F40002046FDF720FC4DE03B46324629462046FDF718FC46E03B46324629462046FDF710FC3FE03B46324629462046FDF708FC38E03B46324629462046FDF700FC31E028
:401F80003B46324629462046FDF7F8FB2AE03B46324629462046FDF7F0FB23E03B46324629462046FDF7E8FB1CE03B46324629462046FDF7E0FB15E03B46324629462046B1
:401FC000FDF7D8FB0EE03B46324629462046FDF7D0FB07E03B46324629462046FDF7C8FB00E000BF00BFBDE8F0810000FE4890ED000A7047FC4890ED010A7047FA480089ED
:402000007047F948807A7047F748C07A7047F648007B7047F448407B7047F348807B7047F148C07B7047F048007C7047EE48807C7047ED48407C7047EB48C07C704700204F
:40204000E94991F8C310042906DAE74991F8C320283101EB0211087B704700B5FFF7EFFF00BDE148008C7047DF4890F824007047DD4890F890007047DB4981F89000704773
:40208000D94890F8C2007047D74890F8EA007047D54981F8EA007047D34890F8E8007047D14981F8E8007047CF4890F8E9007047CD4981F8E9007047CB4890F88E007047BC
:4020C00000B50021FFF7F8FF2D2800D10121084600BDC6484078C5490978884201D1012070470020FCE701460020BF4AD27C8A4202DB032900DC0120704770B50446002523
:40210000B94890F88D00072846D2DFE800F046040C161E2B3800B44991F8B800214677F132FD05463AE0B04AB2F8B41092F8B900224677F141FD054630E0AB4991F8BA00B2
:40214000214677F178FD054628E00420FFF7CBFF0646A54991F8BB002246314677F16EFD05461BE00520FFF7BEFF06469E4991F8BB002246314677F164FD05460EE0062018
:40218000FFF7B1FF0646984991F8BB002246314677F15AFD054601E000BF00BF00BF284670BD2DE9F05F8146884692469B460025BBF1010F04D100208D4908608D49086061
:4021C0008C480068A9EB0000504504D289480068A9EB000400E05446002607E0854909688819FFF78AFF08F80600761CA642F5D333E07F480068FDF727F807467C480068D7
:402200007C490968884217D2601B83B279480068DFF8DCC1DCF800C0A0EB0C0208EB050173480068FFF74AFD7248006870490968401A381A054409E0601B83B208EB05010F
:4022400000226B480068FFF739FD3D44A54204D267480068384466490860A542C9D3654800682044634908602046BDE8F09F2DE9F04705460C4616460027B8465A4890F8CE
:402280008D00072840D2DFE800F040040B141B273300554991F8B80077F1D9FC804635E0514AB2F8B41092F8B90077F1E6FC80462CE04D4991F8BA0077F117FD804625E042
:4022C0000420FFF710FF8146474991F8BB00494677F10EFD804619E00520FFF704FF8146414991F8BB00494677F105FD80460DE00620FFF7F8FE81463B4991F8BB004946CA
:4023000077F1FCFC804601E000BF00BF00BF012D09D111202070721E0123611C4046FFF740FF471C06E00023324621464046FFF738FF07463846BDE8F0872DE9F04104462E
:402340000D4616461F464FF00008052C15D2DFE804F0080903040A0000BF234880F88F400BE000BF00BF204880F88F403A4631462846FFF77CFF804600BF00BF4046BDE83F
:40238000F081002019490978491C184A527891427BD0164949783131144A127891427CD001204FF467421149097801EB81030F49091D21F823209222091F097801EB810372
:4023C0000A49091D01EB83018A72FF220749097801EB81030549091D01EB8301CA720349097801EB810307E0683D0010583E00102402002028020020F94901EB83010A7338
:40240000F749091F097801EB8103F54901EB83014A73F349091F097801EB8103F04901EB83018A73EE49091F097801EB8103EC4901EB8301CA73EA49091F097801EB81035F
:40244000E74901EB83010A74E549091F097801EB8103E34901EB83014A740822E049091F097801EB8103DE4901EB83010A81DC49091F0978491C322908DBD949091F497893
:4024800019B10021D64A121F117006E0D449091F0978491CD24A121F1170704730B502460020CF4B1B1F1B785B1CCD4C241F6478A3427DD0CA4B1B1F5B783133C84C241FD7
:4024C0002478A34274D001204FF46744C44B1B1F1B7803EB8305C24B23F82540A0241B1F1B7803EB8305BE4B03EB85039C72BC4B1B1F1B7803EB8305B94B03EB8503DA7285
:402500001412B74B1B1F1B7803EB8305B44B03EB85031C73B24B1B1F1B7803EB8304B04B03EB84035973FF24AD4B1B1F1B7803EB8305AB4B03EB85039C73A94B1B1F1B7817
:4025400003EB8305A64B03EB8503DC73A44B1B1F1B7803EB8305A24B03EB85031C74A04B1B1F1B7803EB83059D4B03EB85035C7408249B4B1B1F1B7803EB8305984B03EB88
:4025800085031C81964B1B1F1B785B1C322B08DB934B1B1F5B781BB10023914C241F237006E08F4B1B1F1B785B1C8D4C241F237030BD30B502460020894B1B1F1B785B1CFF
:4025C000874C241F6478A3427DD0854B1B1F5B783133834C241F2478A34274D001204FF467447F4B1B1F1B7803EB83057C4B23F82540A1241B1F1B7803EB8305784B03EB83
:4026000085039C72764B1B1F1B7803EB8305744B03EB8503DA721412714B1B1F1B7803EB83056F4B03EB85031C736D4B1B1F1B7803EB83046A4B03EB84035973FF24684BD5
:402640001B1F1B7803EB8305654B03EB85039C73634B1B1F1B7803EB8305614B03EB8503DC735F4B1B1F1B7803EB83055C4B03EB85031C745A4B1B1F1B7803EB8305584B5B
:4026800003EB85035C740824554B1B1F1B7803EB8305534B03EB85031C81514B1B1F1B785B1C322B08DB4E4B1B1F5B781BB100234B4C241F237006E0494B1B1F1B785B1C34
:4026C000474C241F237030BD30B502460020444B1B1F1B785B1C424C241F6478A3427DD03F4B1B1F5B7831333D4C241F2478A34274D001204FF46744394B1B1F1B7803EBAB
:402700008305374B23F82540A2241B1F1B7803EB8305334B03EB85039C72314B1B1F1B7803EB83052E4B03EB8503DA7214122C4B1B1F1B7803EB8305294B03EB85031C73B1
:40274000274B1B1F1B7803EB8304254B03EB84035973FF24224B1B1F1B7803EB8305204B03EB85039C731E4B1B1F1B7803EB83051B4B03EB8503DC73194B1B1F1B7803EB3B
:402780008305174B03EB85031C74154B1B1F1B7803EB8305124B03EB85035C740824104B1B1F1B7803EB83050D4B03EB85031C810B4B1B1F1B785B1C322B08DB084B1B1F47
:4027C0005B781BB10023064C241F237006E0044B1B1F1B785B1C024C241F237030BD00005C3E0010F0B504460020FE4D2D786D1CFC4E7678B54278D0FA4D6D783135F94EE3
:402800003678B54271D001204FF46746F54D2D7805EB8507F34D2D1D25F82760A3262D1F2D7805EB8507EF4D2D1D05EB8705AE72EC4D2D7805EB8506EA4D2D1D05EB860563
:40284000EC72E84D2D7805EB8507E64D2D1D05EB870529730E12E34D2D7805EB8507E14D2D1D05EB87056E73DE4D2D7805EB8507DC4D2D1D05EB8705AA731612D94D2D787E
:4028800005EB8507D74D2D1D05EB8705EE73D54D2D7805EB8507D34D2D1D05EB87052B741E12D04D2D7805EB8507CE4D2D1D05EB87056E740826CB4D2D7805EB8507C94DDB
:4028C0002D1D05EB87052E81C64D2D786D1C322D06DBC44D6D7815B10025C24E357004E0C04D2D786D1CBF4E3570F0BD10B501460020BC4A1278521CBA4B5B789A4276D0AA
:40290000B84A52783132B74B1B789A426FD001204FF46743B34A127802EB8204B14A121D22F82430A423121F127802EB8204AD4A121D02EB84029372AA4A127802EB820395
:40294000A84A121D02EB8302D172FF23A54A127802EB8204A34A121D02EB84021373A14A127802EB82049F4A121D02EB840253739C4A127802EB82049A4A121D02EB8402BC
:402980009373984A127802EB8204964A121D02EB8402D373934A127802EB8204914A121D02EB840213748F4A127802EB82048D4A121D02EB8402537408238A4A127802EB00
:4029C0008204884A121D02EB84021381854A1278521C322A06DB834A527812B10022814B1A7004E07F4A1278521C7E4B1A7010BD2DE9F04704460D4616461F46DDF820808E
:402A00004FF0000977480078401C7649497888427ED0744840783130724909788842F7D0B0B24146FDF773FF46B2B8B24146FDF76EFF47B24FF001094FF467416948007892
:402A400000EB80026748001D20F82210A521001F007800EB80026348001D00EB820081726048007800EB80025E48001D00EB8200C47221125B48007800EB80025948001D75
:402A800000EB820001735748007800EB80025548001D00EB8200457329125248007800EB80025048001D00EB8200817306F17F00C1B24C48007800EB80024A48001D00EB06
:402AC0008200C17307F17F00C1B24648007800EB80024448001D00EB82000174FF214148007800EB80023F48001D00EB8200417408213C48007800EB80023A48001D00EBC8
:402B00008200018137480078401C322808DB00E00BE03448407840B100203249087004E030480078401C2F4908704846BDE8F0872DE9F04706460F4614461D46DDE9088932
:402B40004FF0000A27480078401C2649497888427ED0244840783130224909788842F7D04A4641462046FEF720F904464A4641462846FEF759F805464FF0010A4FF467415F
:402B80001848007800EB80021648001D20F82210B421001F007800EB80021248001D00EB820081720F48007800EB80020D48001D00EB8200C67231120A48007800EB80028E
:402BC0000848001D00EB820001730648007800EB80020448001D00EB8200477339120148007801E0583E001000EB8002FE4800EB82008173FC48001F007800EB8002FA4893
:402C000000EB8200C473210AF748001F007800EB8002F54800EB82000174F348001F007800EB8002F04800EB82004574290AEE48001F007800EB8002EB4800EB82008174C4
:402C40000921E948001F007800EB8002E64800E018E000EB82000181E348001F0078401C322808DBE048001F407858B10020DE49091F087006E0DC48001F0078401CDA4996
:402C8000091F08705046BDE8F0872DE9F04106460C4615461F464FF00008D348001F0078401CD149091F497888427DD0CE48001F40783130CC49091F0978884274D0394615
:402CC0002046FDF724FE044639462846FDF71FFE05464FF001084FF46741C348001F007800EB8002C04820F82210A621001F007800EB8002BC4800EB82008172BA48001FE1
:402D0000007800EB8002B84800EB8200C6723112B548001F007800EB8002B34800EB82000173B148001F007800EB8002AE4800EB820044732112AC48001F007800EB8002A7
:402D4000A94800EB82008173A748001F007800EB8002A54800EB8200C5732912A248001F007800EB8002A04800EB82000174FF219D48001F007800EB80029B4800EB820030
:402D8000417408219848001F007800EB8002964800EB820001819448001F0078401C32280ADB9148001F00E00DE0407858B100208D49091F087006E08B48001F0078401CAE
:402DC0008949091F08704046BDE8F08130B502460020854B1B1F1B785B1C834C241F6478A3427DD0804B1B1F5B7831337E4C241F2478A34274D001204FF467447A4B1B1F28
:402E00001B7803EB8305784B23F82540A7241B1F1B7803EB8305744B03EB85039C72724B1B1F1B7803EB83056F4B03EB8503DA7214126D4B1B1F1B7803EB83056A4B03EBB5
:402E400085031C73684B1B1F1B7803EB8304664B03EB84035973FF24634B1B1F1B7803EB8305614B03EB85039C735F4B1B1F1B7803EB83055C4B03EB8503DC735A4B1B1FD7
:402E80001B7803EB8305584B03EB85031C74564B1B1F1B7803EB8305534B03EB85035C740824514B1B1F1B7803EB83054E4B03EB85031C814C4B1B1F1B785B1C322B08DBC6
:402EC000494B1B1F5B781BB10023474C241F237006E0454B1B1F1B785B1C434C241F237030BD30B5024600203F4B1B1F1B785B1C3D4C241F6478A34278D03B4B1B1F5B784A
:402F00003133394C241F2478A34278D001204FF46744354B1B1F1B7803EB8305324B23F82540A8241B1F1B7803EB83052E4B03EB85039C722C4B1B1F1B7803EB83052A4B92
:402F400003EB8503DA721412274B1B1F1B7803EB8305254B03EB85031C73FF24224B1B1F1B7803EB8305204B03EB85035C731E4B1B1F1B7803EB83051B4B03EB8503997328
:402F80000C0A194B1B1F1B7803EB8305164B03EB8503DC730C0C144B1B1F1B7803EB8305114B03EB85031C740C0E0F4B1B1F1B7803EB83050C4B03EB85035C7408240A4B3D
:402FC0001B1F1B7803EB8305074B03EB85031C81054B1B1F1B785B1C322B0BDB024B1B1F5B781BB1002302E05C3E001007E0FE4C237004E0FC4B1B785B1CFB4C237030BDBD
:403000002DE9F04706460C4615461F46DDF820804FF00009F4480078401CF349497888427DD0F14840783130EF49097888427CD041462046FDF76BFC044641462846FDF768
:4030400066FC05464FF001094FF46741E648007800EB8002E448001D20F82210A921001F007800EB8002E048001D00EB82008172DD48007800EB8002DB48001D00EB82009F
:40308000C6723112D848007800EB8002D648001D00EB82000173D448007800EB8002D248001D00EB820044732112CF48007800EB8002CD48001D00EB82008173CA480078CC
:4030C00000EB8002C848001D00EB8200C5732912C548007800EB8002C348001D00EB82000174C148007800EB8001BF48001D00EB810047740821BC48007800EB8002BA480E
:40310000001D00EB82000181B7480078401C322806DBB548407810B10020B349087004E0B1480078401CB04908704846BDE8F087F0B50446059D0020AB4E3678761CAA4FBC
:403140007F78BE4277D0A84E76783136A64F3F78BE4270D001204FF46747A34E367806EB860CA14E361D26F82C70AA27361F367806EB860C9C4E361D06EB8C06B7729A4E82
:40318000367806EB860C984E361D06EB8C06F4722712954E367806EB860C934E361D06EB8C063773904E367806EB86078E4E361D06EB870671738C4E367806EB86078A4E95
:4031C000361D06EB8706B273874E367806EB8607854E361D06EB8706F373834E367806EB8607814E361D06EB87063574FF277E4E367806EB860C7C4E361D06EB8C067774DA
:403200000827794E367806EB860C774E361D06EB8C063781744E3678761C322E06DB724E767816B10026704F3E7004E06E4E3678761C6D4F3E70F0BDF0B5044600206A4D0C
:403240002D786D1C684E7678B54278D0664D6D783135654E3678B54271D001204FF46746614D2D7805EB85075F4D2D1D25F82760AB262D1F2D7805EB85075B4D2D1D05EB0C
:403280008705AE72584D2D7805EB8507564D2D1D05EB8705EC722612534D2D7805EB8507514D2D1D05EB87052E734F4D2D7805EB85064D4D2D1D05EB860569734A4D2D78A4
:4032C00005EB8506484D2D1D05EB8605AA73464D2D7805EB8507444D2D1D05EB8705EB731E12414D2D7805EB85073F4D2D1D05EB87052E74FF263C4D2D7805EB85073A4D4A
:403300002D1D05EB87056E740826374D2D7805EB8507354D2D1D05EB87052E81324D2D786D1C322D06DB304D6D7815B100252E4E357004E02C4D2D786D1C2B4E3570F0BD6A
:40334000F0B504460020284D2D786D1C264E7678B5427BD0244D6D783135234E3678B54274D001204FF467461F4D2D7805EB85071D4D2D1D25F82760AC262D1F2D7805EB38
:403380008507194D2D1D05EB8705AE72164D2D7805EB8507144D2D1D05EB8705EC722612114D2D7805EB85070F4D2D1D05EB87052E730D4D2D7805EB85060B4D2D1D05EBA6
:4033C00086056973084D2D7805EB8506064D2D1D05EB8605AA73044D2D7805EB8507024D2D1D05EB870501E0583E0010EB731E12FE4D2D7805EB8507FC4D2D1D05EB8705A5
:403400002E74FF26F94D2D7805EB8507F74D2D1D05EB87056E740826F44D2D7805EB8507F24D2D1D05EB87052E81F04D2D786D1C322D06DBED4D6D7815B10025EB4E35709B
:4034400004E0EA4D2D786D1CE84E3570F0BD70B504460025E5480078401CE449497888427DD0E24840783130E0490978884276D001254FF46741DD48007800EB8002DB48A6
:40348000001D20F82210AD21001F007800EB8002D648001D00EB8200817276F13BFCC1B2D248007800EB8002D048001D00EB8200C17276F12FFC0112CC48007800EB8002B5
:4034C000CA48001D00EB82000173C848007800EB8002C648001D00EB820044732112C348007800EB8002C148001D00EB82008173FF21BE48007800EB8002BC48001D00EBB7
:403500008200C173B948007800EB8002B748001D00EB82000174B548007800EB8002B348001D00EB820041740821B048007800EB8002AE48001D00EB82000181AB48007862
:40354000401C322806DBA948407810B10020A749087004E0A5480078401CA4490870284670BD70B503460020A04C2478641C9F4D6D78AC4278D09D4C647831349B4D2D78C9
:40358000AC4271D001204FF46745984C247804EB8406964C241D24F82650AE25241F247804EB8406914C241D04EB8604A5728F4C247804EB84058D4C241D04EB8504E3726F
:4035C0008A4C247804EB8406884C241D04EB860421730D12854C247804EB8406834C241D04EB86046573814C247804EB84067F4C241D04EB8604A27315127C4C247804EB62
:4036000084067A4C241D04EB8604E573FF25774C247804EB8406754C241D04EB86042574724C247804EB8406704C241D04EB8604657408256D4C247804EB84066B4C241D03
:4036400004EB86042581694C2478641C322C06DB664C647814B10024644D2C7004E0634C2478641C614D2C7070BD70B5034600205E4C2478641C5D4D6D78AC4279D05B4C70
:4036800064783134594D2D78AC4272D001204FF46745564C247804EB8406544C241D24F82650AF25241F247804EB84064F4C241D04EB8604A5724D4C247804EB84064B4C37
:4036C000241D04EB8604E3721D12484C247804EB8406464C241D04EB86042573434C247804EB8405414C241D04EB850461733F4C247804EB84063D4C241D04EB8604A2734A
:40370000150A3A4C247804EB8406384C241D04EB8604E573150C354C247804EB8406334C241D04EB86042574150E304C247804EB84062E4C241D04EB8604657408252B4C4B
:40374000247804EB8406294C241D04EB86042581264C2478641C322C06DB244C647814B10024224D2C7004E0204C2478641C1F4D2C7070BD73B52DED020B02460B4669461A
:4037800000201A4C2478641C184D6D78AC427ED0164C64783134154D2D78AC4277D001204FF46745114C247804EB84060F4C241D24F82650AF25241F247804EB84060B4CCF
:4037C000241D04EB8604A572084C247804EB8406064C241D04EB8604E2721512034C247804EB8406014C241D02E00000583E001004EB86042573FE4C247804EB8405FC4CD7
:40380000241D04EB850463730D78F94C247804EB8406F74C241D04EB8604A5734D78F44C247804EB8406F24C241D04EB8604E5738D78EF4C247804EB8406ED4C241D04EBDD
:4038400086042574CD78EA4C247804EB8406E84C241D04EB860465740825E54C247804EB8406E34C241D04EB86042581E04C2478641C322C06DBDE4C647814B10024DC4D2D
:403880002C7004E0DA4C2478641CD94D2C7004B070BD30B502460020D54B1B785B1CD44C6478A34277D0D24B5B783133D04C2478A34270D001204FF46744CD4B1B7803EB2B
:4038C0008305CB4B1B1D23F82540B0241B1F1B7803EB8305C64B1B1D03EB85039C72C44B1B7803EB8305C24B1B1D03EB8503DA721412BF4B1B7803EB8305BD4B1B1D03EB08
:4039000085031C73BA4B1B7803EB8304B84B1B1D03EB84035973FF24B54B1B7803EB8305B34B1B1D03EB85039C73B14B1B7803EB8305AF4B1B1D03EB8503DC73AC4B1B787A
:4039400003EB8305AA4B1B1D03EB85031C74A84B1B7803EB8305A64B1B1D03EB85035C740824A34B1B7803EB8305A14B1B1D03EB85031C819E4B1B785B1C322B06DB9C4BC1
:403980005B7813B100239A4C237004E0984B1B785B1C974C237030BD70B503460020944C2478641C924D6D78AC4278D0904C647831348F4D2D78AC4271D001204FF467453F
:4039C0008B4C247804EB8406894C241D24F82650B125241F247804EB8406854C241D04EB8604A572824C247804EB8406804C241D04EB8604E3721D127D4C247804EB840698
:403A00007B4C241D04EB86042573794C247804EB8405774C241D04EB85046173744C247804EB8406724C241D04EB8604A27315126F4C247804EB84066D4C241D04EB860478
:403A4000E573FF256A4C247804EB8406684C241D04EB86042574664C247804EB8406644C241D04EB860465740825614C247804EB84065F4C241D04EB860425815C4C2478B0
:403A8000641C322C06DB5A4C647814B10024584D2C7004E0564C2478641C554D2C7070BD002053490978491C514A5278914276D04F49497831314E4A127891426FD001205E
:403AC0004FF467424A49097801EB81034849091D21F82320B222091F097801EB81034449091D01EB83018A72FF224149097801EB81033F49091D01EB8301CA723C4909783B
:403B000001EB81033A49091D01EB83010A733849097801EB81033649091D01EB83014A733349097801EB81033149091D01EB83018A732F49097801EB81032D49091D01EBD0
:403B40008301CA732A49097801EB81032849091D01EB83010A742649097801EB81032449091D01EB83014A7408222149097801EB81031F49091D01EB83010A811C49097886
:403B8000491C322906DB1A49497811B10021184A117004E016490978491C154A117070472DE9F04106460C461546002710480078401C0F49497888427ED00D484078313088
:403BC0000B4909788842F7D001274FF467410848007800EB80020648001D20F82210B321001F007800EB80020148001D02E00000583E001000EB82008172FE48007800EB93
:403C00008002FC48001D00EB8200C6723112F948007800EB8002F748001D00EB82000173F448007800EB8002F248001D00EB820044732112EF48007800EB8002ED48001D19
:403C400000EB82008173FF21EA48007800EB8002E848001D00EB8200C173E648007800EB8002E448001D00EB82000174E148007800EB8002DF48001D00EB82004174DD48E7
:403C8000007800EB8002DB48001D00EB82008174601D81B2D748007800EB8002D548001D00EB82000181D348007800EB8001D148001D00EB810000E043E00089082809DA60
:403CC0000821CC48007800EB8002CA48001D00EB82000181042C15DDC648007800EB8001C448001D00EB81002968C0F80F10281DC049097801EB8102BE49091D01EB820199
:403D000048600DE0BB49097801EB8102B949091D01EB820101F10F002246294680F14DFDB4480078401C322806DBB248407840B10020B049087004E0AE480078401CAD49ED
:403D400008703846BDE8F081AB4890F8EB007047A94981F8EB007047A748B0F8B4007047302802DAA44981F88E00704700B50021A14880F8251080F826100020FFF7F0FF0D
:403D8000FF209D4981F8BD0000BD014600209A4AB2F8B6200A4002B101207047002318461946954A92F8C320042A06DA924A92F8C330283202EB031203CA7047012907D1F6
:403DC0008D4AB2F8B62002438B4BA3F8B62006E0894AB2F8B6208243874BA3F8B62070472DE9FC4185480568284680F11EFA0446804840787F49097888427CD07D484078BE
:403E000000EB80017B48001D30F82100B0F5674F71D1794890F8BD00FF2808D07649D1F8940040F2DC5117F0F6FB0028E5D000267048407800EB80016E48001D00EB8100BA
:403E400000896E49096888420BD96C48008881B26848407800EB80026648001D00EB820001816448407800EB80016248001D00EB81000089092827DD5E48407800EB80015A
:403E80005C48001D00EB810050F80A1F216041686160007A20725748407800EB80035548001D00EB83000089A0F109025148407800EB80034F48001D00EB8300416804F1DC
:403EC000090080F17AFC15E04A48407800EB80034848001D00EB830002894648407800EB80034448001D00EB830000F10A01204680F163FC00E033E0FFF750FFCDE9000193
:403F00003C48407800EB80013A48001D00EB810002894FF46741204675F18CFD0646F6B13448407800EB80023248001D00EB8200018920466AF138FC20782F4981F8BD00A6
:403F400033F194FA2C49C1F894002A484078401CC0B228494870322801DB0020487000BF204634F0C6F9BDE8FC8170B500260025002426E0FFF712FF1F4A283202EB04130C
:403F80000CCB801A99411AD2012D0ED11A48283000EB0410D0E900301749283101EB0611D1E900219A1A884100D345B91248283000EB0410407B012801D126460125601CC1
:403FC000C4B2042CD6DB35BB002422E00A48283000EB0410D0E900300749283101EB0611D1E900219A1A884100D385B90248283006E00000583E0010683D0010C8BE190823
:4040000000EB0410407B012801D126460125601CC4B2042CDADB012D07D1EF4800EB0610D0E900211046F5F7C8FD284670BD70B50024002575F1B7FE06463146002075F1D6
:404040001CFE18B175F1AFFE044609E046F26E51002075F112FE10B146F26E5400E00024DD482838B0F8B400A04204D0DA482838A0F8B4400125284670BDD749283981F86B
:40408000C1007047D448283890F8C10070477CB502260024D048283890F8C45075F131FE0168009140680190CB482838B0F8B40060B1C9482838B0F8B40000128DF805006A
:4040C000C548283890F8B4008DF80600052D00DD0525002D1ADD002415E0C4EBC402BE489D3011180722684680F103FB28B1BA48283880F8BE40012607E0601CA84200D169
:404100000026601CC4B2AC42E7DB00BF30467CBD2DE9FF4104460025FF22082102A880F191FBFF208DF80800012C03D101208DF8090002E000208DF8090003208DF80A00F5
:40414000FFF72CFE0822CDE900014FF4674102A875F170FC30B133F189F99F492839C1F898000125284604B0BDE8F08110B50446042C0BDC9848283890F8C200A04205D0F1
:404180009548283880F8C24028F0EEFD10BD10B500240020FFF7E4FD00218F48283880F8251080F8261000208B492839A1F8B600FF2081F8C300084690F88B1080F88C1061
:4041C00000BF13E00021844800EB04104173824800EB04108160804A02EB0412116051607D4800EB04100173601CC4B2042CE9DB0020FFF7BBFF0020FDF752FF33F136F92E
:4042000075492839C1F89C000020A1F8B400012081F88D000020C1F8940081F8C00028F07DFD6E4800786D49487010BD2DE9FF5F00BF0024A146FF22082102A880F102FB35
:4042400000BF1FE0644800EB0410407B01280DD1614901EB0411886840F61C4117F0DBF920B100215C4800EB041041735A4800EB0410407B012803D109F1010000F0FF0975
:40428000601CC4B2042CDDDB4846FFF76FFF5248283890F8250068BBFDF7F2FE002829DD4D48283890F8C300042829DBF5F780FC05460E4600241AE0474800EB0410407B78
:4042C000012812D10020014668407140084307D0414800EB041103C968407140084304D13D48283880F8C34003E0601CC4B2042CE2DB05E033F1BAF837492839C1F89C00EF
:40430000F5F76BFC074634492839D1F89C00394617F081F950B100200146F5F74EFCFFF725FDFF202C49283981F8C3002A48283890F82600012828D100212748283880F8A9
:404340002610007E00F00400042806D022482838007E00F01000102805D100201E49283981F8BF0008E01C48283890F8BF00401C1949283981F8BF00FDF79EFE022814D134
:4043800001210846FFF71AFD0FE01348283890F82500012809D110492839C86940F61C4117F039F908B1FFF7E1FCFDF785FE06280BDB09492839D1F898004FF47A7117F00F
:4043C0002AF910B10020FFF7A3FEFDF775FE312880F0C18704E00000903D0010583E0010DFE810F031003B00460057007000780088008C00AC00C400DF00F3000E01220103
:404400003D015101750189019601BC01D001EB014E025E02AF02CC02DD02F90319043E047804A704E20411054C057B05B305D8050B0634066D068D06B106FF0610071A07A4
:4044400079079507B607FDF71FFE20B9FFF79FFE0120FFF785FC00F07EBF75F18AFB30B100210120FFF7AAFC0220FFF779FCF2E70120FFF78AFC58B10121FE4880F8251056
:4044800032F1F4FFFB49C1F894000320FFF768FCE1E7002075F19EFA18B10420FFF760FC0FE0F449D1F894004FF4FA6117F0B3F838B132F1DBFFEF49C1F89400012075F1E8
:4044C00089FAC8E70120FFF723FE10B10520FFF747FCC0E7E749D1F898004FF47A7117F09AF830B10020FFF713FE10B10620FFF737FCB0E70720FFF733FCACE70020FFF790
:4045000027FC0F208DF80800FE208DF8090000208DF80A00FFF742FC0322CDE900014FF46A4102A875F186FA38B132F19FFFD149C1F894000820FFF713FC8CE7FFF704FC0C
:4045400040B1FFF774FD0020FFF702FC0920FFF707FC0AE0C749D1F894004FF4FA6117F05AF810B10720FFF7FBFB74E700210220FFF724FCC7208DF80800FFF70FFC082238
:40458000CDE900014FF4674102A875F153FA38B132F16CFFB749C1F894000A20FFF7E0FB59E70220FFF7F1FB18B10B20FFF7D8FB0AE0B049D1F8940040F2DC5117F02BF873
:4045C00010B10920FFF7CCFB45E700210420FFF7F5FBC3208DF80800FFF7E0FB0822CDE900014FF4674102A875F124FA38B132F13DFFA049C1F894000C20FFF7B1FB2AE725
:404600000420FFF7C2FB18B10D20FFF7A9FB0AE09849D1F8940040F2DC5116F0FCFF10B10B20FFF79DFB16E700210820FFF7C6FBC2208DF80800FFF7B1FB0822CDE9000122
:404640004FF4674102A875F1F5F938B132F10EFF8849C1F894000E20FFF782FBFBE60820FFF793FB18B10F20FFF77AFB0AE08149D1F8940040F2DC5116F0CDFF10B10D2059
:40468000FFF76EFBE7E600218020FFF797FBC0208DF8080000208DF80A008DF80B008DF80C008DF80D00FFF779FB0822CDE900014FF4674102A875F1BDF938B132F1D6FEDA
:4046C0006C49C1F894001020FFF74AFBC3E68020FFF75BFB18B11120FFF742FB0AE06549D1F894004FF4FA6116F095FF10B10F20FFF736FBAFE65F4890F88D00022803D1F8
:404700001A20FFF72DFB02E01220FFF729FBA2E600211020FFF752FB0020564981F8BE0081F8C40023215348C53033F02FFFDF208DF80800FFF732FB0822CDE900014FF4AC
:40474000674102A875F176F938B132F18FFE4949C1F894001320FFF703FB7CE61020FFF714FB18B11420FFF7FBFA0AE04149D1F8940040F2DC5116F04EFF10B11220FFF788
:40478000EFFA68E6FFF783FC10B101280FD10AE0FDF78AFC18B11520FFF7E2FA02E01720FFF7DEFA07E01520FFF7DAFA03E01A20FFF7D6FA00BF00BF4DE60020FFF75DFC7F
:4047C00000212020FFF7FAFAD2208DF80800294890F8BE00C0EBC0012648C530405C8DF80900244890F8BE00C0EBC000401C2149C531085C8DF80A001E4890F8BE00C0EB1C
:40480000C000801C085C8DF80B001A4890F8BE00C0EBC000C01C085C8DF80C00154890F8BE00C0EBC000001D085C8DF80D00114890F8BE00C0EBC000401D085C8DF80E00C5
:404840000C4890F8BE00C0EBC000801D085C8DF80F00FFF7A3FA0822CDE900014FF4674102A875F1E7F850B132F100FE0149C1F8940001E0683D00101620FFF771FAEAE59B
:404880002020FFF782FA38B9FE49D1F8940040F2DC5116F0C0FE10B11220FFF761FADAE575F12FFA82460020FFF7E7FB00214020FFF784FAD1208DF808009AF800008DF8B2
:4048C00009009AF801008DF80A009AF802008DF80B009AF803008DF80C009AF804008DF80D00E848B0F8B40058B1E648B0F8B40000128DF80E00E34890F8B4008DF80F005C
:4049000007E09AF805008DF80E009AF806008DF80F00FFF743FA0822CDE900014FF4674102A875F187F858B10020D64981F8BF0032F19CFDD349C1F894001820FFF710FACF
:4049400089E54020FFF721FA78B1FFF79BFB18B92C20FFF705FA10E0FFF794FB00F0040058B91A20FFF7FCF907E0C64890F8BF00032802DB1720FFF7F3F96CE5C14890F8B3
:40498000C00004280ADABF49D1F8940042F2107116F041FE10B11A20FFF7E2F95BE50020B849087500218020FFF708FA0020B54981F8B800C1F8A40000240BE0204675F1DE
:4049C00046F9B049D1F8A4100844AE49C1F8A400601CC4B2204675F13AF908B1FF2CEDDB0020A84981F8B900C1F8A80000240EE0A448B0F8B410204675F13FF9A149D1F800
:404A0000A81008449F49C1F8A800601CC4B29D48B0F8B410204675F130F908B1FF2CE7DB0020984981F8BA00C1F8AC0000240BE0204675F15AF99349D1F8AC1008449149FD
:404A4000C1F8AC00601CC4B2204675F14EF908B1FF2CEDDB00208B4981F8BB00C1F8B000002410E00420FDF73EFB07463946204675F13EF98349D1F8B01008448149C1F837
:404A8000B000601CC4B20420FDF72DFB07463946204675F12DF908B1FF2CE3DB002410E00520FDF720FB07463946204675F123F97449D1F8B01008447249C1F8B000601C86
:404AC000C4B20520FDF70FFB07463946204675F112F908B1FF2CE3DB002410E00620FDF702FB07463946204675F108F96549D1F8B01008446349C1F8B000601CC4B2062064
:404B0000FDF7F1FA07463946204675F1F7F808B1FF2CE3DB5B48D0F8A8005A49C1F8A000084690F88D00012827D10846D0F8A000D1F8A41008445349C1F8A0000846D0F850
:404B4000A000D1F8B01008444E49C1F8A000FFF725F94FF478420020114080EA000280EA01031A4309D14748D0F8A0004549D1F8AC1008444349C1F8A000C0208DF8080095
:404B8000404890F8A0008DF80A003E48B0F8A000000A8DF80B003B48D0F8A000000C8DF80C003848D0F8A000000E8DF80D00FFF7F5F80822CDE900014FF4674102A874F180
:404BC00039FF38B132F152FC2E49C1F894001B20FFF7C6F8BFE38020FFF7D7F878B12948007DB8B9274890F88D00022803D12620FFF7B6F80EE01C20FFF7B2F80AE0214957
:404C0000D1F894004FF4FA6116F005FD10B11A20FFF7A6F89FE31B4991F8B80075F117F8B0B10020174981F88F00FFF7B7F807468846144991F8B80075F109F800F1010A9C
:404C40003A46434651464FF4674074F161FF03E002200C4981F88F001D20FFF781F87AE3084890F88F0002281FD1064991F8B80074F1EDFF70B1034890F8B800401C0149C6
:404C800002E00000683D001081F8B8001C20FFF767F81EE00020F94981F8BB00042081F88D001E20FFF75CF813E0F44890F88F0003280ED1F14890F8C000401CEF4981F877
:404CC000C00032F1D3FBED49C1F894001920FFF747F840E30420FDF706FA0746E74991F8BB00394675F104F8D8B10020E34981F88F00FFF753F8074688460420FDF7F3F9F8
:404D00008346DE4991F8BB00594674F1F1FF00F1010A3A46434651464FF4674074F1F8FE03E00220D54981F88F001F20FFF718F811E3D24890F88F00022820D10420FDF7A2
:404D4000D2F90746CD4991F8BB00394674F1D0FF50B1CA4890F8BB00401CC84981F8BB001E20FEF7FDFF1EE00020C44981F8BB00052081F88D002020FEF7F2FF13E0BF483E
:404D800090F88F0003280ED1BC4890F8C000401CBA4981F8C00032F169FBB849C1F894001920FEF7DDFFD6E20520FDF79CF90746B24991F8BB00394674F19DFFD8B10020F4
:404DC000AE4981F88F00FEF7E9FF074688460520FDF789F98346A94991F8BB00594674F18AFF00F1010A3A46434651464FF4674074F18EFE03E00220A04981F88F002120E7
:404E0000FEF7AEFFA7E29D4890F88F00022820D10520FDF768F90746984991F8BB00394674F169FF50B1954890F8BB00401C934981F8BB002020FEF793FF1EE000208F49AE
:404E400081F8BB00062081F88D002220FEF788FF13E08A4890F88F0003280ED1874890F8C000401C854981F8C00032F1FFFA8349C1F894001920FEF773FF6CE20620FDF777
:404E800032F907467D4991F8BB00394674F136FFD8B10020794981F88F00FEF77FFF074688460620FDF71FF98346744991F8BB00594674F123FF00F1010A3A464346514698
:404EC0004FF4674074F124FE03E002206B4981F88F002320FEF744FF3DE2684890F88F0002281DD10620FDF7FEF80746634991F8BB00394674F102FF50B1604890F8BB00E9
:404F0000401C5E4981F8BB002220FEF729FF1BE003205A4981F88D002420FEF721FF13E0564890F88F0003280ED1544890F8C000401C524981F8C00032F198FA4F49C1F8EF
:404F400094001920FEF70CFF05E24C4991F8BA0074F1CBFEB0B10020484981F88F00FEF71DFF07468846454991F8BA0074F1BDFE00F1010A3A46434651464FF4674074F155
:404F8000C7FD03E002203D4981F88F002520FEF7E7FEE0E1394890F88F00022818D1374991F8BA0074F1A1FE50B1344890F8BA00401C324981F8BA002420FEF7D1FE1BE07C
:404FC00002202E4981F88D002620FEF7C9FE13E02A4890F88F0003280ED1284890F8C000401C264981F8C00032F140FA2349C1F894001920FEF7B4FEADE1204AB2F8B41072
:4050000092F8B90074F139FEC0B100201B4981F88F00FEF7C3FE07468846184AB2F8B41092F8B90074F129FE00F1010A3A46434651464FF4674074F16BFD03E002200F4974
:4050400081F88F002720FEF78BFE84E10B4890F88F0002281ED1094AB2F8B41092F8B90074F10BFE60B1054890F8B900401C034981F8B9002620FEF773FE1FE0683D001030
:405080000020F94981F8BC002820FEF769FE27F070FE13E0F44890F88F0003280ED1F24890F8C000401CF04981F8C00032F1DEF9ED49C1F894001920FEF752FE4BE1002148
:4050C0004FF48070FEF77AFE12208DF80800FEF765FE0822CDE900014FF4674102A874F1A9FC58B10020E04981F8BF0032F1BEF9DD49C1F894002920FEF732FE2BE14FF4E5
:405100008070FEF742FE30B1FEF7BCFFD0B92A20FEF726FE16E0D44890F8BF00032811DBD14890F8BC0003280ADACF4890F8BC00401CCD4981F8BC002820FEF711FE01E0C2
:40514000FEF714FE07E174F1DCFD82460020FEF794FF00214FF40070FEF730FED0208DF808009AF800008DF809009AF801008DF80A009AF802008DF80B009AF803008DF89E
:405180000C009AF804008DF80D00B748B0F8B40058B1B548B0F8B40000128DF80E00B24890F8B4008DF80F0007E09AF805008DF80E009AF806008DF80F00FEF7EFFD082247
:4051C000CDE900014FF4674102A874F133FC38B132F14CF9A449C1F894002B20FEF7C0FDB9E04FF40070FEF7D0FD38B99E49D1F8940047F2305116F00EFA10B12C20FEF73A
:40520000AFFDA8E00020984981F8C00081F88D002D20FEF7A5FD9EE0FEF796FD68B10020FEF796FDFEF703FFF0B302208E4981F88D001120FEF794FD4CE0FCF72DFF50B1B3
:40524000FEF793FE18B12E20FEF78AFD42E00020FCF726FF3EE0FCF717FF18B12E20FEF77FFD37E0804890F88C1090F88B0081422ED07D4890F88C00C0EBC0017A48683096
:405280000844016802918188ADF80C1080798DF80E00FEF783FD0822CDE900014FF4674102A874F1C7FB00E014E098B1072102A869F17AFA6C4890F88C00401CC1B26A4838
:4052C00080F88C10052905DB002180F88C1001E0FEF786FD3FE000214FF48060FEF76EFDB2208DF80800FEF759FD0822CDE900014FF4674102A874F19DFB38B132F1B6F864
:405300005949C1F894002F20FEF72AFD23E04FF48060FEF73AFDD0B1FEF728FDFCF7BCFEA8B1002410E0F4F743FC4F4A283202EB04130CCB50405940084303D14A4880F8C2
:40534000C34003E0601CC4B2042CECDB00BF02E0FEF70CFD00BF00BFBDE8FF9F2DE9F04F044689469246DDE909676079A17940EA0120E17940EA014594F8008094F801B031
:40538000FCF75DFE98420CD1B8F1010F08D1B5F5674F04D1BBF1FF0F01D1FEF7E7FC00BF00BFBDE8F08F70B504460D462E4880F8C440052C00DD0524C4EBC40229462A48DA
:4053C000C5307FF1FAF970BD70B504460D46164625488472C572068174F195FC00EE100AF8EE400A2048008900EE100AB8EE400A80EE201A1C4880ED001A70BD1A4B187322
:4054000059739A7370472DE9F0412DED028B06460F4614461D4674F179FC00EE100AF8EE400A00EE104AB8EE400A80EE201AB0EE418A74F16DFC00EE100AF8EE400A00EE41
:40544000105AB8EE400A80EE201AF0EE418A064886744774C4730574B4EEE88AF1EE10FA04D280ED018A04E0683D0010FE48C0ED018ABDEC028BBDE8F0812DE9F05F0446F1
:405480008A4693469846DDE90A6794F800900025B9F1FE0F33D100BF2EE0F348283000EB051103C97040794008430AD0EE48283000EB0510D0E90010002359405840014388
:4054C00018D131F1D3FFE849283101EB051188600121E548283000EB05104173E248283000EB051080F80C80DF48283000EB0510C0C003E0681CC5B2042DCEDB00BFFCF711
:405500009EFD40457DD1B9F1AD0F7BD054DCB9F1250F78D027DCB9F1080F75D008DCB9F1080F72D2DFE809F0A6A7A8A9AAABACADB9F1200F6AD00CDCB9F1090F67D0B9F15A
:405540000A0F65D0B9F1120F71D0B9F1130F5CD1E9E0B9F1210F6BD0B9F1220F69D0B9F1240FF4D1E3E0B9F1A40F74D01ADCB9F1A00F71D00CDCB9F1260F6ED0B9F1270F6B
:405580006CD0B9F1900F6AD0B9F1920FDFD1D3E0B9F1A10F77D0B9F1A20F75D0B9F1A30FD5D1CDE0A9F1A5000828BAD2DFE800F0CACBCCCDCECFD0D1B9F1C00F7ED00EDCBF
:4055C000A9F1AE001128ACD2DFE800F0C5C6C7C8CBD0D1D2D3D4D5D6D7D8D9DADB00B9F1D10F6CD026DCB9F1C50F69D015DCB9F1C10F66D0B9F1C20F7BD0B9F1C30F79D063
:4056000007E041E1A6E093E03CE032E18CE03CE07CE0B9F1C40F9AD1D4E0B9F1C60F6AD0B9F1C70F68D0B9F1D00F90D1DDE06EE07BE07BE0B9F1D60F71D011DCB9F1D20F55
:405640006ED0B9F1D30F6CD0B9F1D40F6AD0B9F1D50F86D1E3E074E06FE06AE06AE06AE0B9F1E00F7BD0B9F1FD0F79D0B9F1FE0F8CD1E0E000BF00BF00BF00BF00BF00BF03
:4056800000BF00BFF5E059E059E0774890F88B00401C754991F88C10884236D0724890F88C00001D704991F88B1088422DD06E4890F88B00C0EBC0016B4803E062E09CE02C
:4056C00081E069E06830084421680160A1888180A1798171644890F88B00401C05280CDB614890F88C0080B100215F4880F88B100BE052E05CE067E067E05B4890F88B0067
:40570000401CC1B2584880F88B10B2E0B1E06078FEF7B3FC01210802FEF750FBA9E07FE073E07AE07AE000BF00BF00BF00BF00BF00BF00BF00BF00BF00BF00BF00BF00BF3A
:4057400000BF00BF00BF00BF00BF00BF00BF00BF00BF00BF00BF00BF00BF00BF89E060E068E001218802FEF729FB82E000BF00BF00BF00BF00BF00BF00BF00BF00BF00BF29
:4057800000BF76E060783849C874A078087501218020FEF713FB6CE06BE063792279A179E079FFF730FE01210820FEF707FB60E0E279A1796079FFF721FE01210420FEF721
:4057C000FDFA56E000BF00BF53E0237994F805C043EA0C22E378C3F34001A078FFF7F4FD01210220FEF7EAFA43E06079FEF745FC01214802FEF7E2FA3BE06079FEF73DFC84
:4058000001214020FEF7DAFA33E06079FEF735FC01212020FEF7D2FA2BE000BF00BF00BF27E06078A11CFFF7BEFD01211020FEF7C5FA1EE01DE031F119FE0B49C86101217A
:40584000094880F82610617880F82410A078E17840EA0121044801842079617940EA012101484184A07901E0683D00101E49087600BF00BF1C4890F8BD002178884203D157
:40588000FF20194981F8BD00BDE8F09F2DE9FC4781460E4617469846DDE90A45B6F5664F14D174F16BF9FE2807DAFCF7C8FB404503D13946484669F1ADFC43463A46314685
:4058C0004846CDE90045FFF7D8FD0AE0B6F5684F07D143463A4631464846CDE90045FFF73DFDBDE8FC870000683D00100246104649B108B9084606E000E000680368002BAF
:40590000FBD10160104670472DE9F04706460C4617469846DDF82090B24600250DE024B139465046A047012803D1A84500D107E06D1C504680F1AAF88246BAF1000FEED192
:4059400000BFB9F1000F01D0C9F800505046BDE8F0872DE9F8430446884615461E460027B8F1000F14D09DB1002000900023324641462068FFF7C8FF074647B93046A84719
:40598000074639462068FFF7B1FF206000E000273846BDE8F8832DE9F04706460C4617464FF0FF39B04600250EE024B139464046A047012800D16D1C404680F167F88046A0
:4059C000B5F1FF3F00D102E0B8F1000FEDD100BF2846BDE8F087014621B10868884201D1012070470020FCE700B5024612B1106800B912601046FFF7EEFF00BD10B50346EA
:405A0000184600241470C0B1B9B1884204D100680C600124147010E00AE004688C4206D10C68046000240C600124147003E000680468002CF1D100BF184610BD38B50446A7
:405A40000D46002000906A4629462046FFF7D6FF38BD002101607047002101607047000070B504460025022614B9DF4D00BF00BF00BF25B132462946DC4840F17AF870BDC9
:405A8000DB480068401CDA49086008460068704770B504460D461646D648206000206060A060314604F10C00F6F7D0F8A0F10C04FFF7E6FF20612575207D022802DB0020E3
:405AC000FFF7CEFF204670BD70B504460D46C948206068686060A868A06005F10C0104F10C00F6F7E2F8A0F10C0428692061287D2075204670BD10B50446BE48206004F188
:405B00000C00F6F7D5F8A0F10C04204610BD70B504462046FFF7EFFF054633F003FB70BD2DE9FC4106460C4615461F46DDF82080FF203870002D1EDD082D1CDC681E04F0BD
:405B400007010844012101EBD003E208306801A9D0F814C03046E04701280CD104F007013B462A4601A8CDF8008007F067FB10B10120BDE8FC810020FBE72DE9FC410646AC
:405B80000C4615461F46DDF820804FF6FF703880002D1EDD102D1CDC681E04F007010844012101EBD003E208306801A9D0F814C03046E04701280CD104F007013B462A468E
:405BC00001A8CDF8008007F0A9FB10B10120BDE8FC810020FBE72DE9FE4306460C4615461F46DDF828804FF0FF303860002D1EDD202D1CDC681E04F007010844012101EB95
:405C0000D003E208306801A9D0F814C03046E04701280CD104F007013B462A4601A8CDF8008007F0EDFB10B10120BDE8FE830020FBE72DE9FF4106460C4615461F46DDF8D9
:405C400028804FF0FF3139607960002D1FDD402D1DDC681E04F007010844012101EBD003E208306801A9D0F814C03046E04701280DD104F007013B462A4601A8CDF8008016
:405C800007F02FFC18B1012004B0BDE8F0810020FAE770B50446FF2520467FF1D6FF012812D120467FF1CBFF00F47000B0F5700F0AD2606828B920467FF1C1FFC0F30725A1
:405CC00002E06068417B0D46284670BD70B50446FF2520467FF1B9FF012809D1A06820B920467FF1ACFFC5B202E0A068417B0D46284670BD2DE9F843054600272868C16942
:405D00002846884701285ED128467FF19EFF002856D0012856D12846FFF7D8FF04462846FFF7B7FF0646FE2C24DB48D128467FF186FF31490840B0F56E0F1BD028467FF178
:405D40007EFF2D490840B0F56A0F38D12868032300226946D0F814C02846E04701282ED19DF8000058BB9DF80100EE2827D19DF8020020BBFE2E22D028467FF160FF00F4D4
:405D80007000B0F5700F0ED228467FF158FF6FF30F0040EA062040EA04084146284633F00CF801270BE028467FF149FF20F0FF0040EA04084146284632F0FFFF012701E08B
:405DC000012700BF00BF3846BDE8F8830246022042B100BF137B184621B100BF0B7B834200D002207047000031E4040825E404082C02002094C019080000FF0370B5044668
:405E000000250226082C1DD2DFE804F004070A0D10131619A14D012614E0A14D012611E0A04D02260EE0A04D02260BE09F4D022608E09F4D022605E09E4D022602E09E4DDC
:405E4000022600BF00BF25B1324629469B483FF190FE70BD2DE9F05F04460F4615461E46DDE90A893A4649462046FFF711FE04469348206084F81D800020A07700BF00BFE8
:405E8000E06865F31E00E06000BF00BF0020C4F81500C4F81900002E71D0607F08286FDC607F00286CD0627F314604F115007EF184FC207D022877DA00BF00BFE06800F075
:405EC000004008B1012000E0002000BF002858D0012864D120467FF1B2FEB0F1005F4AD220467FF1ACFE00F0FF0ABAF1FE0F19DBBAF1FE0F3BD120467FF1A1FE7149084019
:405F0000B0F56A0F06D1607D20B9A07DEE2801D1E07D38B120467FF192FE6A490840B0F56E0F24D1217D04F10802504632F0CAFF20467FF184FE00F47000B0F5700F13D210
:405F400020467FF17CFEC0F3072BBBF1FE0F07D0217D221D584632F0B5FF0120A07702E00020FFF74BFF05E00120A07702E00120FFF744FF02E00220FFF740FF13E01BE011
:405F800016E020467FF15BFEB0F5006F02D20120A07702E00320FFF731FF04E004E00420FFF72CFF00BF0AE00520FFF727FF06E00620FFF723FF02E00720FFF71FFF2046D3
:405FC000BDE8F09F10B504462046FFF794FD0446204610BD70B504462046FFF7F3FF054633F0A0F870BD014601207047024602F115000860012070472DE9F04104460D4671
:4060000016460027607FB04207D835B1627F04F1150128467EF1D1FB01273846BDE8F0812DE9F04104460D4616461F464FF00008F019617F884209D845B104F115008119DC
:406040003A4628467EF1B9FB4FF001084046BDE8F0810146487F70470146887F704770B5044620467FF1EBFDC5B2217D04F10802284632F027FF20467FF1E1FD00F4700052
:40608000B0F5700F09D220467FF1D9FDC0F30725217D221D284632F015FF70BDD5E40408F1E4040808E5040829E504084AE5040862E5040876E504088AE50408C1E40408CE
:4060C000D4C40A080000FF0370B504460025022614B1012C06D102E0564D022602E0564D022600BF00BF25B13246294653483FF140FD70BD2DE9F04104460F4616461D4600
:406100004F4820603946201D3EF181FF041F257366730020A073E073022D01DBFFF7D4FF607BFF2802D10120FFF7CEFF2046BDE8F08170B5044642482060207B022807DA9B
:40614000607BFE2804DA617B207B002232F05CFE204632F065FE2546284606F0C3FB00BF201D3FF19FF8041F204670BD70B504462046FFF7DEFF054632F0D4FF70BD2DE90F
:40618000FC5F05460C4600BF281D32F078FF074688466E7B4FF00009287B217B884246D14FF00109687BFE2804DA697B287B224632F02AFE607BFE2804DA617B207B2A46AF
:4061C00032F022FE607B6873EA46211D50463EF11EFF824600BF6946281D7FF121FD834668463FF15FF866733A46434668463EF103FF83465946201D7FF112FD82466846F5
:406200003FF150F8687BFE2803DA284632F008FE02E028467FF190FC607BFE2803DA204632F0FEFD02E020467FF186FC00BF4846BDE8FC9FADE50408C1E504089CE5040819
:40624000A0C30A0870B5044600255CB1002007E0265C2C2E03D114601870012502E0401C8842F5D31DB900201060FF201870284670BD2DE9F04105460F4614461E464FF0D3
:4062800000083346224639462846FFF7DBFFD8B12068401B18D42068401BB84214D23078401C2168084420602168481B0AE0295C2A2906D12178491B411A31704FF00108FE
:4062C00002E0401CB842F2D3B8F1000F03D100202060FF2030704046BDE8F0812DE9F04105460F4614461E464FF000083346224639462846FFF7BDFFD8B12068401B18D456
:406300002068401BB84214D23078401C2168084420602168481B0AE0295C2A2906D12178491B411A31704FF0010802E0401CB842F2D3B8F1000F03D100202060FF20307093
:406340004046BDE8F0812DE9F04105460F4614461E464FF000083346224639462846FFF7BDFFD8B12068401B18D42068401BB84214D23078401C2168084420602168481BB5
:406380000AE0295C2A2906D12178491B411A31704FF0010802E0401CB842F2D3B8F1000F03D100202060FF2030704046BDE8F0812DE9F04105460F4614461E464FF0000893
:4063C0003346224639462846FFF7BDFFD8B12068401B18D42068401BB84214D23078401C2168084420602168481B0AE0295C2A2906D12178491B411A31704FF0010802E001
:40640000401CB842F2D3B8F1000F03D100202060FF2030704046BDE8F0812DE9F04105460F4614461E464FF000083346224639462846FFF7BDFF20B32068401B21D420681B
:40644000401BB8421DD23078401C2168084420602168481B0AE0295C2A2906D12178491B411A31704FF0010802E0401CB842F2D3B8F1000F05D12078401B381A30704FF00A
:406480000108B8F1000F03D100202060FF2030704046BDE8F0812DE9F04705460F46164698464FF0000900241FE029190422F8A031F0EFFFC0B9241D285D502803D1641CA0
:4064C0002819306001E028193060204609E0295C2C2905D1011B88F800104FF0010902E0401CB842F3D302E0641CBC42DDD3B9F1000F04D100203060FF2088F800004846AC
:40650000BDE8F0872DE9F04705460E46174698464FF00009002426E029190422DCA031F0B8FFF8B9241D285D502800D1641C15E0285D2C2811D1641C28193860204609E052
:40654000295C2A2905D1011B88F800104FF0010902E0401CB042F3D302E0641CB442E7D300BF02E0641CB442D6D3B9F1000F04D100203860FF2088F800004846BDE8F08721
:406580002DE9F04705460F46164698464FF0000900241FE029190422BFA031F07AFFC0B9241D285D502803D1641C2819306001E028193060204609E0295C2C2905D1011B3F
:4065C00088F800104FF0010902E0401CB842F3D302E0641CBC42DDD3B9F1000F04D100203060FF2088F800004846BDE8F0872DE9F04705460E46174698464FF0000900249A
:4066000026E029190422A4A031F043FFF8B9241D285D502800D1641C15E0285D2C2811D1641C28193860204609E0295C2A2905D1011B88F800104FF0010902E0401CB042DA
:40664000F3D302E0641CB442E7D300BF02E0641CB442D6D3B9F1000F04D100203860FF2088F800004846BDE8F08701468C4870470146886D704710B5044620463DF11EFB72
:4066800004468848206000206060A060E06020616061A061E06120626062A062E06220636063A063E06320646064A065204610BD10B5044620463DF128FB0446204610BDC5
:4066C00070B504462046FFF7F3FF054632F02AFD70BD70B5044600250226052C13D2DFE804F00306090C0F006F4D02260BE06F4D022608E06E4D022605E06E4D022602E03A
:406700006D4D022600BF00BF25B13246294664483FF12FFA70BD2DE9FC4704460F4690461D460A9E4FF00009002088F800003070002D7BD028706870172F78D2DFE807F073
:406740000C1A2836445264788694BED1E4FDFCFBFAF9F87777F7F600E06850B100200190414601A8E268904781469DF80400287000BF3CE1206950B100200190414601A852
:406780002269904781469DF80400287000BF2EE1606950B100200190414601A86269904781469DF80400287000BF20E1A06950B100200190414601A8A269904781469DF883
:4067C0000400287000BF12E1E06950B100200190414601A8E269904781469DF80400287000BF04E1206A70B100200190414601A8226A90478146BDF804002870BDF80400A2
:406800000012687000BFF2E0606A70B100200190414601A8626A90478146BDF804002870BDF804000012687000BFE0E0ECE0DDE0A06A50B100200190414601A8A26A9047DC
:4068400081469DF80400287000BFD0E0E06A50B100200190414601A8E26A904781469DF80400287000BFC2E0206B78B10020019000904246694601A8236B984781469DF86B
:40688000040028709DF80000687000BFAFE00000424C442C000000004150502C00000000E0E5040894C80A08FCE5040832E6040860E604088DE60408B2E60408606B78B1BD
:4068C0000020019000904246694601A8636B984781469DF8040028709DF80000687000BF85E0A06B78B10020019000904246694601A8A36B984781469DF8040028709DF872
:406900000000687000BF72E0E06BC0B10020019000904246694601A8E36B984781469DF8040028709DF80000687007E04EE03FE030E021E059E057E010E001E000BF56E084
:40694000206C50B100200190414601A8226C904781469DF80400287000BF48E0606C50B100200190414601A8626C904781469DF80400287000BF3AE0A06C50B10020019083
:40698000414601A8A26C904781469DF80400287000BF2CE0E06C50B100200190414601A8E26C904781469DF80400287000BF1EE0206D50B100200190414601A8226D904722
:4069C00081469DF80400287000BF10E0606D50B100200190414601A8626D904781469DF80400287000BF02E000BF00BF00BF00BF687810B10220307006E0287810B101203B
:406A0000307001E0002030704846BDE8FC87FEB50546286881682846884700285ED001285DD0022802D003285BD159E02E4630467FF12AF908BBFF208DF8040000208DF8E6
:406A40000500002411E00DF1070002AB421E21460090FE48FFF75FFE28B19DF80500401CC0B28DF80500601CC4B2162CEBDD022201A930463CF13FFE2FE0002700241DE08E
:406A80008DF804400DF10600431C421E21460090EE48FFF740FE78B130467FF1F5F8401EB84207D19DF80600C21C01A930463CF122FE05E0781CC7B2601CC4B2162CDFDDF5
:406AC00000BF96F8290038B9FF208DF80400012201A930463CF10FFE00BF02E000BF00BF00BF00BFFEBD7CB504462068816820468847002872D0012871D0022802D0032896
:406B00006ED189E02546002001902A20009028467FF1BAF80C2877D2DFE800F0061218242A363C484E5A637001A8C9490968884706469DF80420314628463CF1DCFD67E00E
:406B40000122694628463CF1D6FD61E001A8C1490968884706469DF80420314628463CF1CAFD55E00122694628463CF1C4FD4FE001A8B9490968884706469DF804203146CA
:406B800028463CF1B8FD43E00122694628463CF1B2FD3DE001A8B1490968884706469DF80420314628463CF1A6FD31E00122694628463CF1A0FD2BE001A8A949096888478B
:406BC00006469DF80420314628463CF194FD1FE00122694628463CF18EFD19E01AE01AE01BE001A89F490968884706469DF80420314628463CF17FFD0AE005E00122694609
:406C000028463CF178FD03E00020FFF762FD00BF00BF02E000BF00BF00BF00BF7CBD7CB504462068816820468847002851D0012850D0022802D003284ED14CE025460020A7
:406C400001902A20009028467FF11EF806283AD2DFE800F0030F1521273301A882490968884706469DF80420314628463CF143FD2DE00122694628463CF13DFD27E001A8B3
:406C80007A490968884706469DF80420314628463CF131FD1BE00122694628463CF12BFD15E001A872490968884706469DF80420314628463CF11FFD09E001226946284607
:406CC0003CF119FD03E00120FFF703FD00BF00BF02E000BF00BF00BF00BF7CBDFEB504462068816820468847002839D0012838D0022802D0032836D134E02546002002905E
:406D00002A20019028467EF1BFFF48B959480068804700900122694628463CF1ECFC1EE028467EF1B1FF401E00F0010090B928467EF1AAFF401EC0F3470702A938464E4A5E
:406D40001268904706469DF80820314628463CF1D2FC04E0012201A928463CF1CCFC02E000BF00BF00BF00BFFEBD10B504463D48006870B13848006858B13948006840B144
:406D80003348006828B13348006810B13348006810B90220FFF79DFC3448006828B13248006810B13248006810B90320FFF791FC3148006810B12F48006810B90420FFF701
:406DC00088FC00224FF6C551204604F01CFA00224FF68D41204604F016FA00224FF6DA61204604F010FA00224FF68E41204604F00AFA00224FF64251204604F004FA002275
:406E00004FF63251204604F0FEF910BD70B504460125A06810B1A06880470546284670BD2DE9FF4F89B00646DDF87480DDE918741A9D01200890B06D401CB0650F48386068
:406E40000020206006202870002119E03C2000208CEB040890EB040884EB040894EB040888EB040880EB04089CEB040898EB0408A0EB0408A8EB0408A4EB040830020020D3
:406E80001B9801701C9801600020C8F800004FF642520C98811A90427ED00ADCA0F57C40A0F18D00002878D0012877D0A52876D1F3E0832903D0B1F5CC7FF8D152E00020DA
:406EC000079007A8B749096888479DF81C102068084420602068401C206007A8B249096888479DF81C102068084420602068401C206007A8AD49096888479DF81C10206802
:406F0000084420602068401C206007A8A849096888479DF81C102068084420602068401C206007A8A349096888479DF81C102068084420602068401C206007A89E4909686D
:406F400088479DF81C102068084420602068401C20600020386006202870AFF27540C8F800000CE1002007902068401C20604FF0000910E007A94846904A126890479DF8FF
:406F80001C102068084420602068401C206009F1010000F0FF0903E010E0C5E08FE0EBE08748006880474845E4DC0020386006202870AFF2D720C8F80000E0E04FF6FF70BB
:406FC000079007200690032005904FF6FF700490012003904FF6FF7002907068002859D002A803A9CDE9001004AB05AA06A907A8D6F804C0E04701284CD1BDF81C00A0F5DD
:40700000FA6000F03F006F490870084600789DF8181001F0030140EA81106A4908709DF81800C0F380004870084640789DF8141001F0030140EA4100624948700846407819
:407040009DF8181001F0180108435E49487008464078BDF8101001F0070140EA411059494870BDF81000C0F3C70088700020C87008719DF80C00C007000E4871BDF8080002
:407080008871BDF80800000AC871082020600620287001E00020089071E03046FFF7B6FE48490870FF2048708870C870087148718871C87108202060062028705FE04FF00F
:4070C000000A0020079083460690814615E006A805AB07AA494600903046FFF71CFB40B10BF1010000F0FF0B9DF8180050441FFA80FA09F1010000F0FF09B9F1160FE6DDC2
:407100000AF10200032101FB0B0020602068082801D2082020600020386006202870AFF21170C8F800002AE0002007900320206007A82549096888479DF81C1020680844C6
:40714000206007A82149096888479DF81C1020680844206007A81E49096888479DF81C102068084420600020386006202870AFF25150C8F8000002E00020089000BF00BF26
:4071800008980DB0BDE8F08F70477047704710B51048FFF770FA04460F4AAFF6EB2131F045F910BD8CEB040890EB040884EB040894EB040888EB040880EB0408A4EB04088B
:4071C000A8EB04083002002098EB04089CEB0408A0EB04083C2000200080000870B5044600250226052C13D2DFE804F00306090C0F006C4D02260BE06B4D022608E06B4DDB
:40720000022605E06A4D022602E06A4D022600BF00BF25B13246294667483EF1AAFC70BD2DE9F04F89B004460F4690469946C4F800801298606027721398607284F80A9001
:407240000020E072206808B1A07A10B90020FFF7C5FF606810B90120FFF7C0FF607A10B90220FFF7BBFF207A022802DB0320FFF7B5FF524A5249204605F056FF18B9042078
:40728000FFF7ACFF63E0227AA17A206803F08AFC0790002657E0E07A617A884250DA08A80090237AA27A3046216803F0E1FB002846D04FF0000B002006900898006881681F
:4072C0000898884702280CD104A8089931F0B9FE0120069004A93B483DF16EFE08B1012000E0002082460390069810B104A83DF1D9FF00BFDA4522D04FF0000B1C2031F0B5
:4073000019FF824601A8089931F09BFE4FF0010B217A002301AA504607F0F0FD82465546BBF1000F02D001A83DF1BCFFE07A401CE072606810B128466168884700BF00E083
:4073400004E0701C86B207988642A4DB00BF204609B0BDE8F08F10B50446184A1849204606F004FB204610BD02460020086013480088824204DA1248006850F82200086034
:40738000086808B1012070470020FCE70B48008870470146087A70470146C87A70470146487A70476CA2190880A21908B1A21908E5A21908F9A2190848A219083C02002004
:4073C0003802002040A219080146FD4870470146D1F84401704770B50346002401B91AB300201FE000EB80061D1D05EB461595F89E50ADB100EB80061D1D05EB46156D680F
:407400008D420DD100EB80061D1D05EB46152D68954205D100EB80061D1D05EB461403E0451CE8B20228DDDB204670BD2DE9F84F81468A4693461F46DDE90B680A9D0020ED
:4074400000905A4651464846FFF7C5FF04464FF0FF30386028603060C8F80000A4B17834606938602068C0EBC0002860E06930602069783CC8F8000028683168884201D955
:4074800030682860012000900098BDE8F88F0146D1F84C01704700211C3040F81C1C40F8181C40F8141C40F8101C8165C165491E0166002141668166491EC166090A01677C
:4074C000002141678167C16780F8801080F8811080F882101C3800BF07E04FF0FF3300F1100242F821304A1CD1B21929F5DB704710B5044620463CF1E1FB0446B1482060AC
:407500000223A022AFF27101201D7EF10AFC041F002004F5A27420603CF166FA60600020A06020736073A4F5A274204610BD10B5044620463CF1E9FB0446204610BD70B5F0
:4075400004462046FFF7F3FF054631F0EBFD70BD70B5044600250226352C1ED2DFE804F01B1E2124272A2D303336393C3F4245484B4E5154575A5D606366696C6F727578FA
:407580007B7E8184878A8D909396999C9FA2A5A8ABAEB1B4B7008C4D02269BE08B4D022698E08B4D022695E08A4D022692E08A4D02268FE0894D02268CE0894D022689E025
:4075C000884D022686E0884D022683E0874D022680E0874D02267DE0864D02267AE0864D022677E0854D012674E0854D022671E0844D02266EE0844D02266BE0834D022651
:4076000068E0834D022665E0824D012662E0824D01265FE0814D01265CE0814D022659E0804D012656E0804D012653E07F4D022650E07F4D01264DE07E4D00264AE07E4D7D
:40764000002647E07D4D002644E07D4D002641E07C4D00263EE07C4D00263BE07B4D022638E07B4D002635E07A4D002632E07A4D00262FE0794D00262CE0794D002629E08E
:40768000784D002626E0784D002623E0774D012620E0774D01261DE0764D01261AE0764D012617E0754D022614E0754D002611E0744D00260EE0744D00260BE0734D00260F
:4076C00008E0734D022605E0724D012602E0724D002600BF00BF25B13246294638483EF148FA70BD2DE9F84304460D460126204631F0B0FC88B1002600BFE06868B12046A2
:4077000031F0A8FC0746E0688046009742466348D5E91F1305F028FB06463046BDE8F8832DE9F0438FB004460D4616464FF00008E06FB0F1FF3F40D0D4F89400B04201D24A
:40774000D4F89460771B40F2F960874200D90746D4F88400A84231D8D4E920100844A8422CD34FF000097C34D4E90101691A401A606060680090A0682A1A54F87C190023DC
:40778000464805F0BBFB20B90120FFF7E1FE4FF01108C4F88450E0E0D4F88000B8420ED2A06800287CD0012374342268216A6069CDE90203CDE9001273E0DAE0D3E0B5E0F5
:4077C00033A319085CC819084FA3190877A3190899A31908CCA3190808A4190838A4190871A41908B1A41908D5A41908F0A419080DA519082CA5190851A5190871A519083A
:4078000090A51908DFA5190819A6190860A6190870A6190890A61908ABA61908C0A61908DBA6190800A7190821A7190831A719084BA7190867A719087EA7190895A719088E
:40784000B8A71908DDA71908F5A719081BA8190835A8190854A819086DA819087EA8190899A81908ACA81908D1A81908F4A8190816A919082EA9190847A9190863A9190866
:4078800086A91908ADA91908CEA91908EEA919080AAA190816AA190844AA1908982000203EE0D4E90310743C43182246AFF2CB1104A83BF1E9FE04A8A1688847606F401CC8
:4078C000606700BF9DF8390030B100BF079848B904A831F0BFFB28B10220FFF739FE4FF0140819E004A831F0B5FB98B100BF9DF8380020B90320FFF72BFE4FF0110804A880
:4079000031F0A8FBD4F880100844C4F880004FF0000901E009F1010904A83BF1D8FE14E00420FFF715FE4FF012080EE08034D4E9001008446169803C884205D90520FFF746
:4079400007FE4FF0150800E00BE009F1010020B90620FFF7FDFD4FF01408B8F1000F3FF41BAF00BF04E00720FFF7F2FD4FF0150800BF40460FB0BDE8F0832DE9F84304461F
:407980000E46A06FC0EBC005D4F89400471B4FF00008FF220721701C7CF154FF94F89D00401C3070072F00D90727E06FB0F1FF3F3BD0D4E920100844E919884222D2A06FB3
:4079C000401CC0EBC0022046D4F88410FFF7A8FEA8B9D4E920100844E91988420FD3D4F88400A8420BD80097D4F884002B1A721CF848E16F05F048F808B1012000E000209E
:407A0000804620E0D4F88400A8420BD80097D4F884002B1A721CEF48E16F05F035F808B1012000E0002080460DE0E06840B1E06841193A46701C7CF1C0FE4FF0010802E037
:407A40000020FFF785FD4046BDE8F8833EB504460D46002C56D094F89E000A2824D2DFE800F01D1E05060708090A0B0C00BF00BF00BF00BF00BF00BF00BFA06868B185F08F
:407A800001026846D4F88810F4F754F86846A16888476846F4F753F800BF00BF00BFCD48E16F05F08CF800BF00BF00201C3444F81C0C44F8180C44F8140C44F8100CA0658A
:407AC000E065401E206600206066A066401EE066000A206700206067A067E06784F8800084F881001C3C00BF07E04FF0FF3204F1100141F82020411CC8B21928F5DB002019
:407B000084F89E003EBD70B505460026002421E004EB8401281D00EB411090F89E00B8B9AD480068804704EB8402291D01EB4211C1F89000012104EB8402281D00EB421069
:407B400080F89E1004EB8401281D00EB411603E0601CC4B2022CDBDB304670BD2DE9FE4F83460F4690461D460C9E4FF000099B48804573D840F2F96080456FD9002D6DD0E7
:407B8000002EFCD02868C16828468847012865D13068C168304688470128F8D1324629468F48FFF718FC0446002C7DD18C48FFF7AAFF0446002C78D0FDF762FFC4F8880028
:407BC0000E9818B1D4F888100E980160266065600F98A06000206067A067401EE0670020C4F88000C4F88400C4F88CB07A4800688047C4F89000C4F894804FF0FF30C4F85B
:407C00009800002084F89C0084F89D000D98012809D1E760E068002863D10820FFF798FC4FF009095DE00FB30020E06004F17C026848D4F8941005F017F848B1D4F8940076
:407C4000009000233A466348E16F05F08DF830B90920FFF77DFC4FF0110942E05AE0002080346060606944F880093AE0A06890B340F2F961D4F89400884201D98A4601E05E
:407C8000D4F894A004F17C025146524804F0ECFFD8B1072200212046FFF742FD8146B9F1000F17D00A2001E031E02AE0FFF750FC00226846D4F88810F3F73CFF6846A168F4
:407CC00088476846F3F73BFF04E00B20FFF740FC4FF0110905E0FFE70C20FFF739FC4FF01209B9F1000F07D1052084F89E0001203B4981F851010CE001212046FFF7A6FE7F
:407D000007E00D20FFF724FC4FF0100901E04FF00F0901E04FF00E094846BDE8FE8FF0B589B005460E4617461C46FF208DF81C008DF81D708DF81E008DF81F008DF8200098
:407D4000E0B28DF82100200A8DF82200200C8DF823000020029003900490059006202B46082207A9CDE900604FF4484004F020FB10B9012009B0F0BD0020FBE72DE9F041BE
:407D8000064600BF70680746002433E000252AE004EB84011248001D00EB4110103050F82500B8421ED14FF0FF3104EB84020C48001D00EB4210103040F82510064800687B
:407DC000804704EB84020649091D01EB4211C1F890000AE098200020C4BE1908F9FFFF066C4300106D1C192DD2D300BF192D00D202E0641C022CC9D3BDE8F0812DE9F04155
:407E0000044600270025002617B10E20FFF7A0FB012D02D10F20FFF79BFB012E02D11020FFF796FBAFF2CB2003F099FA21464FF4474003F037F921464FF4484003F032F9D4
:407E4000BDE8F08170B504460D462946FE48D4F848213BF1ECFD38B91120FFF779FBD4F84401401CC4F84401012084F85001D4F84C01401CC4F84C0170BD70B505460E46D4
:407E8000002421E004EB8401281D00EB411090F89E00C0B17EB104EB8401281D00EB41100068B04207D004EB8401281D00EB41104068B04207D104EB8402291D01EB42105C
:407EC0000121FFF7C3FD641C022CDBD370BD2DE9F04192B080460C4694F89E000A2853D2DFE800F0F8F705536C85C1F9F5F465682668D4F88800B0F1FF3F01D1E06898B37A
:407F000015208DF84000FF208DF8410001208DF8420000208DF843008DF8440014F88C0F8DF845002088000A8DF8460054F88C09000C8DF8470000200290039004900590B4
:407F400006203346082210A9CDE900504FF4484004F02EFAC0B9BD4800688047C4F89000032084F89E000FE0FFE7022229463046D4F88C30FFF7D3FE30B101212046FFF7D0
:407F800065FD1220FFF7E4FA4CE16568266841F28831D4F8900005F044FD70B1032229463046D4F88C30FFF7BAFE30B101212046FFF74CFD1320FFF7CBFA33E165682668ED
:407FC00040F6B831D4F8900005F02BFD70B1032229463046D4F88C30FFF7A1FE30B101212046FFF733FD1420FFF7B2FA1AE1783454F8785C54F8746C14208DF84000207FB1
:408000008DF84100A08B000A8DF84200E069000C8DF84300E069000E8DF84400207D8DF84500A08A000A8DF846006069783C000C8DF84700002002900390049005900620F2
:408040003346082210A9CDE900504FF4484004F0AFF938B97D4800688047C4F89000062084F89E00DEE025686668D4F89800B0B941F26801D4F8900005F0D3FC28B3032224
:4080800029463046D4F88C30FFF749FEE8B101212046FFF7DBFC1520FFF75AFA15E041F28831D4F8900005F0BCFC70B1032229463046D4F88C30FFF732FE30B1012120467D
:4080C000FFF7C4FC1520FFF743FAABE088E06EE001E0A6E0A4E02568666862E0FF2700200AE004F1100151F82010B1F1FF3F01D1074603E0411CC8B21928F2DB192F4EDAB3
:4081000010A92046FFF739FCB0B30021AFF2933204F1100000EB8700CDE9021007203346CDE90050CDE90421082210A94FF4474004F03EF908BBA06F401CA06794F89D0015
:40814000401C84F89D00414800688047C4F89000A06FC0EBC000D4F89410884203D3082084F89E001CE0D4F89810A06F884217D1062084F89E0013E000E016E002222946ED
:408180003046D4F88C30FFF7CAFD38B101212046FFF75CFC1620FFF7DBF901E005E004E000BF94F89E00072898D000BF3AE02568666841F28831D4F8900005F032FC70B15B
:4081C000032229463046D4F88C30FFF7A8FD30B101212046FFF73AFC1720FFF7B9F921E02069B0F1FF3F1AD1194BD4E90002D4F89410CDE90203CDE9001205A8E368E26F2B
:40820000D4F88C103BF115FB05A803F034FD00212046FFF71BFC05A83BF15EFB00BF01E000BF00BF00BF94F89E00A8B140F2DC51D4F8900005F0F5FB70B101212046FFF764
:4082400005FC182006E0000044420010C4BE190833A31908FFF77CF912B0BDE8F0812DE9F34F8DB00D4600200C906868002876D028680028FBD0286802689168884700281D
:408280006DD16F68D5F80090E868B0F5474F68D0B0F5484F73D1287D162871D004DC142807D015286DD10FE117286BD0FF28F9D177E2697EA87E41EA0021E87E41EA004891
:4082C000697DA87D41EA0021E87D41EA0041287E41EA00664A4639460D98FFF77CF80446002C5DD140F2FA6086424CD3FE48864249D80D98FFF707FC04468CB3C4F8009048
:4083000067600020A067FDF7BBFBC4F88800C4F88C80C4F894600020C4F8980084F89D0004F10C0004F17C01D4F89420CDE900210290EE48D4E90032D4F88C1004F04FFE32
:40834000EB4800688047C4F89000022084F89E0001200C9001210D9880F851112CE0B9E300E078E24346022239464846FFF7D7FC10B31920FFF7ECF801200C901CE0A1E33D
:408380001BE03FE2C3E14346FE2239464846FFF7C6FC88B11A20FFF7DBF801200C900BE04346012239464846FFF7B9FC20B11B20FFF7CEF801200C904BE2A97DE87D41EADF
:4083C0000021287E41EA004A697EA87E41EA0021E87E41EA00486E7D4A4639460D98FEF7FAFF0446002C62D0D4F88C0040454CD194F89E00032836D1FF2E22DCA06F5045B5
:408400000DD1BB480068804744F8900F00206073A6600420A073903C01200C9053E00C2239464846D4F88C30FFF779FC60B301212046FFF70BFB1C20FFF78AF801200C902F
:4084400041E00B2239464846D4F88C30FFF767FCD0B101212046FFF7F9FA1D20FFF778F801200C902FE0092239464846D4F88C30FFF755FC40B101212046FFF7E7FA1E20CA
:40848000FFF766F801200C901DE00A2239464846D4F88C30FFF743FCA8B101212046FFF7D5FA1F20FFF754F801200C900BE04346092239464846FFF732FC20B12020FFF7FD
:4084C00047F801200C90C4E1A97DE87D41EA0021287E41EA0046697EA87E41EA0021E87E41EA004A95F815803A4649460D98FEF772FF0446002C7DD094F89E0006287AD117
:40850000B8F1FF0F01DD4FF0FF08B8F1000F73D0A06F00F1010BD4F88C0050456DD15E450CD094F89C00022868DA002E66D0701EC0EBC000D4F8841088425FD3D4F8940002
:40854000401E0721B0FBF1F0401C08EB0601491E884276D308EB0600401EB0F1807F70D25E4503D1002084F89C0006E0701EA06794F89C00401C84F89C0016208DF8280037
:408580008DF8298014F8780F8DF82A002088000A8DF82B002068000C8DF82C00207D8DF82D00A08A000A8DF82E006069783C000C8DF82F000020029003900490059006209D
:4085C0004B4608220AA9CDE900704FF4484003F0EFFE00286AD1464800688047C4F89000A06F4044C4F89800002084F89D00A06F401C04E07EE065E059E046E033E0C0EBA1
:40860000C002A06FC0EBC0012046FFF789F828B9072084F89E0001200C9047E0FE2239464846D4F88C30FFF77AFB68B301212046FFF70CFA2120FEF78BFF01200C9035E0C9
:40864000FFE70F2239464846D4F88C30FFF767FBD0B101212046FFF7F9F92220FEF778FF01200C9022E0052239464846D4F88C30FFF755FB40B101212046FFF7E7F9232004
:40868000FEF766FF01200C9010E00E2239464846D4F88C30FFF743FB40B101212046FFF7D5F92420FEF754FF01200C902EE00020C4F898000E4800688047C4F890000120C0
:4086C0000C9023E0042239464846D4F88C30FFF726FBD8B101212046FFF7B8F92520FEF737FF01200C9011E0F9FFFF0698200020C4BE19085346FE2239464846FFF70FFBF5
:4087000020B12620FEF724FF01200C90A1E0697EA87E41EA0021E87E41EA00463A4649460D98FEF758FE044674B394F89E00082818D1697DA87D41EA0021E87D41EA0041C1
:40874000287E41EA0060D4F8941088420AD1D4F88C00B04206D100212046FFF777F901200C901DE0FE2239464846D4F88C30FFF7D6FAA8B101212046FFF768F92720FEF7FC
:40878000E7FE01200C900BE03346FE2239464846FFF7C5FA20B12820FEF7DAFE01200C9057E02920FEF7D4FE697EA87E41EA0021E87E41EA00464A4639460D98FEF70BFE05
:4087C000044654B1D4F88C00B04206D101212046FFF73CF92A20FEF7BBFE3A4649460D98FEF7F9FD044654B1D4F88C00B04206D101212046FFF72AF92B20FEF7A9FE0120A6
:408800000C9026E03A4649460D98FEF7E4FD04468CB1FE2239464846D4F88C30FFF77FFAB0B101212046FFF711F92C20FEF790FE01200C900CE04FF0FF33FE223946484662
:40884000FFF76DFA20B12C20FEF782FE01200C9000BF00BF3CE14A4639460D98FEF7BBFD0446002C79D094F89E00042876D1A06F401CC0EBC0000990A06FC0EBC008A06FF4
:4088800000F1010AD4F89400A0EB080008900AF1010BD4F89400A0EB0800401E0721B0FBF1F007902E7D0898072801D90720089094F89D00401CB0427ED10898CDE90080DF
:4088C00005F11503B548E268E16F04F0F3FA002873D0D4F894100998814240D817208DF828008C34207A8DF829002089000A8DF82A00A068000C8DF82B00A068000E8DF8EE
:408900002C0020788DF82D002088000A8DF82E0054F88C09000C8DF82F000021AFF6A33204F11000CDE9021006204B46CDE90070CDE9042108220AA94FF4484003F038FDCB
:40894000002809D1964800688047C4F89000092084F89E0001200C9093E0A5E092E0D4F89800B04248D115208DF828000798FF2803D9FF208DF8290003E00798C0B28DF8F9
:4089800029000BF0FF008DF82A004FEA1B208DF82B004FEA1B408DF82C0014F88C0F8DF82D002088000A8DF82E0054F88C09000C8DF82F00002001E03CE029E002900390D2
:4089C0000490059006204B4608220AA9CDE900704FF4484003F0ECFC58BB71480068804744F8900F44F818AC002060730320A073903C01200C9044E0694800688047C4F8A6
:408A00009000C4F878A084F89D6001200C9038E0022239464846D4F88C30FFF780F940B101212046FFF712F82D20FEF791FD01200C9026E094F89D00B04211D108223946AA
:408A40004846D4F88C30FFF76AF9D0B101212046FEF7FCFF2E20FEF77BFD01200C9010E0072239464846D4F88C30FFF758F940B101212046FEF7EAFF2F20FEF769FD0120FF
:408A80000C901EE0062239464846D4F88C30FFF746F9B0B101212046FEF7D8FF3020FEF757FD01200C900CE04FF0FF33062239464846FFF734F920B13120FEF749FD0120EC
:408AC0000C9005E03220FEF743FD01200C9000BF00BF0CE0686828B93320FEF739FD01200C9004E03420FEF733FD01200C900C980FB0BDE8F08F2DE9F041044694F850014C
:408B000001281FD1002084F85001002517E02548D4F848113AF1FBFF0646002766B1012084F8500131462046FFF799FB20B131461C483BF11EF8012707B902E06D1C0A2D05
:408B4000E5D300BF94F8510101281AD1002084F85101002513E005EB8501201D00EB411090F89E0050B1012084F8510105EB8502201D00EB42112046FFF7A9F96D1C022DD9
:408B8000E9D3BDE8F08110B50748FEF7B1FC0446064A07492FF04AFC10BD000098200020C4BE1908444200106C430010008000082F75010870B504460025022614B1012C5E
:408BC00006D102E0AE4D022602E0AE4D022600BF00BF25B132462946AB483CF1CAFF70BD10B50446A948206000206060A84AA949204604F099FA10B90020FFF7DBFF2046F3
:408C000010BD2DE9F04706460F46904674684FF0000A17B9B8F1000F36D008E02068B84204D16068404501D1A24602E0A468002CF4D100BFBAF1000F23D10C2030F07AFA9E
:408C400081460020C9F80000C9F804004D46C9F8080085B12F60C5F80480A860AA46706808B975600CE0746800E0A468A0680028FBD1A56004E00120FFF79CFF4FF0000A2B
:408C800005E04FF0000A02E00120FFF793FF5046BDE8F08770B505460E467C48286000206860746805E02846D4E90012FFF7A9FFA468002CF7D1764A7649284604F034FAA6
:408CC00010B90020FFF776FF284670BD10B50446206818B9606808B9A46006E0002020606060A060204630F01DFA10BD2DE9F04105460F466C680026B0460FE0A7420BD155
:408D000016B9A068686001E0A068B0602046FFF7DDFF4FF0010803E02646A468002CEDD100BF4046BDE8F08110B5044657482060574A5849204604F019FE03E02046616888
:408D4000FFF7D4FF60680028F8D1204610BD70B504462046FFF7E8FF054630F0E3F970BD0246002008604A480088824204DA4948006850F822000860086808B101207047C0
:408D80000020FCE742480088704770B505460C4600262CB1002221462846FFF732FF0646304670BD2DE9F04106460C461546002735B12CB12A4621463046FFF722FF07463A
:408DC0003846BDE8F08170B505460C4600262CB1224600212846FFF714FF0646304670BD2DE9F04106460F4674680025A846BFB114E06068B8420FD115B9A068706001E0C7
:408E0000A068A8602046FFF761FF4FF001080DB9746803E0AC6801E02546A468002CE8D14046BDE8F0812DE9F041074688467C6820E0266865680020206060603EB11DB1EE
:408E400029464046B04708E04046B04705E025B128684146826828469047A068A04203D026606560A46805E00020A060204630F059F901E0002CDCD100BFBDE8F081000020
:408E8000E7E7040817E80408CDE7040848C819084C0100104801001070B5044600250226082C1DD2DFE804F004070A0D10131619FB4D022614E0FB4D012611E0FA4D0126E6
:408EC0000EE0FA4D02260BE0F94D012608E0F94D012605E0F84D022602E0F84D022600BF00BF25B132462946F5483CF142FE70BD70B504460D4628197BF1C2FB27F1E8F891
:408F0000C0B200EE100AB8EE400ADFEDEE0A20EE200ABCEEC00A10EE100AC0B270BD2DE9F04104460D4690464346FE2229462046FDF7E0F80446E4480C3444F80C0C002072
:408F40006060A060E060206120756075FE20A075284630F094F80646FFF7CAFFE075002020766076A076E07601202077002060770C3CD64AD649204604F0D6F810B900201A
:408F8000FFF78AFF2046BDE8F08110B50446CE482060CE4ACE49204604F0E8FC2046FDF7C8F80446204610BD70B504462046FFF7ECFF054630F0B6F870BD02460020086041
:408FC000C2480088824204DAC148006850F822000860086808B1012070470020FCE7BB480088704730B591B00446132501F03CFF30B300208DF84000EE208DF84100002024
:409000008DF84200012000210622CDE90124CDE90310032010ABAF4A0121009006A83BF1A4F800BF9DF83C0005462DB906A8AA490968884700B90D2506A83AF13BFF00BFFD
:40904000284611B030BD024601207047704770470146002070470146487BFE2805DA91F82000082801D1012070470020FCE770B504460D4694F82000A84205D0974800681F
:409080008047606184F8205070BD10B50446207B022807DA607BFE2804DA617B207B00222FF0B2FEFE20607300212046FFF7DFFF002010346074FE20A07400202060A060BD
:4090C000E06020756075A075E0750120207600206076103C00BF204602F034FA00BF10BD014691F822007047014691F82000704770B504460D462046FFF7F6FF48B9FE2D03
:4091000002DA84F8225002E0FE2084F82200012603E00120FFF7C0FE0026304670BD014691F826007047014691F827007047014691F82800704780F82810704701460869F6
:409140007047014688697047002180F8261080F82710704770B504460E462046FFF7C4FF0D283FD2DFE800F0070809363738393A0A3B3C3D0B0000BF00BF00BF00BF94F8B4
:409180002200B04221D0FE2E17DA207B022814DA207B31467CF1C4FC38B9012584F8226004212046FFF763FF13E00025012084F829000220FFF770FE0BE00025012084F892
:4091C00029000320FFF768FE03E00025012084F829000CE000BF00BF00BF00BF00BF00BF00BF00BF00250420FFF756FE00BF00BF284670BD2DE9FC4705460C462846FFF70F
:4092000073FF0D2842D2DFE800F007080938393A3B3C0A3D3E3F400000BF00BF00BF4FF0010805F10409A24648462FF028FF06460F4650462FF023FF46404F403E4301D05B
:40924000012000E00020B8B120462FF018FF0646FFF74EFE85F823002E1D20462FF00FFFCDE90001009830600198706000BF00BF00212846FFF7FBFE0EE000BF00BF00BF4D
:4092800000BF00BF00BF00BF00BF00BF4FF000080520FFF701FE00BF00BF4046BDE8FC8750E8040880E80408A1E80408D6E8040804E904083EE9040875E90408A8E904085D
:4092C00036E804089A99193F24C80A084402002040020020FEFFEA00C0BE1908C4BE190810B5014600BF48680246002017E0F84B1B6853F82030DB6993420ED10123F44C33
:40930000246854F8204084F8243000BF0B7AF04C246854F8204084F82530431C98B2ED4B1B889842E3DB10BDF0B591B00446002701F09AFD002858D020462FF07CFE05463A
:409340000E46E8B28DF83C00280A40EA0660C0B28DF83D00280C40EA0640C0B28DF83E00280E40EA0620C0B28DF83F00F0B28DF84000300A8DF84100300C8DF84200300E0B
:409380008DF843000121AFF2A702207B0623CDE90130CDE903210820009094F82200CE4940EA01020FAB012105A83AF1DEFE00BF0998E06105A83AF1CBFD90B1002084F89C
:4093C000240084F8250005A8C44909688847012807D1C34800688047A061002084F82900012705A83AF166FD00BF384611B0F0BD10B504462046FFF777FE082805D1204653
:40940000FFF792FF08B1012010BD0020FCE770B590B00446002601F027FD00284ED02046FFF762FE0D2816D2DFE800F0090A0B0C0D0E0F10071112131400657B0DE000BFFA
:4094400000BF00BF00BF00BF00BF00BF00BF00BF00BF00BF00BFFE2500BF00BF00208DF83C00EE208DF83D0000208DF83E0001210022207B0623CDE90130CDE90321032096
:409480000090984845EA00020FAB05A83AF16DFE00BF0998E06105A83AF15AFD50B105A88E4909688847012804D18D4800688047A061012605A83AF1FDFC00BF304610B089
:4094C00070BD70B5044600252046FFF70DFE082807D12046FFF79BFF18B10125012084F82900284670BD2DE9F041044694F82800C8B9207B022807DA607BFE2804DA617BCF
:40950000207B00222FF080FCFE20607300212046FFF7ADFD00201C34607120602072607260731C3CFEE12046FFF7DEFD0D281CD2DFE800F0071C303946A0F8F7F6F5F4F348
:40954000F2002068016A2046884794F82200FE2807D194F82110206842692046904784F8220001212046FFF782FDDAE194F82900012804D103212046FFF779FD09E094F884
:409580002310606904F04DFA18B102212046FFF76EFDC6E12046FFF73AFF18B103212046FFF765FDBDE194F8232002F1FA01606904F037FA18B104212046FFF758FDB0E161
:4095C000002532E094F82210207B7CF1A9FA30B194F82210207B7CF1A3FAA04208D12046FFF7A2FE18B106212046FFF740FD23E0201D2FF035FD18B194F82100FE2801DB3E
:40960000012519E094F82100401C84F8210094F82110206842692046904784F8220094F82200FE2801DB012506E094F82200FE2802DA207B0228C5DB00BF012D0ED10020DD
:4096400084F8210094F82110206842692046904784F8220005212046FFF709FD94F82200FE2802DA207B022803DB0B212046FFF7FEFC56E164E094F82210207B7CF150FA9A
:4096800060B194F82210207B7CF14AFAA04205D094F82210207B7CF143FAC0B120462FF0CAFC05460E4694F82210207B7CF138FA07462FF0C0FC281A8E4115D22046FFF706
:4096C00033FE18B106212046FFF7D1FC3FE00BE0400200204402002000FFEE00C0BE1908C4BE190800FFEA00201D2FF0B9FC38B90B212046FFF7BBFC0620FFF7CDFB26E00B
:4097000094F82100FE280EDB0B212046FFF7AFFC0720FFF7C1FB1AE0F1E0E1E0C0E089E06AE03DE020E094F82100401C84F8210094F82110206842692046904784F82200F4
:4097400094F82200FE2802DA207B022893DB00BF94F82200FE2802DA207B022803DB0B212046FFF784FCDCE094F8240001280DD194F82500012804D107212046FFF777FCD3
:409780000DE004212046FFF772FC08E0FA21606904F047F918B104212046FFF768FCC0E0607BFE2823DA207B022820DA617B207B7CF1B6F9A04204D009212046FFF757FCA0
:4097C00019E0FA21606904F02CF940B108212046FFF74DFC2068C169204688470BE094F82900012807D12046FFF79EFD03E009212046FFF73CFC94E0607BFE2815DA207B95
:40980000022812DA617B207B7CF18AF9A04204D009212046FFF72BFC0BE094F82900012807D12046FFF780FD03E009212046FFF71EFC76E094F82200FE2830DA207B022852
:409840002DDA94F82210207B7CF16AF938B320462FF0F1FB05460E4694F82210207B7CF15FF907462FF0E7FB281A8E4108D22046FFF75AFD98B10A212046FFF7F8FB0EE002
:40988000002084F8210094F82110206842692046904784F8220002212046FFF7E8FB40E094F82400012811D194F82500012808D108212046FFF7DBFB2068C16920468847EE
:4098C0000DE009212046FFF7D2FB08E0FA21606904F0A7F818B109212046FFF7C8FB20E0002084F82100FE2084F822002046FFF71BFD18B10C212046FFF7B9FB11E094F847
:40990000290001280CD194F82200FE2804D10B212046FFF7ACFB03E004212046FFF7A7FB00BF00BFBDE8F08110B5002407E00649096851F82400FFF7D6FD601C84B20348C3
:4099400000888442F3DB10BD40020020440200200146FB48704710B50246052300200DE0141D04EB8014646A8C4205D1141D04EB801494F83B3003E0441CE0B20528EFDB16
:40998000184610BD0146D1F8440170470146D1F84C01704770B503460024002014E01D1D05EB80156D6A8D420CD101261D1D05EB801585F838601D1D05EB801585F83920E4
:4099C000012403E0451CE8B20528E8DB204670BD10B50446002120463BF155FE04460020203444F8140C44F8100C44F80C0C44F8080C401E44F8040C20606060A0600020AC
:409A0000E06020826082A082FF20A0750020E07520766076A076E07620776077203C204610BD10B5044620463AF148F90446C548206005234022AFF26701201D7CF171F963
:409A4000041F002004F5A274206039F1CDFF60600020A06020736073A4F5A274204610BD10B50446B748206005234022B649201D7AF139FF20463AF148F90446204610BDB0
:409A800070B504462046FFF7EBFF05462FF04AFB70BD70B5044600250226132C44D2DFE804F00A0D101316191C1F2225282B2E3134373A3D4000A54D022635E0A44D022642
:409AC00032E0A44D02262FE0A34D02262CE0A34D022629E0A24D022626E0A24D022623E0A14D022620E0A14D02261DE0A04D02261AE0A04D022617E09F4D002614E09F4D7A
:409B0000022611E09E4D00260EE09E4D00260BE09D4D002608E09D4D022605E09C4D012602E09C4D012600BF00BF25B13246294683483CF11EF870BD70B5054600BF6868AB
:409B40000646002413E0944800EB8410C069B0420BD100BF287A10B90020FFF79AFF01218D4800EB841080F83A10601CC4B2052CE9DB70BD2DE9FE43054600BF6868804614
:409B80000024AAE0844800EB8410C069404578D12868816828468847002873D0012872D0022802D003286FD186E02F46FF22082101A87AF147FE00BFB869B0B9764800EB52
:409BC0008410008E072807DC734800EB841090F830008DF8040002E0FF208DF80400012201A9384639F187FD63E06B4800EB8410008E072825DC684800EB8410806960B1D7
:409C0000654800EB8410028E634800EB841000F1180101A82EF088FC0DE05F4800EB8410008E00905C4800EB8410002301AA016A5A4802F029FF072201A9384639F15BFDCD
:409C400037E000BFD7F81C9038467CF11AF8A9EB0006082E00D908264F4800EB8410806998B138467CF10DF8411E4B4800EB8410806901EB00093246494601A87AF19DFD83
:409C800012E028E016E016E023E038467BF1F9FFA0F10109404800EB841000964B4601AA016A3E4802F0F0FE324601A9384639F122FD0EE000BF00BF00BF287A10B90120F4
:409CC000FFF7E7FE0121344800EB841080F8371000BF00BF04E0601CC4B2052CFFF652AFBDE8FE8370B504460D46002C26D02B48216A02F064FF20463BF15AFC0020203479
:409D000044F8140C44F8100C44F80C0C44F8080C401E44F8040C20606060A0600020E06020826082A082FF20A0750020E07520766076A076E07620776077203C70BD000063
:409D400067AA19080CC90A08EF5B190886AA1908B3AA1908D8AA190828AB190846AB190860AB19087CAB190897AB1908B3AB1908D2AB1908E7AB190815AC190848AC190849
:409D800077AC1908ABAC1908E2AC190805AD190811AD190836AD1908C4440010982000202DE9F04F89B006460F4614469846DDE9149BDDE9125AE0B28DF81C0011208DF89B
:409DC0001D009DF81D0008F0070140EA41008DF81D009DF81D0004F4E06140EAE1008DF81D00E8B28DF81E00280A8DF81F00280C8DF820008DF821A009F0FF008DF822001E
:409E00004FEA29208DF8230000211698CDE9021BCDE9040106203346082207A9CDE900704FF4584002F0C4FA18B9012009B0BDE8F08F0020FAE72DE9F84304460D4601268C
:409E400020462FF007F9A8B1002600BFE06888B120462FF0FFF8074620467BF112FF8146E068804600974B464246F648296A02F07BFF06463046BDE8F88370B504460025BA
:409E800015B10220FFF705FEEF48006810B90320FFF7FFFDED48006810B90420FFF7F9FDEB48006810B90520FFF7F3FDE948006810B90620FFF7EDFDE748006810B9072070
:409EC000FFF7E7FDE548006810B90820FFF7E1FD21464FF4594001F0E5F821464FF4574001F0E0F870BD30B50346002401B9DAB1002017E01D1D05EB801595F83D507DB131
:409F00001D1D05EB80152D698D4209D11D1D05EB8015ED68954203D11D1D05EB801403E0451CE8B20528E5DB204630BD2DE9F04704460D4600BF05F10C00F1F7E1FE0746C9
:409F4000B7F5574F15D0B7F5594F48D12946C448D4F8482139F16BFD38B90920FFF799FDD4F84401401CC4F84401012084F8510139E000BF68688046A8688146424649469C
:409F80002046FFF7B0FF064606B3B64800688047F06230463BF112FCB0F1FF3F0DD1294630463BF111FBC8B90A20FFF772FDD4F84401401CC4F8440110E00B20FFF769FD93
:409FC000D4F84401401CC4F8440107E00C20FFF760FDD4F84401401CC4F8440103E01020FFF757FD00BF00BFD4F84C01401CC4F84C01BDE8F08770B505460E46002419E0C9
:40A00000281D00EB841090F83D0090B15EB1281D00EB8410C068B04205D0281D00EB84100069B04205D1291D01EB84100121FFF759FE641C052CE3D370BD2DE9F04F91B040
:40A0400082460C4694F83D00082872D2DFE800F0F9F804F7F6F5F4F3E56894F83A00012868D1804800688047E06294F83B0008287ED2DFE800F00413B9CBCCCDBDCE94F81D
:40A080003670A06A40EA0761628E2846704F636A3F68B847052084F83D00C0E00020109004F1140010AB04F13001021DCDE9031302920590618E606ACDE9001094F8363021
:40A0C00094F83C102846634FA26A3F68B8479DF8400000281AD1A069C8B1218E04F12002584802F0C1FD78B1208E009000235548A269216A02F038FE30B95248216A02F051
:40A100005EFD4FF0FF3020620020A06168E06069002865D0218E04F120024A4802F0A4FD00285DD04FF000080027B9464FF0010B50E002E274E0208EB84239D90122218E59
:40A14000606A3B46CDE90018CDE902022246AFF2193105A839F198FA05A86169884708F1010800BF9DF83D0040B100BF089800E050E030B905A82EF06DFF10B14FF0000BEC
:40A1800012E005A82EF066FF60B100BF9DF83C0008B94FF0000B05A82EF05CFF07444FF0000901E009F1010905A839F190FA06E0208EB84202D24FF0000B00E00EE0BBF1AC
:40A1C000000F07D11F48216A02F0F9FC4FF0FF30206203E009F101000028ACD100BF00BF052084F83D001AE0042084F83D0016E094F83630A06A40EA03612846174B626ADD
:40A200001B689847052084F83D0008E000BF00BF00BF00BF01212046FFF764FD00BF09E041F28831E06A03F0FCFB18B101212046FFF758FD81E14BE121E185E03DE013E0B2
:40A2400070E16EE198200020F0EB0408F4EB0408F8EB0408FCEB040800EC040804EC040844420010C4BE19082669E5684FF4FA71E06A03F0D6FBA8B100204FF6FF72FF239C
:40A28000CDE9022001930490D01C0090628E052331462846FFF784FD70B101212046FFF721FD09E041F28831E06A03F0BAFB18B101212046FFF716FD3FE1E56894F83B009C
:40A2C00008283AD2DFE800F0323304343536373820463BF173FAB0F1FF3F1CD0012321460DA8626AF1F73AFC54F8240FA17CCDE90010227E0DA92846FD4F63683F68B8471D
:40A30000FC4800688047A06005206076243C0DA8F1F736FC09E047F23051E06A03F081FB18B101212046FFF7DDFC0BE000BF00BF00BF00BF00BF00BF00BF01212046FFF762
:40A34000D1FC00BF00BFF8E02669E56894F83800012871D194F8390001286FD194F83B00082863D2DFE800F0440445464748494A208EB0F5DF6F25DCA06918B9206AB0F102
:40A38000FF3F1FD0208E471C082F00D208270021AFF61F0204F11C00CDE9021006202B46CDE90060CDE904213A464FF4574001F0FFFF30B9CF4800688047E062062084F883
:40A3C0003D0014E000204FF6FF72FF23CDE9022001930490581C0090628E052331462846FFF7DEFC18B101212046FFF77BFC22E000BF00BF00BF00BF00BF00BF00204FF6C4
:40A40000FF72FF23CDE902200490CDE90003628E042331462846FFF7C3FC30B1B54800688047E062072084F83D0004E001212046FFF758FC00BF21E016E0FFE700204FF6CD
:40A44000FF72FF23CDE9022001930490581C0090628E052331462846FFF7A2FC70B101212046FFF73FFC09E047F23051E06A03F0D8FA18B101212046FFF734FC5DE02669E5
:40A48000E56894F83700012817D100204FF6FF72FF23CDE902200490CDE90003628E042331462846FFF77CFC88B1924800688047E062072084F83D0009E041F28831E06A71
:40A4C00003F0AFFA18B101212046FFF70BFC34E02669E5684FF4FA71E06A03F0A2FAA8B100204FF6FF72FF23CDE9022001930490D01C0090628E052331462846FFF750FCEF
:40A5000070B101212046FFF7EDFB09E041F28831E06A03F086FA18B101212046FFF7E2FB0BE000BF4FF4FA61E06A03F07AFA18B101212046FFF7D6FB00BF00BF11B0BDE8E9
:40A54000F08F70B505460026002418E0281D00EB841090F83D0080B9664800688047291D01EB8411C8620121281D00EB841080F83D10281D00EB841603E0601CC4B2052C9F
:40A58000E4DB304670BD2DE9F04F89B006460D4600200890686800287ED0286800287CD0E868B0F5594F79D12868026891688847002874D1D5F804902F68A97DE87D41EA46
:40A5C0000021287E41EA004A297D687D00F0E00041EAC00BA97EE87E41EA00200790687E0690687DC0F34208687DC0F3001005903A4649463046FFF776FC0446002C7DD113
:40A600003046FFF79EFF0446002C78D020463AF1CFFFE760C4F8109000206061A061401EE0612062FBF72CFA6062C4F828A0069884F83600059884F83C00A4F832B084F851
:40A640003B804FF6FF70A0862A4800688047E0620020208684F8370084F8380084F8390084F83A0004F13400009094F83B2049463846DFF884C0079BDCF800C0E04701287C
:40A6800021D10021A08EFF23CDE90201481ECDE900030491628E03E087E180E178E176E10B4649463846FFF77BFB38B1032084F83D00012086F85001089067E10121204697
:40A6C000FFF710FB62E1022084F83D00AFF6973104F11C004FF6FF72FF23CDE90132CDE903014FF0FF300090628E0023494607E000EC0408C4BE1908F0EB040823E00DE049
:40A700003846FFF74DFB20B1012086F8500108903CE101212046FFF7E5FA37E100204FF6FF72FF23CDE9022001930490022001230022494600903846FFF732FB0028BCD09E
:40A740000120089022E194F83D00082878D2DFE800F0878889048A8B8C78A06A504558D1608E584555D194F836100698814250D194F83B0040454CD194F83C100598814200
:40A7800047D107980090A38E94F83B2049463846DFF8C8C2DCF800C0E047012821D1022084F83D00002084F83A00AD4800688047E062AFF67B4104F11C004FF6FF72FF2395
:40A7C000CDE90132CDE903014FF0FF300090628E002349463846FFF7E3FA88B3012008902EE000204FF6FF72FF23CDE902200193049041F2030001230022494600903846B2
:40A80000FFF7CEFAE0B10D20FFF743F90120089016E000204FF6FF72FF23CDE90220019304904FF4805001230022494600903846FFF7B6FA20B10E20FFF72BF90120089055
:40A84000A3E0B8F1040F04D100212046FFF74AFA03E001212046FFF745FA0120089094E000BF00BF00BF00BF00BF0F20FFF711F994F83B00082874D2DFE800F00416283ADC
:40A8800071724C5E00204FF6FF72FF23CDE9022001930490102001230022494600903846FFF77EFA08906EE000204FF6FF72FF23CDE90220019304901120012300224946AE
:40A8C00000903846FFF76CFA08905CE000204FF6FF72FF23CDE9022001930490122001230022494600903846FFF75AFA08904AE000204FF6FF72FF23CDE902200193049009
:40A90000132001230022494600903846FFF748FA089038E000204FF6FF72FF23CDE9022001930490162001230022494600903846FFF736FA089026E000204FF6FF72FF234C
:40A94000CDE9022001930490172001230022494600903846FFF724FA089014E001E000BF00BF00204FF6FF72FF23CDE90220019304901F2001230022494600903846FFF7AE
:40A980000FFA089000BF00BF00BF00BF00BF05E01020FFF77EF80120089000BF0AE01120FFF777F80120089004E01220FFF771F801200890089809B0BDE8F08F2DE9F04117
:40A9C000044694F8510101281FD1002084F85101002517E02348D4F8481139F198F80646002766B1012084F8510131462046FFF7CAFD20B131461B4839F1BBF8012707B93F
:40AA000002E06D1C0A2DE5D300BF94F85001012816D1002084F8500100250FE0201D00EB851090F83D0040B1012084F85001201D00EB85112046FFF700FB6D1C052DEDD31E
:40AA4000BDE8F08110B50848FEF7EBFF0446074AAFF6F3712DF0EAFC10BD0000F4EB0408C4BE190844420010C0440010008000082DE9FF4F85B081468A461C46129EF64818
:40AA8000056800203060022C78DA804600273BE0002000900490C4EBC410F04901EBC00050F8270098B1C4EBC4100A4602EBC00050F8271002A82EF0C4FA0120049002AAA7
:40AAC000504607993AF1EFFB08B1012000E0002083460190049810B102A83AF1E3FB00BF009883450ED0C14508D1C4EBC410DB4901EBC00050F82700306007E008F10100B8
:40AB00001FFA80F8781CC7B2FE2FC1DB3068A0BB30E04FF0000B00200490686888B16868007BA0420DD102A869682EF08AFA0120049002AA504607993AF1B5FB08B1012030
:40AB400000E0002007460190049810B102A83AF1A9FB00BF5F4508D0C14502D1686830600AE008F101001FFA80F828467AF18EFF054600BF002DCCD100BF00BF306818B11F
:40AB8000012009B0BDE8F08F0020FAE7F8B506460C46154623460022114630460095FFF767FFF8BD2DE9F74F82B01446AA4805680027022C5FDA00262EE04FF0000BD94680
:40ABC000C4EBC410A54901EBC00050F8260098B1C4EBC4100A4602EBC00050F8261068462EF02FFA4FF001096A46DDE902013AF15AFB08B1012000E000208246D046B9F1EA
:40AC0000000F02D068463AF14DFB00BFD84501D0781C87B2701C86B2FE2ECEDB29E04FF0000AD046686888B16868007BA0420DD1684669682EF005FA4FF001086A46DDE929
:40AC400002013AF130FB08B1012000E0002081464E46B8F1000F02D068463AF123FB00BF564501D0781C87B228467AF10FFF054600BF002DD3D1384605B0BDE8F08F10B5EF
:40AC80000446224600210846FFF78CFF10BD2DE9F74F82B00E4615466F48076800202860022E6CDA00242DE04FF0000BD9466C48006850F82400007BB0420FD1684800681D
:40ACC00050F8241068462EF0BCF94FF00109694602982EF002FA08B1012000E000208246D046B9F1000F02D068463AF1DBFA00BFD84505D05A48006850F82400286005E026
:40AD0000601C84B2574800888442CDDB00BF2868A0BB002436E04FF0000BD946C6EBC6104E4901EBC00050F8240090B1C6EBC6100A4602EBC00050F8241068462EF081F9C2
:40AD40004FF00109694602982EF0C7F908B1012000E000208246D046B9F1000F02D068463AF1A0FA00BFD8450AD0C6EBC6103B4901EBC00050F82400286005E005E035E06D
:40AD8000601C84B2FE2CC6DB00BF286868BB29E04FF0000BD946786880B17868007BB0420CD1684679682EF04CF94FF00109694602982EF092F908B1012000E00020824628
:40ADC000D046B9F1000F02D068463AF16BFA00BFD84502D07868286006E038467AF156FE074600BF002FD3D100BF00BF286818B1012005B0BDE8F08F0020FAE72DE9F04143
:40AE000006460C46144805680027002020600AE0B74202D16868206007E028467AF136FE0546781C87B2002DF2D100BF206810B10120BDE8F0810020FBE770B506480468C2
:40AE4000002505E020467AF121FE0446681C85B2002CF7D1284670BD54010010144600104002002044020020FA480078704770B5044600250226102C39D2DFE804F0080B6B
:40AE80000E1114171A1D202326292C2F3235F24D02262CE0F14D022629E0F14D022626E0F04D022623E0F04D022620E0EF4D02261DE0EF4D02261AE0EE4D012617E0EE4D4F
:40AEC000012614E0ED4D012611E0ED4D01260EE0EC4D01260BE0EC4D012608E0EB4D022605E0EB4D022602E0EA4D022600BF00BF25B132462946E8483AF13BFE70BD0160C0
:40AF00004260836070472DE9F04705460E4617461C464FF0000A0EB9002F60D0022C5EDADE4830F814004FF6FF71884257DA00201FE0DB4951F8241051F820100968B142A6
:40AF400015D1D74951F8241051F820104968B9420DD1D34951F8241051F820108968A94205D1CF4951F8241051F820A006E0411C88B2CA4931F814108142DADCBAF1000FD9
:40AF800027D10C202EF0D6F880462B463A463146FFF7B5FF8046C146B9F1000F13D0CA46BE4800EB4402BE4800EB8401484602F0BBF868B90620FFF75AFF48462EF0B2F864
:40AFC0004FF0000A04E00620FFF751FF4FF0000A08E00620FFF74BFF4FF0000A02E00620FFF745FF5046BDE8F0872DE9F04107460D4600268DB1012600240CE023460022D7
:40B0000029463846FFF77FFF08B1012000E000200640601CC4B2022CF0DB3046BDE8F0812DE9F04106460C461546002734B12B46002221463046FFF766FF07463846BDE891
:40B04000F0812DE9F04180460D461646002796B18DB1012700240CE02346324629464046FFF751FF08B1012000E000200740601CC4B2022CF0DB3846BDE8F0812DE9F041BC
:40B0800006460C4615461F464FF000083DB134B13B462A4621463046FFF735FF80464046BDE8F0812DE9F04107460C4600268CB1012600250CE02B46224600213846FFF7CF
:40B0C00022FF08B1012000E000200640681CC5B2022DF0DB3046BDE8F0812DE9F04106460C461546002734B12B46224600213046FFF709FF07463846BDE8F0812DE9F041AC
:40B1000004460D4617461E46DDF818802046FAF7A0FC04466560A760E660C4F810802046BDE8F0812DE9F84F05460E46174699465C4804684FF0000A0DB9002E38D011E0AF
:40B140006068A8420AD1A068B04207D1E068484504D12069B84201D1A24605E020467AF195FC0446002CEBD100BFBAF1000F19D114202DF0DFFF80464B46324629460097A9
:40B18000FFF7BCFF8046444644B1A246214645480068FAF7ABFB4349086002E00E20FFF766FE08E00E20FFF762FE4FF0000A02E00E20FFF75CFE5046BDE8F88F2DE9F04142
:40B1C00004460D461646002734B133462A4600212046FFF7A7FF07463846BDE8F0812DE9F04104460D4616461F464FF000083CB135B13B46324629462046FFF793FF804682
:40B200004046BDE8F0812DE9F04104460D461646002734B133462A4621460020FFF782FF07463846BDE8F08170B504460D4616462046FAF70EFC04466560A660204670BD37
:40B240002DE9F04105460E46174804684FF0000865B338E074010010ADAD1908D2AD1908FAAD190834AE19085FAE19088CAE1908ABAE1908D5AE190802AF190828AF1908CA
:40B2800065AF190888AF1908B1AF1908E2AF1908FAAF190827B0190860AD19087001001060010010580100105C0100102FE06068A84204D1A068B04201D1A04605E0204683
:40B2C0007AF1E4FB0446002CF1D100BFB8F1000F17D10C202DF02EFF074632462946FFF7A3FF07463C4644B1A0462146FE480068FAF7FCFAFC49086002E00020FFF7B7FD2C
:40B3000008E00020FFF7B3FD4FF0000802E00020FFF7ADFD4046BDE8F08170B50446002524B100212046FFF78BFF0546284670BD70B504460D4600262CB125B12946204614
:40B34000FFF77EFF0646304670BD70B504460D462046FAF77EFB04466560204670BD2DE9F0410546E1480468002735B308E06068A84201D1012705E020467AF187FB0446EB
:40B38000002CF4D100BFB7B908202DF0D3FE06462946FFF7DAFF0646344644B101272146D2480068FAF7A2FAD049086002E00120FFF75DFD04E0002702E00120FFF757FD48
:40B3C0003846BDE8F0812DE9FF4F89B0044617AD95E8E00F002008906068B8B1A06858B1A0688DE8E00F0790D4F804C0169B0AA807C8E047089019E08DE8E00FD4F804C037
:40B40000169B0AA807C8E04708900FE0A06868B104A8A0E8000F16988DE8E100A0680168D1F80CC00AA90EC9E047089008980DB0BDE8F08F2DE9FF4F89B006460F469846D8
:40B44000DDE917ABDDF85890A9480468002522E021690B9881421AD1E06828B1E068B04202D0E068B84212D1DDE91923DDE91B108DE8000FCDE90423CDE906103A463146BF
:40B4800020460B9BFFF79FFF054605B105E020467AF1FCFA0446002CDAD100BF4DBB9448046823E06FF07F41206988421AD1E068C0B1E068B04202D0E068B84212D1DDE9FF
:40B4C0001923DDE91B108DE8000FCDE90423CDE906103A46314620460B9BFFF774FF054605B105E020467AF1D1FA0446002CD9D100BF1DBB7E4804681DE06FF07F41206976
:40B50000884214D1E06890B9DDE91923DDE91B108DE8000FCDE90423CDE906103A46314620460B9BFFF74FFF054605B105E020467AF1ACFA0446002CDFD100BF28460DB0F7
:40B54000BDE8F08F2DE9F04105466A480468002719E06068A84212D1214666480068FAF76DFA644908600020606034B126463046FAF772FA80462DF0D5FD012705E020462C
:40B580007AF184FA0446002CE3D100BF3846BDE8F08170B504460D462046FAF75AFA04466560204670BD2DE9F041054651480468012708E06068A84201D1002705E0204679
:40B5C0007AF164FA0446002CF4D100BF012F13D108202DF0AFFD06462946FFF7DAFF064634463CB1214643480068FAF77FF94149086000E0002700BF3846BDE8F0812DE921
:40B60000F34F9DB006463068816930468847804630462DF009FD189000BF307D04463046FAF754FB05463046FAF733FB8146002014901898B0F56A4F71D0B0F56E4F05D004
:40B64000A0F57E40D83800286AD189E2FE2D68DAB9F1FF0F65D1B8F1080F7DD13068082215A90369304698470128F6D1C4EBC410214901EBC00050F8250019909DF8540067
:40B6800000239DF85520190241EA12611702384343EA01029DF856300021090441EA13411F04134640EA070243EA01009DF857300021090641EA132142EA036201439DF826
:40B6C000580008439DF859100B02114618439DF85A2040EA02409DF85B2040EA0260CDE91A104FF0000A09E05C0100106801001058010010540100101446001000201390E0
:40B70000199850B111A819992DF09BFC0120139011A91AA839F150FC20B1012003E0C9E1A3E2B9E1002007461090139810B111A839F1B8FD00BF57457ED0199878B1FE2032
:40B74000199948731998FFF72EFF0020C4EBC411FC4A02EBC10100E09AE141F825000020199000270EA8DDE91A2339F145FC19AA21460D90FFF78BFA80F0010080F0010AF4
:40B78000D3460EA839F18EFDDA46BA451CD01998407BFE280ADA0020C4EBC411E94A02EBC101199A527B41F8220002E01998FFF7C9FE19984573C4EBC411E24A02EBC1010B
:40B7C000199841F8250061E101201490DE4850F82400401CDC4941F824004FF0000B64E0002008900DA90C90584603F0FAFB70B10AA8DDE91A2339F1FFFB012022460C9086
:40B800000AA90D9803F025FC08B1012000E00020074609900C9810B10AA839F143FD00BF089887423DD00D981990002707A819992DF007FC07A900E029E1C44839F19CFBC9
:40B840000690059007A839F12DFD0598B84227D01998407BFE2809DA0020C4EBC411B94A02EBC101199A527B41F822001998071D04A8DDE91A2339F1BFFB029002982DF0B5
:40B88000FEFBCDE90001009838600198786000BF00BF039704A839F105FD1998457308E000BF0BF101001FFA80FB03F0ACFB584596DC1E9801287CD1199800287AD1002786
:40B8C0005FE0002007900CA90B903846FBF74CFDF8B10C98007AA0421BD10C98807AC0B10C980068A8B109A8DDE91A2339F184FB01200B900C9A917A106809AA39F1D3FC52
:40B9000038B10C98C07A0C99497A884201DA012000E00020834608900B9810B109A839F1C1FC00BF0798834529D0002007901C202DF000FC834605A8DDE91A2339F15CFB90
:40B9400001200023079005AA2146584603F0D6FA0D90079810B105A839F1A4FC0D9845730C98C07A401C0C99C8720C98406818B10C9841680D9888470D98199005E0781CEE
:40B9800087B2FBF703FDB8429BDC1998F0B94FF0000B10202DF0CEFB07460AA8DDE91A2339F12AFB4FF0010B23462A460AA9384601E040E00BE03CF103FC07461990BBF1D1
:40B9C000000F02D00AA839F16DFC00BF55E04FF0000B0BA819992DF034FB0BA91AA839F1EBFA07460A900BA839F15CFC0A9F5F4520D019980D9000200A9010202DF09AFB6A
:40BA0000834608A8DDE91A2339F1F6FA012023462A460A9008A958463CF1D2FB834619900A9810B108A839F13DFC0DA919A803F06EFC00BF21E0002009908346199860B1D3
:40BA40000BA819992DF0FDFA4FF0010B0BA91AA839F1B2FA08B1012000E0002007460A90BBF1000F02D00BA839F11CFC00BF0998874201D00020199000BFC4EBC411314AF2
:40BA800002EBC101199841F8250000BF00BF0CE00720FFF7ECF908E0FE2D03D10820FFF7E6F902E00920FFF7E2F93068016A30468847DBE0B8F1030F4ED3B8F1080F4BD8DA
:40BAC0003068082215A9036930469847012843D19DF854009DF8551040EA01209DF8561040EA0140B0F56E4F2AD100BF70681990199850B11998006881681998884720B98A
:40BB00000120199981F8290019E0B9F1FF0F16D1002710E00E49096851F827007AF1AEF8A04206D101200A49096851F8271081F82900781C87B2074800888742EADB00BFE7
:40BB40000DE0000014460010384E001058AD190840020020440200200A20FFF788F985E0B9F1FF0F7DD1B8F1090F76D13068092215A903693046984701286ED1002011906B
:40BB800030462DF021F919909DF8540000239DF855101A0242EA11620F02384343EA02019DF856201B0443EA124340EA024241EA03009DF857300021090641EA132142EA93
:40BBC000036201439DF8580001439DF859000302104641EA03029DF85A100F04014642EA07009DF85B2040EA0260CDE91A100020109082461998D8B112A8DDE91A2339F141
:40BC0000FBF94FF0010A11AA214612A8FFF73FF870B11198006881681198884740B9119800688269199911989047012800D100E0002083465F46BAF1000F02D012A839F12B
:40BC400031FB00BF1098874204D09DF85C101198FDF780FA08E004E0FFE70B20FFF707F902E00C20FFF703F900E000BF00BF14981FB0BDE8F08F2DE9FC5F0746F848007836
:40BC8000012878D1002F76D0F64800688047834600BF387D04463868016A38468847022C6ADA00BF7868064638688169384688474FEAC009386881683846884700285CD0F1
:40BCC000012802D0022859D100E000BF384679F1B6FFE549C1F8940038680822B431036938469847E048543050F82400401CDE49543141F8240001F1200040F824B03846AD
:40BD000079F1A3FFD8B1012833D1D748443050F8241009F140000144D348443040F824100520B9FBF0F048444B30CF494C3151F824100144CC484C3040F8241019E0CA489A
:40BD4000443050F8241009F12C000144C648443040F824100520B9FBF0F048443330C2494C3151F824100144BF484C3040F8241000BF00BF02E038E1FCE000BF00BF386826
:40BD8000C1693846884701287AD13846F9F781FFFF2807D0002E73D030688168304688470028F1D138462DF03FF9019001213846FFF725FC00903846F9F76BFFFF281ED1F2
:40BDC000002517E0A948006850F82500B0420FD0A649096851F8250079F150FFA04207D1A04800688047A149096851F825100861681C85B29E4800888542E3DB0CE000BF9D
:40BE00007868064646B1306881683046884718B9944800688047306138462CF0D5FF0646002E7DD0009801281AD19248D0F8008012E0D8F8040058B1D8F8080020B13046BB
:40BE4000D8E90121904703E03046D8F804108847404679F11BFE8046B8F1000FE9D100BF3068816830468847012807D17D4800688047B0613946304603F07FFA002554E076
:40BE800059E07D4850F8240050F8250081680198814209D0784850F8240050F8250080686FF07F4188423ED1734850F8240050F825000068F0B1704850F8240050F82500E6
:40BEC000406870B16C4850F8240050F825004168694850F8240050F8250002683846904721E0654850F8240050F8250001683846884718E0604850F8240050F8250040689C
:40BF000088B15D4951F8241051F8251048685A4951F8241051F82510496809688A6800E008E039469047681C85B2544830F81400A842A6DC00BF38688168384688470128EA
:40BF400017D138462CF040FF064696B1306881683046884768B938462DF066F8B0F56E4F02D1012086F82700012086F8260086F8290000BF002516E04149096851F82500E3
:40BF80003F49096851F8251009688A6839469047012806D13A49096851F825003946FCF742FF681C85B2374800888542E4DB2D48006880470646594601F0A8FC82462A4896
:40BFC000D0F89810514507D2C0F898A0384679F136FE2549C1F89C002348B0F8AE00504502D20220FEF743FF00BFBDE8FC9F2DE9F04106460027002426E000251AE01E48A8
:40C0000050F8240050F82500B04211D11A4B53F8243053F82500194B03EB4402164B03EB840101F0A3FC30462DF07CF8012706E0681C85B2114830F81400A842DFDC012FA9
:40C0400000D103E0601C84B2022CD6DB3846BDE8F0812DE9F041064600279EB300242FE074010010C4BE1908044E001040020020440200205C0100106001001070010010F8
:40C08000480100104C010010002512E0F74850F8240050F825004068B04208D1F34951F8241051F82500FFF7A2FF074301E0681C85B2EF4830F81400A842E7DC601C84B2B2
:40C0C000022CE1DB3846BDE8F081F8B505462C46002000906A462146E6480068F9F78EFCE44908609DF80000012807D134B126463046F9F7B1FC07462DF014F89DF80000E7
:40C10000F8BD2DE9F0410446DA480568002774B10BE0284679F1BAFC0646A868A04203D12846FFF7D2FF07433546002DF1D13846BDE8F081F8B505462C46002000906A460C
:40C140002146CD480068F9F759FCCB4908609DF80000012807D134B126463046F9F77CFC07462CF0DFFF9DF80000F8BD2DE9F04704460D46012620462CF06CFFD8B1002617
:40C1800000BFE068B8B100BF276A20462CF062FF3918E06981420ED8012620462CF05AFF8146E0680746206A00EB05084A463946404678F102FB3046BDE8F0872DE9FF4FC8
:40C1C00095B0834690461C46DDF88C90DDE92857132615B14FF0FF302860A848007801287AD10026BBF1000F03D0BBF1010F74D124E0082C20D8229A2A99269801AB85C3DC
:40C200000491E0B24346009059460BA8169A37F1ACFF00BF9DF8500006464EB915B100BF0F9828600BA896490968884700B90D260BA837F13FFE00E00826B4E0082C7DD83D
:40C24000B8F1000F5AD12798002857D1002F55D08246401E12900020119010900DF14C0825B1F9F70DFC12901298286040E0A2453BD20122109912985346CDE90041CDE98A
:40C28000020213AAAFF21B1105A837F1FDF905A8B8471098401C80B2109000BF9DF83D0030B100BF089828B905A82CF0D3FE08B1142616E005A82CF0CDFE78B105A82CF0E8
:40C2C000C9FE5044A04200D9082605A82CF0C2FE82440020119004E066E05FE01198401C119005A837F1F3F900E005E006B103E01198401C0028BAD100BF00BF5EBBDDE9A6
:40C3000024122A9802AB86C305902698E3B24246CDE9000909A8169937F15DFE00BF9DF8480006469EB915B100BF0D98286009A853490968884710B90D2608E00CE0B9F105
:40C34000000F04D04F4800688047C9F8180009A837F1B0FD00BF20E00E264B48D0F800A012E0279924988DE8A3004B4622464146DAF804C01698E04706460E2E00D00AE014
:40C38000504679F183FB8246BAF1000F03D0DAF804000028E5D100BF00BF04E001260D20FEF765FD00BF00BF304619B0BDE8F08F2DE9F04F8BB005460E4617461C46DDE954
:40C3C000159ADDF850800B200A90CCB1204679F155FC8346DDE917211998CDE905A2CDE90710FF203B4632462946CDE900B4CDE90309CDF808800120FFF7E0FE0A9002E073
:40C400000520FEF734FD0A980BB0BDE8F08F2DE9F04F8BB005460E4617461C46DDE9159ADDF850800B200A90C4B1204679F126FC8346DDE917211998CDE905A2CDE907105A
:40C4400000203B4632462946CDE900B4CDE9038902900120FFF7B2FE0A9002E00520FEF706FD0A980BB0BDE8F08F00006001001070010010580100105C01001074010010C8
:40C48000C0BE1908C4BE1908680100102DE9F0438DB006460C4615461F46DDF850804FF0150900200C900B900A90099006200890002007900BA80AA907AA08ABCDE9033227
:40C4C000CDE9051009A80CA93B463246CDE90081029029462046FEF7ADFF012814D100209DF81C30DDE90A21CDE90232CDE904109DF820002346CDE900503046099A0C993D
:40C50000FFF756FF814602E00F20FEF7B0FC48460DB0BDE8F0832DE9F04F89B004460D4616461F46DDE914ABDDE912890620FF21002201923346CDE907ABCDE9058900974B
:40C54000CDE9022104902A4621460020FFF736FE09B0BDE8F08F2DE9FF4105468846F948007801287ED1002D7CD000BF287D0446022C78DAB8F1010F60D128688169284637
:40C580008847C600F04850F82400401CEE4941F82400EE4800688047EB49283141F82400284679F152FBD8B1012833D1E648083050F8241006F140000144E348083040F82F
:40C5C00024100520B6FBF0F081194B31DE48103050F824000144DC48103040F8241019E0D948083050F8241006F12C000144D648083040F824100520B6FBF0F081193331A8
:40C60000D148103050F824000144CF48103040F8241000BF00BF00212846FEF7F0FF28462CF0D2FB074647B1386881683846884718B9C64800688047B8610FE0C248203852
:40C6400050F82400401CC049203941F82400BF4800688047BC49203141F82400A86910B100BF01E02DE00EE0286906464346324629466846EFF78EFB6846A9698847684636
:40C68000EFF79AFB00BF002616E0B149096851F82600AF49096851F8261009688A6829469047012806D1AA49096851F826002946FCF7B9FB701C86B2A64800888642E4DB0F
:40C6C00000BFBDE8FF812DE9F041A048006880470746A1480068B0F1FF3F2AD09E480168384601F013F9054697485C3890ED240AF0EE400ADFED991AB7EE001A00EE105A90
:40C70000B8EE400A01F00CF98F485C3880ED240AD0F8A400A84203D28B485C38C0F8A45089485C38B0F8B200A84202D20320FEF79EFB8948076039F1A1FC2CF0DBFB01208F
:40C7400080490870FDF7F0F8854806681FE07F4800688047074630680268D16988477B48006880478046394601F0D0F8054676485C38B0F8AC00A84208D2306802681169F3
:40C78000884780460222774939F1F3F97668002EDDD16D495C39086A4FF47A7101F041F900286CD069480068804767495C390862002462E0644A4C3A52F82410443252F84F
:40C7C000240001F0A3F860495C3941F8240001F1540050F82410443840F82410143000EB840090ED001AF0EE410A57485C3850F8240001EE100AB8EE411AB0EE410AF2EE5F
:40C80000041AB7EE001A01F08BF84F48383800EB840080ED000A4C4A443A52F82410443252F8240001F072F84749543941F82400454850F82410443840F82410143000EB4F
:40C84000840090ED001AF0EE410A3F48543850F8240001EE100AB8EE411AB0EE410AF2EE041AB7EE001A01F05BF83748303800EB840080ED000A601CC4B2022C9ADB334824
:40C8800000688047074634480168384601F03EF805462D485C3890ED230AF0EE400ADFED2F1AB7EE001A00EE105AB8EE400A01F037F825485C3880ED230AD0F8A000A84223
:40C8C00003D221485C38C0F8A0501F485C38B0F8B000A84202D20420FEF7C9FABDE8F081704770472DE9F04106461D48046831461D4837F189F905E0206801688A69314623
:40C9000090476468002CF7D1184805680AE0284679F1BCF80746E868B04202D12846FFF7D4FB3D46002DF2D1BDE8F08110B51048FFF7D6FF04460F4AAFF259012BF076FDEB
:40C9400010BD000074010010604E0010C4BE1908480100104C0100106C0100100000FA443801001073AD19084442001058010010500100100080000841F25C41095800EE02
:40C98000101AB8EE400ADFEDF70A60EE200AB3EE091A80EE810A70474FF4A351095800EE101AB8EE400ADFEDEF0A60EE200AB3EE091A80EE810A704730B5024600201FE007
:40C9C00001EB810303EBC10402F10C0303EB041393F8CC305B1CDCB201EB810303EBC10502F10C0303EB051383F8CC4001EB810303EBC10402F10C0303EB04131968012002
:40CA0000192916D201EB810303EBC10402F10C0303EB041393F8CC305BB101EB810303EBC10402F10C0303EB041393F8CC30FE2BC6DB30BD30B5034600200024146019297F
:40CA400021D201EB810404EBC10503F10C0404EB051494F8CC40B4B101EB810404EBC10503F10C0404EB05142468B4F1FF3F0AD101EB810404EBC10503F10C0404EB0514E6
:40CA8000241D1460012030BD2DE9FC5F07460D4692461C46DDF83090002001908046002650E0C820B4FBF0F0B0423CD804EB0901701C00EBC00202EB0010B1EBC00F10D906
:40CAC000C820B4FBF0F0B04205D1C820B4FBF0F100FB114B01E04FF0000BCBF1C80000900FE0C820B4FBF0F0B04205D1C820B4FBF0F100FB114B01E04FF0000BA9EB080025
:40CB0000009005EB850202EBC50307F10C0202EB0312121D02EB0B010AEB0800009A77F14CFE00988044C84502D10120019017E005EB850000EBC50107F10C0000EB0110B5
:40CB40000568761C192D0BD205EB850000EBC50107F10C0000EB011090F8CC000028A0D100BF0198BDE8FC9F2DE9F84F0646884614461D46DDE90A794FF0000AB8F1FF3F3B
:40CB800009D03B462A4641463046CDF80090FFF77BFF824610E07CB1306830B1E0194A46294633689847824606E0E1194A46284677F103FE4FF0010A5046BDE8F88F70B5D9
:40CBC0000246002041E001EB810404EBC10502F10C0404EB05142368012001EB810404EBC10502F10C0404EB051494F8CC40641EE5B201EB810404EBC10602F10C0404EBD4
:40CC0000061484F8CC5001EB810404EBC10502F10C0404EB051494F8CC40A4B9851E01EB810404EBC10602F10C0404EB0614256041F25C44A45834B141F25C44A458641EBC
:40CC400041F25C45AC50194600BF19290BD201EB810303EBC10402F10C0303EB041393F8CC30002BAFD170BD2DE9F04704460F4615464FF00008781EC821B0FBF1F000F194
:40CC8000010A4FF000094FF0FF362E6000205AE000EB800101EBC00204F10C0101EB021191F8CC10F1BB00EB800101EBC00204F10C0101EB021191F8CC10491CCAB200EB4D
:40CCC000800101EBC00304F10C0101EB031181F8CC2041F25C410959192911D241F25C410959491C41F25C42115111460A59091D09598A4204D941F25C410A59091D0A51DD
:40CD000009F10109192E16D206EB860101EBC60204F10C0101EB021108604FF0FF3200EB800100E00EE001EBC00304F10C0101EB03110A6000E028600646D14502D14FF08A
:40CD4000010802E0401C1928A2D3B8F1000F06D120462968FFF733FF4FF0FF3028604046BDE8F0870000C8422DE9FC5F04460D4692461E46DDF830900020019080460027E9
:40CD800085E0C820B6FBF0F0B8423CD806EB0901781C00EBC00202EB0010B1EBC00F10D9C820B6FBF0F0B84205D1C820B6FBF0F100FB116B01E04FF0000BCBF1C800009081
:40CDC0000FE0C820B6FBF0F0B84205D1C820B6FBF0F100FB116B01E04FF0000BA9EB080000900AEB080105EB850202EBC50304F10C0202EB0312121D02EB0B00009A77F15B
:40CE0000DCFC00988044C84502D1012001904DE005EB850000EBC50104F10C0000EB01100068192829D305EB850000EBC50104F10C0000EB011201212046FFF715FFE0B1EF
:40CE400005EB850000EBC50104F10C0000EB011090F8CC1005EB850000EBC50204F10C0000EB0210006800EB800202EBC00204F10C0000EB021080F8CC1005EB850000EBD0
:40CE8000C50104F10C0000EB011005687F1C192D0CD205EB850000EBC50104F10C0000EB011090F8CC0000287FF46BAF00BF0198BDE8FC9F2DE9F84F04460F4615461E4604
:40CEC000DDE90A894FF0000AB7F1FF3F09D04346324639462046CDF80090FFF745FF824609E045B1A06830B105EB08014A463046A368984782465046BDE8F88F2DE9FC4700
:40CF00008146884614461D460A9E4FF0000AB8F1190F46D2002E42D0AC421ED24FF0010A002717E001200090A019C31B01AA41464846FFF7A9FD48B101200090A819C31B52
:40CF400001AA41464846FFF70FFF10B94FF0000A27E07F1CB742E5D323E0AC421CD94FF0010A002715E00120E31901AA414600904846FFF789FD40B10120EB1901AA41460B
:40CF800000904846FFF7F0FE10B94FF0000A08E07F1CB742E7D304E04FF0010A01E04FF0010A5046BDE8FC8770B504460025022624B1012C05D0022C09D105E0494D0226D2
:40CFC00005E0494D022602E0484D022600BF00BF25B132462946464838F1CBFD70BD2DE9F84F0646884691469A46DDE90BB44FF0FF30CBF8000000202060706858B300940D
:40D00000D6F804C05246494640460A9BE0470746381E04D0012809D0022814D10FE0206808B1012000E00020054613E0002020605A4630460A99FFF717FE05460AE0002015
:40D040002060002506E00220FFF7AEFF00202060002500BF05E05A4630460A99FFF704FE05462846BDE8F88F10B504464FF0FF302060002084F8CC00C821201D2BF0A8FA19
:40D08000204610BD70B50446002020606060A0601923D022AFF22F0104F10C0078F141FEA0F10C04002141F25C400151001D01510025002615B10020FFF776FF012E02D1D6
:40D0C0000120FFF771FF204670BD704710B50948FFF7D8FF0446084AAFF211012BF0A6F910BD0000FFE904083CEA04087CEA0408E0E90408982000200080000870B504466A
:40D100000025022614B1012C06D102E0FE4D022602E0FE4D022600BF00BF25B132462946FB4838F126FD70BD2DE9F04107460D4614464FF00008002657B320884FF6FF7123
:40D14000884229DA2188491C0904880B2BF0EEFF0646F6B14FF0010800200AE0296851F8201046F8201000212A6842F82010411C88B221888142F1DC208846F8207028687C
:40D1800010B128682BF0CAFF2E602088401C208002E00020FFF7B2FF4046BDE8F0810246082909DCC1F1080302FA03F3DAB250B2C1F10803184100E050B2704702461029F8
:40D1C00009DCC1F1100302FA03F39AB210B2C1F11003184100E010B270470246202907DCC1F120039A401046C1F12003184100E0104670472DE9F74F9046B8F1400F16DC5E
:40D20000C8F14002DDE9009A4846514677F18EF8CDE90001DDE90067C8F1400234463D462046294677F195F806460F4601E0DDE900673046394603B0BDE8F08F2DE9FC4706
:40D2400007460D4616461C46DDF828804FF00009FF202070002F5ED0002E5CDD082E5ADCB8F1000F03D0B8F1010F53D131E04FF001090020207000BF1AE005F00702C2EBD6
:40D28000C00251B200290ADA227800EBD503FB5CC1F1000C43FA0CF31A43227007E0227800EBD503FB5C8B40DBB21A432270401C711E05F007021144012202EBD10181423A
:40D2C000DBD82078C6F10802FF2111410840207020E0701E05F007010844012101EBD00A002008E000EBD5017A5C411CAAEB010101AB5A54401C5045F4D300200090A81903
:40D30000404200F007012346324601A8FFF796FF814600BF00BF4846BDE8FC872DE9FC4707460D4616461C46DDF828804FF000094FF6FF702080002F5FD0002E5DDD102E8F
:40D340005BDCB8F1000F03D0B8F1010F54D132E04FF001090020208000BF1AE005F00702C2EBC00251B200290ADA228800EBD503FB5CC1F1000C43FA0CF31A43228007E018
:40D38000228800EBD503FB5C8B409BB21A432280401C711E05F007021144012202EBD1018142DBD82088C6F110024FF6FF7111410840208020E0701E05F0070108440121A3
:40D3C00001EBD00A002008E000EBD5017A5C411CAAEB010101AB5A54401C5045F4D300200090A819404200F007012346324601A8FFF794FF814600BF00BF4846BDE8FC87C9
:40D400002DE9FE4707460D4616461C46DDF82C804FF000094FF0FF302060002F5ED0002E5CDD202E5ADCB8F1000F03D0B8F1010F53D131E04FF001090020206000BF19E01A
:40D4400005F00702C2EBC00251B200290ADA00EBD503FB5CC1F1000C23FA0CF322681A43226006E000EBD503FB5C8B4022681A432260401C711E05F007021144012202EB50
:40D48000D1018142DCD8C6F120024FF0FF31D14020680840206020E0701E05F007010844012101EBD00A002008E000EBD5017A5C411CAAEB010101AB5A54401C5045F4D316
:40D4C00000200090A819404200F007012346324601A8FFF795FF814600BF00BF4846BDE8FE872DE9F04F8BB080460D4616461C4600200590411E21606160B8F1000F7DD06E
:40D50000002E7BDD402E05E057B1190881B119083AB1190879DC149810B1012874D150E00120059000212160616000272FE005F00700C0EBC70040B204900498002812DA37
:40D5400007EBD50018F800000021049A5242D2B2CDE906102AF0D7FED4E9003218431143C4E9000112E007EBD50018F800900020D4E900AB049A08904846089976F1D6FE75
:40D580004AEA000A4BEA010BC4E900AB7F1C701E05F007010844012101EBD000B842C6D8C6F14002891ED4E900A70A91084609912AF0A9FE0AEA000207EA0103C4E90023A9
:40D5C00022E0701E05F007010844012101EBD007002008E000EBD50118F80120411C791A02AB5A54401CB842F4D300200090A819404200F007012346324600E005E002A8D0
:40D60000FFF76FFF059000BF00BF05980BB0BDE8F08F2DE9FE4705460C4616461F46DDF82C904FF0000A002D7ED0002E7CDD202E7ADCB9F1000F03D0B9F1010F55D155E01D
:40D64000C6F120024FF0FF3020FA02F10F404FF0010A00203FE0C20021FA02F204F007039A4000EBD403EB5C23EA020200EBD403EA54C20021FA02F204F00703C3F108032D
:40D68000DA4000EBD4035B1CEB5C934300EBD402521CAB54C30027FA03F204F007039A40D2B200EBD403EB5C1A4300EBD403EA54C30027FA03F204F00703C3F10803DA4081
:40D6C000D2B200EBD4035B1CEB5C134300EBD402521CAB54401C721ED31702EB53734FF0010C0CEBE3038342B5D831E0701E04F007010844012101EBD008002008E000EBDE
:40D70000D4016A5C411CA8EB010101AB5A54401C4045F4D300200090A019404200F007013B46324601A800E013E0FFF772FF70B1002008E0411CA8EB010101AA515C00EB3D
:40D74000D402A954401C4045F4D34FF0010A00BF00BF5046BDE8FE872DE9F04F99B082460C469346DDE9225600200690BAF1000F7DD0BBF1000F7ADDBBF1400F77DC2498FE
:40D7800010B1012874D189E0CBF140024FF0FF310891084607912AF0B6FD074688463D4006EA0806012006904FF000096BE04FEAC90238464146CDE917872AF0A4FD04F02C
:40D7C0000702CDE9151076F1B1FD09EBD4011AF8011021EA000009EBD4010AF801004FEAC90238464146CDE913872AF08CFD04F00702C2F10802CDE911102AF084FD09EB51
:40D80000D401491C1AF80110814309EBD400401C0AF800104FEAC90228463146CDE90F652AF071FD04F00702CDE90D1076F17EFDC0B209EBD4011AF80110084309EBD401D2
:40D840000AF801004FEAC90228463146CDE90B652AF059FD04F00702C2F10802CDE909102AF051FDC1B209EBD400401C01E049E047E01AF80000084309EBD401491C0AF8E0
:40D88000010009F10109ABF10100C11700EB5171012202EBE101494589D832E0ABF1010004F007010844012101EBD007002008E000EBD4011AF80120411C791A03AB5A543D
:40D8C000401CB842F4D30020CDE90056029004EB0B00404200F007015A4603A8FFF73CFF70B1002008E0411C791A03AA515C00EBD4020AF80210401CB842F4D30120069041
:40D9000000BF00BF069819B0BDE8F08F02468A4201D3501A03E0C1F1FF331344581C7047B0EE402AF0EE602A81EE210AF0EE400AB7EE000AF4EEC00AF1EE10FA04DDB7EE47
:40D94000000AF0EE400A08E0F5EEC00AF1EE10FA03D29FED440AF0EE400AB7EE000A30EE600A20EE220A02EE200A70472DE9F04107460C4615464FF0000800262068002880
:40D9800042D0002010E0216851F82010B94209D14FF001080021226842F820102988491E298004E0411C88B229888142EBDC288828B920682BF0B2FB0020206024E0B8F16C
:40D9C000010F21D1298888002BF0B0FB0646A6B1002100200CE0226852F8202032B1226852F8202046F821204A1C91B2421C90B22A88521C8242EEDC02E00120FFF77EFB63
:40DA000020682BF08BFB26604046BDE8F08170B5044615480068804705462146FFF776FF70BD2DE9F04104460D460F48006880470646A64207D3301BA84201D3012000E0D4
:40DA40000020074609E0C4F1FF303044401CA84201D3012000E0002007463846BDE8F0817047704700000000C4BE190870B50446002502260C2C2BD2DFE804F006090C0FF5
:40DA80001215181B1E212427F84D022620E0F84D02261DE0F74D02261AE0F74D022617E0F64D022614E0F64D002611E0F54D01260EE0F54D01260BE0F44D012608E0F44DED
:40DAC000022605E0F34D012602E0F34D012600BF00BF25B132462946F04838F14AF870BD70B504460D462046F7F7B3FF04466560204670BD2DE9F0410546E948046800279E
:40DB000008E06068A84201D1274605E0204677F1BDFF0446002CF4D100BFB7B908202BF009FB06462946FFF7DBFF0646344644B127462146DA480068F7F7D8FED8490860FB
:40DB400002E00020FFF792FF03E00020FFF78EFF00273846BDE8F081F8B505462C46002000906A462146CE480068F7F747FFCC4908609DF80000012807D134B1264630461E
:40DB8000F7F76AFF07462BF0CDFA9DF80000F8BD70B588B004460D461646E0B28DF81C00200A8DF81D00200C8DF81E000020029003900490059006202B46032207A9CDE9E1
:40DBC00000604FF46A40FEF7F3FB10B9012008B070BD0020FBE70146B04870470146D1F8F40070470146D1F8F80070470146D1F8FC0070470146D1F8000170470146D1F819
:40DC0000040170470146D1F80C01704770B50546002600241EE004EB4401281D00EBC100007DA8B99F480068804704EB4402291D01EBC2010861012104EB4402281D00EB69
:40DC4000C200017504EB4401281D00EBC10603E0601CC4B20A2CDEDB304670BD2DE9F043044607ADE0CD4FF0000CE1B3DAB3002050E000EB400904F1040808EBC90898F8A1
:40DC80001480B8F1000F41D000EB400904F1040808EBC908D8F80C80984537D100EB400904F1040808EBC90898F81580A8452DD100EB400904F1040808EBC90898F81680A5
:40DCC000B04523D100EB400904F1040808EBC908D8F80480884519D100EB400904F1040808EBC90800E017E0D8F80880904506D0082F0BD803F47048B8F5704F06D100EB6D
:40DD0000400904F1040808EBC90C05E000F1010808F0FF000A28ACDB6046BDE8F08370B505465F480468002608E06068A84201D1012605E0204677F1A9FE0446002CF4D1B3
:40DD400000BF304670BD2DE9F04F91B007460E4690461D46DDE91AA900201090002E72D02846FFF7DCFF00286ED1B8F1000F6DD1012010904FF0000BA3E00FA95846FBF7A6
:40DD80001CF9002871D000BF317B0F98027B91426BD100200E900D900C900B9006200A90002009900DA80EA909AA0AABCDE90332CDE905100BA80CA953462A46CDE90091FA
:40DDC000029031460F98FDF735FB00286ED0012802D002286CD16AE00B982B463246CDE900A9029038460F99FFF738FF044664BB00209DF82430DDE90D12CDE90232CDE976
:40DE000004109DF828000021CDE9001028460F9BDDE90B21FEF7CCFA08B33846FFF7F6FE0446A4B1C4F800800F986060A660E56084F815A084F816901A4800688047206150
:40DE40000220207510E04BE148E109E03FE00320FFF70CFED7F8FC00401CC7F8FC0003E0104800688047206126E026E0DAB1190818B2190868B219087CB21908A6B2190808
:40DE8000BDB21908DFB21908F7B2190822B3190845B3190851B3190876B31908B2B1190848020020C4BE190800E001E000BF03E00420FFF7DBFD00BF00BF0BF101001FFA5E
:40DEC00080FBFBF78CF858453FF757AF02E100200E900D900C900B9006200A90002009900DA80EA909AA0AABCDE90332CDE905100BA80CA953462A46CDE90091029031461F
:40DF00004046FDF797FA20B1012835D002287CD1AAE001208DF81C00FF208DF81D008DF81E008DF81F00304677F1A5FE8DF82000E8B28DF82100280A8DF82200280C8DF814
:40DF400023000020029003900490059006204346082207A9CDE900604FF46840FEF728FA48B90520FFF782FDD7F80001401CC7F8000101201090ABE00B982B463246414689
:40DF8000CDE900A902903846FFF768FE0446002C63D19DF82430DDE90D12CDE90232CDE904109DF828004346CDE900602846DDE90B21FEF7FDF948B33846FFF727FE0446E5
:40DFC00094B101201090C4F80080C4F80480A660E56084F815A084F81690F848006880472061022020753EE003208DF81C00FF208DF81D008DF81E008DF81F00304677F192
:40E000003AFE8DF82000E8B201E05DE022E08DF82100280A8DF82200280C8DF823000020029003900490059006204346082207A9CDE900604FF46840FEF7BAF998B90620D7
:40E04000FFF714FDD7F8F400401CC7F8F4000120109008E00120109005E0D8480068804720610120109033E000208DF81C00FF208DF81D008DF81E008DF81F00304677F12D
:40E08000FAFD8DF82000E8B28DF82100280A8DF82200280C8DF823000020029003900490059006204346082207A9CDE900604FF46840FEF77DF930B9D7F80401401CC7F894
:40E0C00004010120109003E00420FFF7CFFC00BF00BF00BF012087F8110101E001201090109811B0BDE8F08F00210160416081606FF07F41C160002101610175FF21417561
:40E100008175704710B50446204635F1D7FD0446AB4820600A231822AFF23301201D77F100FE041F002044F8F40F6060A060E060206135F159FC60610020A0612077607759
:40E14000F43C204610BD10B50446204635F1DDFD0446204610BD70B504462046FFF7F3FF05462AF0DFFF70BD70B50446002515B10120FFF77BFC4FF46E40FFF7BBFC214630
:40E180004FF46A40FCF78EFF70BD7CB504460D46286808226946036928469847012816D129468848D4F8082135F141FC38B90220FFF75CFCD4F8F800401CC4F8F8000120D8
:40E1C00084F81001D4F80C01401CC4F80C017CBD30B50246002036E000EB4004131D03EBC4031B7D73B3B1B100EB4004131D53F834308B420FD000EB4004131D03EBC403F6
:40E200005B688B4207D000EB4004131D03EBC4039B688B4216D1002400EB4005131D03EBC5031C7500EB4005131D43F8354000EB400503EBC5035C6000EB4005131D03EBE1
:40E24000C5039C60401C0A28C6D330BD2DE9F04F8FB006460F4690461D46DDE919A9189C4FF0000B00200E900D900C900B900A9006200990B8F1000F3DD10CA80DA90EAAFF
:40E2800009ABCDE90332CDE905100AA80BA953462246CDE90091029029463846FDF7CAF8F0B1012802D002281ED11AE000209DF83830DDE90C12CDE90232CDE904109DF818
:40E2C000240000213B46CDE900102046DDE90A21FEF76EF808B9012000E00020834609E000BF4FF0010B05E00420FFF7BFFB4FF0010B00BFA5E00CA80DA90EAA09ABCDE96E
:40E300000332CDE905100AA80BA953462246CDE90091029029463846FDF78CF820B1012835D002287ED152E001208DF81C00FF208DF81D008DF81E008DF81F00284677F1EE
:40E340009AFC8DF82000E0B28DF82100200A8DF82200200C8DF823000020029003900490059006203B46082207A9CDE900504FF46840FEF71DF848B90520FFF777FBD6F83F
:40E380000001401CC6F800014FF0010B57E000209DF83830DDE90C12CDE90232CDE904109DF824003B46CDE900502046DDE90A21FDF7FEFF40B9012007E00000C4BE1908DE
:40E3C000B8C91908444200100020834637E000208DF81C00FF208DF81D008DF81E008DF81F00284677F147FC8DF82000E0B28DF82100200A8DF82200200C8DF82300002061
:40E40000029003900490059006203B46082207A9CDE900504FF46840FDF7CAFF40B9D6F8040100E005E0401CC6F804014FF0010B05E00420FFF71AFB4FF0010B00BF00BF87
:40E4400000BF58460FB0BDE8F08F30B589B005460C46207D02286BD1A07D617DE268CDE9002102902846D4E901132268FFF7EEFE10B1002020755DE040F2DC512069FFF7B4
